:020000040800F2
:100000009C5C00201705000885040008090F000803
:10001000890400088B0400088D040008000000001B
:100020000000000000000000000000008F04000835
:1000300091040008000000009304000895040008E3
:1000400097040008990400089B0400089D04000818
:100050009F040008A1040008A3040008A5040008E8
:10006000A7040008A9040008AB040008AD040008B8
:10007000AF040008B1040008B3040008B504000888
:10008000B7040008B9040008BB040008BD04000858
:10009000BF040008C1040008C3040008C504000828
:1000A000C7040008C9040008CB040008CD040008F8
:1000B000CF040008D1040008D3040008D5040008C8
:1000C000D7040008D9040008DB040008DD04000898
:1000D000DF040008E1040008E3040008E504000868
:1000E000E7040008E9040008EB040008ED04000838
:1000F000EF040008F1040008000000000000000008
:100100000000000000000000F3040008F5040008EF
:100110000000000000000000F7040008F9040008D7
:10012000FB040008FD040008FF04000801050008A6
:100130000305000805050008070500080905000873
:100140000B05000800000000000000000000000097
:10015000000000000000000000000000000000009F
:1001600000000000000000000D0500080F05000859
:100170001105000800000000130500080000000041
:08018000000000001505000855
:10020000DECEA5ED02003078463337320000000024
:100210000000000000004457325F313530370000E5
:100220000000000000004170706C69636174696FC8
:100230006E00000000000000000000000000000050
:100240000000000000000404C500DAF7DECEA5EDD2
:100250000200307846333732000000000000000012
:10026000000053504C6174436F6E74726F6C6C6518
:1002700072004170706C69636174696F6E00000098
:10028000000000000000000000000000000000006E
:0802900000000000FE00DAF797
:10029800710B000818000000A90D000803000000F9
:1002A800E5130008060000008D160008090000008C
:1002B800F518000802000000E91900081000000005
:1002C800A51B0008FF000000911E00080C0000009C
:1002D80051200008000000009D21000805000000D2
:1002E800F53F000812000000D54300080A0000008E
:1002F800094800080A000000255000081400000002
:10030800B154000808000000C95B0008070000009D
:100318007162000810000000596600081300000010
:10032800017800081300000061FA000816000000B8
:100338000505010817000000993D01081600000096
:10034800693E010817000000CD4F010815000000A4
:100358002F49072291438D462E492F480A1A06D065
:100368000722914381F30988022282F314882B48DB
:100378002B492C4A00F039F82B482C492C4A00F01C
:1003880034F82C482C492D4A00F02FF82C482D49D8
:100398002D4A00F02AF82D482D492E4A00F025F85C
:1003A8002D482E492E4A00F020F82E482E490022CA
:1003B80000F026F82D482E49091A082903DB0022E7
:1003C8000260043001601F481F49884205D0026856
:1003D800043003B4904703BCF7E700208646EC4698
:1003E80000200021234A9047FEE7884207D0521A8E
:1003F80005D0037801300B700131013AF9D170470B
:10040800884202D002700130FAE770471A487047F4
:100418009C5C00209C6400209C5C002078B0010853
:1004280088010020200200207005000870050008DF
:100438008081010810B101089C6400209C640020A0
:1004480070050008700500087005000870050008B0
:100458007005000870050008808101088081010886
:1004680078B0010820020020505900209C59002033
:100478009C5900204D2E0008FFFFFFFFFEE7FEE716
:10048800FEE7FEE7FEE7FEE7FEE7FEE7FEE7FEE73C
:10049800FEE7FEE7FEE7FEE7FEE7FEE7FEE7FEE72C
:1004A800FEE7FEE7FEE7FEE7FEE7FEE7FEE7FEE71C
:1004B800FEE7FEE7FEE7FEE7FEE7FEE7FEE7FEE70C
:1004C800FEE7FEE7FEE7FEE7FEE7FEE7FEE7FEE7FC
:1004D800FEE7FEE7FEE7FEE7FEE7FEE7FEE7FEE7EC
:1004E800FEE7FEE7FEE7FEE7FEE7FEE7FEE7FEE7DC
:1004F800FEE7FEE7FEE7FEE7FEE7FEE7FEE7FEE7CC
:10050800FEE7FEE7FEE7FEE7FEE7FEE7FEE7134845
:10051800854600F022F84EF68850CEF200000168B9
:1005280051F47001016000BF00BF00BFF1EE100A76
:1005380050F04070E1EE100A4FF0000080F314888C
:100548004EF63C71CEF20001086850F04070086029
:10055800034804490160FFF7FBBE70470080002094
:0805680008ED00E000000008AE
:10057000F8B5044601F024FB06F046F8064640F2C2
:100580002025C2F200054FF000072B689869042C63
:1005900017D8DFE804F0030609101300C0F3400287
:1005A00010E0C0F380120DE000F01102012A14BF28
:1005B0000022012206E0C0F3800203E0C0F34012F3
:1005C00000E03A4672B910F4807F0ED100F01001BD
:1005D000CBB26BB906F018F8801B0528D5D94FF0BF
:1005E0000000F8BD4FF00100F8BD4FF00000F8BD6D
:1005F0004FF00000F8BD00BFF8B540F22024C2F271
:10060000000426684FF0FF35F561FF2B34BF1D460F
:10061000FF254FF000044FF0540767F3090461F31E
:100620008A2465F31744FF2B94BF0023012363F34F
:10063000186462F3596460F34D347460002914BF88
:1006400003200020FFF794FF002814BF2846002055
:10065000F8BD00BF2DE9F04F83B00446894615462A
:10066000002A72D040F22023C2F200031868026808
:1006700042F0010101604FF001004FF000010A4615
:100680000346FFF7B9FF002848D040F22023C2F20A
:100690000003186884624FF00100FFF769FF00282B
:1006A0003FD04FF001004FF0030740F22028C2F284
:1006B000000800E035464FF001010A462B46FFF7DF
:1006C0009BFF824680B3CB462E4600F1FF3202F0FC
:1006D000010101913846FFF74BFF00283AD126E08F
:1006E0003846FFF745FF10B3D8F80020516AA146FD
:1006F00009F8011B06F1FF363846FFF739FF0028DD
:100700004DD114E04FF00400FFF732FF90B14FF0ED
:100710000000002ECED14FF001000DE04FF00000A0
:100720000AE04FF0000007E04FF0000004E04FF057
:10073000000001E04FF0000040F22021C2F2000171
:100740000B684FF000021A6001E04FF0010003B0A7
:10075000BDE8F08FD8F80040636A89F8003009F1ED
:100760000104A14605F1FF360AEB0600A842C9D0F4
:10077000019A002AB4D03846FFF7FAFE0028D6D0F6
:10078000D8F800104B6A8BF8013004F10104A1463F
:1007900006F1FF360AEB0600A842A1D1B2E7D8F86D
:1007A0000030586A607009F10104A14606F1FF3675
:1007B0000AEB0602AA4293D1A4E700BF10B582B0AB
:1007C0001446B9BB4FF0120001A94FF00302FFF726
:1007D00041FF90B39DF804309DF805004FEA0021D9
:1007E00041EA03409DF80620104313F0800F18BF24
:1007F00040F07F4000280FDB14F046FC4FF04042F1
:100800004FF6FF73C4F25F1314F050FF14F016FD9F
:1008100020604FF0000012E014F036FC4FF00002B0
:100820004FF07A5314F08CFE14F008FD20604FF066
:10083000000004E04FF0140001E04FF0180002B097
:1008400010BD00BF08B51F290AD8084611464FF051
:100850000102FFF7FFFE00280CBF1820002008BD92
:100860004FF0140008BD00BF2DE9F04F87B0019193
:100870009A468DF817204FF001038AF800301F299F
:100880005CD840F22021C2F200010C68226842F0DC
:10089000010626600DF117094FF0020B4FF001041D
:1008A00040F22026C2F200065F46CDF810A000E01C
:1008B000D34620464FF000014FF001025B46FFF7A0
:1008C0009BFE8046002849D07CB9CDF8089044466C
:1008D00008F1FF3101F0010203923846FFF748FEAC
:1008E000002855D1DDF810A043E0336801989862E4
:1008F0000BF1FF3BB8F1010808BFDA4613D0E4E77B
:100900003846FFF735FE60B33168A94619F8013B58
:100910008B6204F1FF343846FFF72AFE00285FD1CE
:10092000DDF810A025E04FF00400FFF721FED8B15C
:100930004FF00004BAF1000FBAD106E04FF000000A
:100940008AF800004FF014001FE040F22021C2F2AC
:1009500000010B684FF00000186016E0DDF810A0F1
:1009600007E0DDF810A004E0DDF810A001E0DDF8FC
:1009700010A040F22020C2F2000002684FF00001F7
:1009800011608AF800104FF0180007B0BDE8F08F32
:10099000336899F80000029D05F101059862A946A7
:1009A00008F1FF340BEB040AC8EB0A0A002CBAD09A
:1009B00003990029A4D03846FFF7DAFD0028D6D0E5
:1009C0003368029A507805F101059862A94604F14E
:1009D000FF340BEB040CC8EB0C0A002C90D1A2E7FF
:1009E00030686A7809F101058262A94604F1FF3492
:1009F0000BEB040EC8EB0E0A002C81D193E700BF6D
:100A0000F0B585B00C460B2800F2A1800B2900F24E
:100A1000A18000EB800248F28413C0F6010303EBCF
:100A200082010A7C002A40F0988004EB840148F29D
:100A30008413C0F6010303EB8102117C012940F00D
:100A40008F8048F28413C0F6010300EB800253F854
:100A5000222004EB840153F821309A4240F0838035
:100A6000012A02D0022A33D119E041F21C06C4F255
:100A70000206376847F40011316041F23003C4F2D6
:100A800002031A686FF304121A6040F22025C2F2C2
:100A9000000545F20046C4F200062E6018E041F25F
:100AA0001C05C4F202052E6846F480072F6041F24F
:100AB0003001C4F202010A686FF345120A6040F285
:100AC0002023C2F2000345F60005C4F200051D60B4
:100AD00048F28417C0F6010700EB800007EB8003A3
:100AE000187999684FF0000600964FF001050195BE
:100AF000DA6802924FF003022B4600F0D3FD04EBBC
:100B0000840407EB84042079A16800960195E368CA
:100B100002934FF003022B4600F0C4FD40F2202167
:100B2000C2F20001086848F28012C0F601021368A0
:100B3000036141F2020040F28811C2F2000140F26A
:100B40002422C2F2000208F05DFC28460DE04FF0BE
:100B500000000AE04FF0000007E04FF0000004E062
:100B60004FF0000001E04FF0000005B0F0BD00BF05
:100B700000B583B04FF003004FF0000140F6F932AA
:100B8000C0F6000202F0DAFC4FF0010040F6094125
:100B9000C0F6000140F6E932C0F6000202F0CEFCD9
:100BA0004FF004004FF0050102460FF0D5FB4FF067
:100BB000000000904FF0FF0301934FF00A014FF047
:100BC0000B024FF0010301F087FE4FF004004FF0DD
:100BD0000501FFF715FF48F29420C0F6010005F06B
:100BE000C7FF03B000BD00BF08B519B94FF003003F
:100BF00014F0B6F908BD00BF08B5012903D14FF0C4
:100C0000010014F0ADF908BD08B54FF0070000F081
:100C1000E7FD08BD08B501464FF0080000F0E0FD13
:100C200008BD00BF48F2B023C0F601031A684EF6B3
:100C30000C50CEF200000260FEE700BF08B5FFF7DF
:100C4000F1FF00BF51E8002FBFF35F8F41E80003C1
:100C5000012B3FF4F7AF1046704700BF13461A460A
:100C60002DE9F00F092AC0F00980B1E8F80FA0E8DB
:100C7000F80FA2F10902092ABFF4F7AF4FF00C03F5
:100C800003FB02F21D4B1A44974600F032B800BF36
:100C900000BF00BF00BF0B68036000F02AB800BFB0
:100CA00000BF91E8180080E8180000F022B891E831
:100CB000380080E8380000F01CB891E8780080E83F
:100CC000780000F016B891E8F80080E8F80000F02D
:100CD00010B891E8F80180E8F80100F00AB891E84E
:100CE000F80380E8F80300F004B891E8F80780E81A
:100CF000F807BDE8F00F7047134600008A0C0008A3
:100D000013461A462DE9F00F0B460C460D460E46CB
:100D10000F46884689468A468B46092AC0F00780D6
:100D2000A0E8F80FA2F10902092ABFF4F9AF4FF0C9
:100D3000080303FB02F2144B1A44974600F020B854
:100D400000BF00BF046000F01BB800BF80E83000A7
:100D500000F016B880E8700000F012B880E8F000EB
:100D600000F00EB880E8F00100F00AB880E8F00367
:100D700000F006B880E8F00700F002B880E8F00F55
:100D8000BDE8F00F704713463C0D0008EFF31180EB
:100D90004FF0800181F3118870474FF0000000BFD1
:100DA00080F31188704700BF30B440F20003C0F6F2
:100DB000000340F28812C0F60002D01A4FEAA001E8
:100DC000B1F5C47F04D81346264A9A4201D324E0E1
:100DD000FEE7254D254C601B20F003054FF0000376
:100DE00040F20002C2F2000240F20001C0F600012F
:100DF00005F10400C5F380045D589D5003F1040320
:100E0000834226D109E05C589C5003F104035C58EE
:100E1000D45003F104038342F5D14EF60853CEF2C9
:100E2000000340F20002C2F200021A604FF0B50166
:100E3000CBF26B1145F69C10C2F2000001604EF639
:100E40001453CEF200031A6842F01001196030BC4E
:100E50007047002CD7D05C589C5003F104038342A8
:100E6000D1D1DAE700000008040000088B01000877
:100E700010B4034600283ED002F1100440F20000F6
:100E8000C2F2000040F82430002A0ADA12F10C0FF6
:100E900035DB02F10C024EF61850CEF20000115470
:100EA0002DE04EF20014CEF200040F299CBF090180
:100EB000C9B24EF20043CEF20003D1541146002ACB
:100EC000B8BF02F11F014FEA611004EB80014FF03F
:100ED0001F03C8F200031340002B05DA03F1FF32B1
:100EE00062F01F0303F1010358B24FF0010202FA4E
:100EF00000F30B6003E0002AC8DB024CD5E710BC0E
:100F0000704700BF80E100E01EF0040F0CBFEFF35C
:100F10000880EFF3098020E9F00F00F001B800BF6E
:100F200010B5026845F65013C2F200031A6041681A
:100F3000596082689A60C168D96002691A61416922
:100F4000596182699A61C169D961026A1A62416A0A
:100F50005962826A9A62C16AD962026B1A63416BF2
:100F60005963826B9A63C16BD96300F140001864C6
:100F70004EF62850CEF2000002685A6417F0C0F80E
:100F8000002800F0FB8148F2B420C0F6010017F001
:100F9000BDF84EF62C54CEF200042368002B05DA7F
:100FA00048F2C420C0F6010017F0B0F84EF62C51FC
:100FB000CEF20001086810F0020F05D048F2D420EC
:100FC000C0F6010017F0A2F84EF62852CEF2000249
:100FD0005478002C72D048F2EC20C0F6010017F0D3
:100FE00095F84EF62853CEF20003597811F0010F10
:100FF00005D048F2FC20C0F6010017F087F84EF645
:101000002850CEF20000427802F00204E3B22BB185
:1010100048F21C30C0F6010017F078F84EF628515F
:10102000CEF20001487800F00402D4B22CB148F2AC
:101030004030C0F6010017F069F84EF62853CEF2A2
:101040000003597801F00800C2B22AB148F26430B6
:10105000C0F6010017F05AF84EF62854CEF20004FC
:10106000637803F01001C8B228B148F28430C0F6AA
:10107000010017F04BF84EF62852CEF200025478D9
:1010800004F02003D9B229B148F2A430C0F601001F
:1010900017F03CF84EF62850CEF20000427802F0ED
:1010A0008004E3B253B14EF63851CEF20001096824
:1010B00048F2C430C0F6010017F028F84EF6285068
:1010C000CEF20000428894B2002C5ED048F2E430A8
:1010D000C0F6010017F01AF84EF62853CEF20003BE
:1010E000598811F0010F05D048F2F430C0F6010024
:1010F00017F00CF84EF62850CEF20000428802F0AD
:101100000204A3B22BB148F22040C0F6010016F051
:10111000FDFF4EF62851CEF20001488800F004028F
:1011200094B22CB148F24440C0F6010016F0EEFF34
:101130004EF62853CEF20003598801F0080082B21F
:101140002AB148F28440C0F6010016F0DFFF4EF6E7
:101150002854CEF20004638803F4807188B228B169
:1011600048F2B440C0F6010016F0D0FF4EF6285207
:10117000CEF20002548804F4007399B229B148F207
:10118000D040C0F6010016F0C1FF4EF62850CEF256
:1011900000000278002A63D048F2E840C0F601005F
:1011A00016F0B4FF4EF62854CEF20004237813F064
:1011B000010F05D048F2F840C0F6010016F0A6FF76
:1011C0004EF62851CEF20001087800F00202D4B2A7
:1011D0002CB148F21850C0F6010016F097FF4EF6F9
:1011E0002853CEF20003197801F00800C2B22AB1E8
:1011F00048F23050C0F6010016F088FF4EF6285431
:10120000CEF20004237803F01001C8B228B148F2EE
:101210005450C0F6010016F079FF4EF62852CEF277
:101220000002147804F02003D9B229B148F27850B2
:10123000C0F6010016F06AFF4EF62850CEF200000C
:10124000027802F08004E3B253B14EF63451CEF28C
:101250000001096848F29850C0F6010016F056FFE8
:1012600045F65014C2F20004216A48F2C450C0F698
:10127000010016F04BFF616A48F2D850C0F6010039
:1012800016F044FFA16A48F2EC50C0F6010016F0D7
:101290003DFFE16A48F20060C0F6010016F036FF3B
:1012A000216848F21460C0F6010016F02FFF616853
:1012B00048F22860C0F6010016F028FFA16848F245
:1012C0003C60C0F6010016F021FFE16848F2506072
:1012D000C0F6010016F01AFF216948F26460C0F6FA
:1012E000010016F013FF616948F27860C0F6010052
:1012F00016F00CFFA16948F28C60C0F6010016F0F0
:1013000005FFE16948F2A060C0F6010016F0FEFE9C
:10131000216B48F2B460C0F6010016F0F7FE216CB4
:1013200048F2C860C0F6010016F0F0FE616B48F2AA
:10133000DC60C0F6010016F0E9FEA16B48F2007017
:10134000C0F6010016F0E2FE45F69810C2F2000069
:10135000026848F22470C0F601001146126816F0C7
:10136000D5FE40F2BC73C2F200031A6848F23C702A
:10137000C0F601001146126816F0C8FEFFF75EFCC9
:1013800010BD00BF00B504F039FE002808BF5DF8AD
:1013900004FBEFF30981EFF3118221E9F40F5DF80B
:1013A00004EB1EF0100F08BF21ED108A41F804ED88
:1013B0000B4C2268002A18BF516004F091FE22688D
:1013C000516851F804EB1EF0100F08BFB1EC108A01
:1013D000B1E8F40F82F3118881F3098870470000A7
:1013E0009859002008B541F28530C0F600004FF052
:1013F000FF016FF00102FFF73BFD08BDF8B507469E
:101400000C461E460799089D14F0030F00D0FEE716
:1014100022B1A4EB8500A0F1480401E004F14800EA
:10142000012D01D8A16205E02A46FFF717FCA7EBC2
:101430008507A7624FF0000363604FF01130E06250
:101440004FF0223121634FF0333262634FF0443367
:10145000A3604FF05530E0604FF0663121614FF0EE
:10146000773262614FF08833A3614FF09930E061C9
:101470004FF0AA3121624FF0BB3262624FF0CC33A1
:10148000A363E663069820644FF0807161646FF097
:101490000202226005F11200F8BD00BF62B64EF6EE
:1014A0000453CEF200031A6842F08050186000BF67
:1014B00010B540F20403C4F600031C6848F29471AE
:1014C000C0F601010A6824EA020448F27C72C0F600
:1014D0000102106804431C6040F20443C4F6000398
:1014E0001868496820EA0100526840EA02041C605A
:1014F00040F60403C4F600031868186040F604417F
:10150000C4F600010A680A6041F20404C4F600044B
:101510002368236041F20440C4F6000001680160C2
:1015200040F20C01C4F600010C6848F68402C0F6D3
:101530000102136824EA030448F2AC73C0F6010305
:10154000186804430C6040F20C41C4F600010C68BA
:10155000506824EA0004586804430C6040F60C010B
:10156000C4F600010C68906824EA000498680443FB
:101570000C6040F60C41C4F600010C68D06824EA07
:101580000004D86804430C6041F20C01C4F6000169
:101590000868126920EA02001B6940EA03040C6033
:1015A00041F20C41C4F600010868086048F61C03CB
:1015B000C0F601031A6840F21404C4F60004226065
:1015C000596840F21440C4F6000001604FF0000377
:1015D00040F61402C4F60002136040F61444C4F648
:1015E0000004236041F21401C4F600010B6041F2D3
:1015F0001440C4F60000036040F20001C4F600018C
:101600000C6848F2C472C0F60102136824EA0304AD
:1016100048F69C03C0F60103186804430C6040F2CE
:101620000041C4F600010C68506824EA00045868C0
:1016300004430C6040F60001C4F600010C68906899
:1016400024EA0004986804430C6040F60041C4F6A4
:1016500000010C68D06824EA0004D86820430860C0
:1016600041F20001C4F600010868126920EA020094
:101670001B691843086041F20041C4F600010A6882
:101680000A604FF0010002F0D9FD10BD08B541F22B
:101690001403C4F202031A6842F4FC001860FFF756
:1016A00007FF08BD2DE9F0019DF814709DF8186042
:1016B000079D48F2DC74C0F6010454F820004FEA9C
:1016C0004104FF2F12D0D0F80C8048F6DC0CC0F695
:1016D000010C5CF8277007FA04FC4FF0030707FAC7
:1016E00004F728EA07074CEA0707C760FF2B11D069
:1016F000D0F804C048F63407C0F6010757F8237045
:1017000007FA01F74FF0010303FA01F32CEA030390
:101710003B434360FF2E10D0876848F67403C0F641
:10172000010353F8266006FA04F64FF0030303FAA8
:1017300004F327EA030333438360B5F1FF3F16D078
:101740004FEAD10303F1080350F8236001F00701C9
:101750004FEA810105F00F0505FA01F54FF00F077B
:1017600007FA01F126EA0101294340F82310FF2A74
:1017700010D001684FF0030303FA04F321EA0303D6
:1017800048F63C01C0F6010151F8222002FA04F4A7
:101790001C430460BDE8F001704700BF48F2F473D9
:1017A000C0F6010353F820100A6848F64C03C0F64F
:1017B000010353F820100A4048F6E803C0F601037D
:1017C00053F82000824214BF00200120704700BF60
:1017D00048F2DC73C0F6010353F82000006970473B
:1017E00048F64C03C0F6010353F820307BB139B101
:1017F00048F6B401C0F6010151F82020136070478B
:1018000048F25472C0F6010252F82000036070479B
:1018100040F23023C2F200031B689BB1A8B91A68DA
:101820006FF300021A604FF00000586240F234215A
:10183000C2F2000108801A6842F0010018604FF0FF
:10184000010070474FF0000070474FF000007047F4
:1018500010B483B040F23023C2F200031B6803B31C
:1018600010BB40F23422C2F20002586A148840EAE7
:101870000440019000BF00BF00BF00BF00BF586A16
:10188000148840EA04400090019C00988442ECD106
:10189000DDED017AB8EEE70A81ED000A4FF00100B4
:1018A00004E04FF0000001E04FF0000003B010BC76
:1018B000704700BF40F23023C2F200031B689BB1A7
:1018C000A8B91A686FF300021A6059624FEA114111
:1018D00040F23420C2F2000001801A6842F0010197
:1018E00019604FF0010070474FF0000070474FF053
:1018F0000000704741F22403C4F20203186847F263
:101900000402C4F20002136840F23622C2F200025E
:101910004FF00001117013F0010F03D04FF00400DD
:10192000107032E04FEA106212F0600F07D040F200
:101930003621C2F200014FF020020A7025E002F0C9
:101940000401C9B239B140F23623C2F200034FF0AC
:101950004000187019E0C3F3400343EAD06010F070
:10196000010F07D040F23621C2F200014FF0800291
:101970000A700AE002F01002D1B231B140F236230F
:10198000C2F200034FF00100187041F22401C4F2CA
:1019900002010A6842F080730B6047F20000C4F253
:1019A0000000016841F00802026045F69813C2F297
:1019B0000003186840F23821C2F200010860704745
:1019C00040F23623C2F200031878704708B54FF290
:1019D000AC71C1F6FF714FF00C0214F0AFFD4FF087
:1019E0000C0008BD0000000010B542F20803CEF262
:1019F00004031A6842F01000186041F6A120C0F6F6
:101A000000004FF00F014FF03602FFF731FA41F2BC
:101A10001C01C4F202010C6844F010030B6041F297
:101A20000004C4F2000448F63C72C0F601021068DB
:101A3000206049F22C11C0F60101886913F03CFBCB
:101A400015A3D3E9002313F07BFD4FF000024FF004
:101A50000003C3F6F07313F02DFC13F099FB41F271
:101A60002C03C4F20003188041F22800C4F20000E5
:101A70004FF00002028048F64071C0F6010108688C
:101A800041F20C03C4F200031860228842F0010105
:101A9000218010BDAFF300802D431CEBE2362A3FBE
:101AA000684620F007018D4601B541F21003C4F2EB
:101AB00000034FF000021A6004F0B0FDBDE80140E1
:101AC0008546704770B50446B0F5CC7F2FD940F2FB
:101AD0003233984216D940F26560844215D940F6F7
:101AE000CB418C4214D941F69712944213D943F258
:101AF0002F36B44212D946F25F639C4298BF062546
:101B00000ED90FE04FF001050AE04FF0020507E0A3
:101B10004FF0030504E04FF0040501E04FF0050528
:101B2000072D06D1FFF78AF84FF0070501E04FF0C7
:101B30000005FFF72BF9064604EB84044FEAC400C6
:101B400048F64471C0F6010151F83520B0FBF2F3BC
:101B50009CB2012C05D9B4F5805F04D3FFF76EF871
:101B600001E04FF0020443F20000C4F2000045F22D
:101B70005551016048F64472C0F6010202EBC505FA
:101B80006B6843F20401C4F200010B6043F20802E7
:101B9000C4F2000214604AF6AA2303603046FFF73D
:101BA000FFF870BD08B543F20003C4F200034CF621
:101BB000CC421A604FF0C800FFF784FF08BD00BF99
:101BC00043F20003C4F200034AF6AA221A607047E7
:101BD00010B5044643F20C03C4F20003186810F079
:101BE000010F74D04FF0320005F0D0FF43F20C012A
:101BF000C4F200010A6812F0010F68D04FF0320001
:101C000005F0C4FF43F20C03C4F20003186810F09F
:101C1000010F5CD04FF0320005F0B8FF43F20C0129
:101C2000C4F200010A6812F0010F50D04FF03200E8
:101C300005F0ACFF43F20C03C4F20003186810F087
:101C4000010F44D04FF0320005F0A0FF43F20C0129
:101C5000C4F200010A6812F0010F38D04FF03200D0
:101C600005F094FF43F20C03C4F20003186810F06F
:101C7000010F2CD04FF0320005F088FF43F20C0129
:101C8000C4F200010A6812F0010F20D04FF03200B8
:101C900005F07CFF43F20C03C4F20003186810F057
:101CA000010F14D04FF0320005F070FF43F20C0129
:101CB000C4F200010A6812F0010F08D04FF03200A0
:101CC00005F064FF43F20C03C4F200031B682046D6
:101CD000FFF7F8FE10BD00BF02469CF8043043B188
:101CE000DCF8000040B140F26421C2F2000141F88A
:101CF0002200DCF8000050B940F26423C2F2000375
:101D000053F8220049F64042002808BF10467047A9
:101D10004FF00000704700BF40F20C03C4F6000310
:101D20001A681A6040F20C40C4F6000001680160B5
:101D300040F60C03C4F600031A681A6040F60C4023
:101D4000C4F600000168016041F20C03C4F6000310
:101D50001A681A6041F20C40C4F600000168016084
:101D600040F20003C4F600031A681A6040F2004013
:101D7000C4F600000168016040F60003C4F60003E9
:101D80001A681A6040F60040C4F60000016801605D
:101D900041F20003C4F600031A681A6041F20040E1
:101DA000C4F6000001680160704700BF38B50D46F9
:101DB000044600B3132801D9FEF740FF49F22C1363
:101DC000C0F6010353F8240055B1B0FBF5F14FEA1A
:101DD000114202F10103B0FBF3F0B0FBF5F502E0B4
:101DE0004FF000052A4649F2DC01C0F6010151F826
:101DF00024309A62DD6238BD30B583B000918DF831
:101E000004200346B0B94FF000042046FFF780FFDE
:101E100038B1EC462046FFF75FFF01462046FFF74A
:101E2000C5FF04F1010425462046FFF771FF002895
:101E300029D020E048F68072C0F6010212F8200096
:101E4000012816D148F68071C0F6010101EB830428
:101E5000637803EB830048F61012C0F6010252F8D3
:101E60002040EC462046FFF737FF01462046FFF7AB
:101E70009DFF03B030BDEC462046FFF72DFF014625
:101E80002046FFF793FF04F10104142CBDD1F0E7C5
:101E900070B54FF0000001460246FFF7ADFF49F272
:101EA000DC05C0F601054FF0010448F69076C0F657
:101EB00001062046FFF72CFFB0B112E02046FFF7E5
:101EC00027FF10B168683168016004F10104204601
:101ED00005F10405FFF71CFF70B10AE0FFF71CFFD6
:101EE00070BD6B6832681A6004F1010405F10405E5
:101EF000E4E76B6832681A6004F1010405F1040537
:101F0000142CDBD1EAE700BF38B52DED028B054676
:101F100041F21803C4F20203186810F4007F57D18D
:101F200040F23C20C2F2000048F68871C0F6010180
:101F300003F0E2FA41F20404C4F2020422684FF012
:101F4000020161F38F32226041F21803C4F20203EE
:101F5000186840F400741C601A6842F001011960AE
:101F600042F20443C4F201034FF00000186048F647
:101F70008C74C0F60104226842F20C41C4F20101E3
:101F80000A6048F67C73C0F60103186842F21044F8
:101F9000C4F20104206048F68072C0F601021168A4
:101FA00042F22C43C4F20103196048F68470C0F673
:101FB0000100046842F20841C4F201010C600A68A1
:101FC00042F004030B600846046814F0040FFBD1D0
:101FD00040F23C20C2F200004FF0000103F0A4FAEE
:101FE00042F20044C4F20104616B4FF0110262F34B
:101FF00004016163E36C4FF0050005F0C7FDA368C1
:1020000043F48000A06021460A6812F0020FFBD062
:1020100042F20043C4F2010393ED138A40F23C20E4
:10202000C2F2000003F08EFB4FF2BA70C1F6FF70EF
:10203000018807EE901AB8EE670AF8EE480A80EEBB
:10204000208A85ED008A4FF00100BDEC028B38BD7F
:1020500008B572B648F69873C0F601031A684EF6D2
:102060003470CEF20000026048F6A871C0F601019B
:102070000A684EF68853CEF200031A6048F6A47040
:10208000C0F60100016842F20802CEF204021160BB
:1020900048F69473C0F60103186842F20C01CEF2C0
:1020A0000401086041F20003C4F202031A6842F41A
:1020B0008030186019460B6813F4003FFBD048F6D7
:1020C000AC72C0F60102106841F20401C4F20201D0
:1020D000086048F6A073C0F601031A6842F20000D7
:1020E000C4F20200026041F20001C4F202010B6876
:1020F00043F080720A600846016811F0007FFBD04F
:1021000041F20403C4F202031A684FF0020060F3C4
:1021100001021A6019460B6803F00C02082AFAD172
:1021200041F21800C4F20200016841F001030360AB
:1021300042F21C02C4F20202106848F27421C0F696
:1021400001010A6848F69C73C0F601031B68504001
:10215000184222D048F27421C0F60101087800F03C
:102160000401C8B2C8B942F21C01C4F202010868F5
:1021700020EA0300134018434FF60003C1F6FF7333
:102180005A68D1B261F317405B68C3F3074262F348
:102190001F604FF0FF3100F0A3F908BD41F21403B6
:1021A000C4F202031A6842F001001860704700BFD1
:1021B00070B41646002A47D040F20802C4F2020268
:1021C000146814F0010F06D040F20C05C4F20205A9
:1021D0002A68002AFCD140F20804C4F202044FF03D
:1021E0000005256048F6B472C0F60102156840F299
:1021F0000402C4F20202156040F21002C4F20202AC
:10220000116040F21401C4F20201086040F20C00B7
:10221000C4F20200066048F6B072C0F6010211680E
:102220002160206840F0010222606BB140F20C0195
:10223000C4F202010B68002BFCD140F20800C4F28A
:1022400002004FF00002026070BC704742F21003BF
:10225000C4F20203186810F0800F0DD042F204019E
:10226000C4F2020140F22312C4F267520A6048F637
:10227000AB13CCF6EF530B6042F21000C4F2020035
:10228000016801F08002002A14BF0220002070477C
:1022900042F21003C4F20203186810F0800F07D155
:1022A00042F21001C4F202010A6842F080030B609E
:1022B000704700BF40F20003C0F60003984208D305
:1022C00040F20001C0F6040188422CBF002001202A
:1022D00070474FF0000070472DE9F04706460D4665
:1022E000FFF7E8FF002855D02846FFF7E3FF002856
:1022F00053D0AE4254D8FEF749FD8246FFF7A6FF01
:102300000446B8BB41F28830FFF762FC48F6BC7364
:10231000C0F601031A6842F21000C4F20200026023
:1023200042F21409C4F20209804642F20C07C4F2D8
:102330000207FFF745FCC9F80060D8F8001041F02B
:102340004003C8F8003006F500663A6812F0010F45
:10235000FBD1386810F0200F0AD0396841F0200313
:102360003B60B542E5D24FF06400FFF731FC01E07D
:102370004FF0020448F6C072C0F60102106842F243
:102380001001C4F202010860FFF782FF5046FEF719
:1023900007FD07E04FF0020404E04FF0020401E003
:1023A0004FF002042046BDE8F08700BFF8B50746AD
:1023B0000C4616460846FFF77DFF002800F089808E
:1023C00006F1FF302018FFF775FF002800F0848029
:1023D00040F2CC73C2F2000353E8002F02F1010275
:1023E00043E800210129F7D0FFF730FF0546002818
:1023F0004BD148F6C471C0F601010A6842F21000E0
:10240000C4F20200026014F0010F09D037F8013C59
:1024100024F8013C04F1010407F1010706F1FF363D
:10242000012E25D904F1020207F10200A6F1020CE7
:102430004FEA5C0C04F1040E0EEB4C0E42F20C0160
:10244000C4F202010B6813F0010FFBD130F8023C1B
:1024500022F8023C02F1020200F102007245F1D1C1
:102460000CF101024FEA420024183F1806F0010661
:102470000EB13978218048F6C874C0F6010422688C
:1024800042F21003C4F202031A60FFF701FF40F2A8
:10249000CC73C2F2000353E8002FA2F1010243E81B
:1024A0000024012CF7D053E8002FB2F1004F0DD1DA
:1024B0004FF0000243E80024012CF4D04EF6045003
:1024C000CEF20000016841F080510160BFF32F8F10
:1024D00004E04FF0020501E04FF002052846F8BD88
:1024E00030B585B004460D4668464FF0FF014FF009
:1024F000100214F047F8E3B203F00402D0B200284F
:1025000040F0B58003F00201CBB223B14FF01100CF
:102510008DF8000003E06FF055028DF80020C4F341
:1025200007218DF80210C4F307438DF804304FEAF9
:1025300014648DF806408DF80850FEF727FC054618
:10254000FFF784FE002840F0868042F20800C4F2C3
:10255000020040F22312C4F26752026048F6AB1147
:10256000CCF6EF51016042F21003C4F202031C6882
:1025700014F4007F6FD048F6CC70C0F601000268FA
:1025800042F21001C4F202010A600B6843F04004F9
:102590000C6042F20C00C4F20200026812F0010F5B
:1025A000FBD142F21003C4F202034FF000011960A4
:1025B00042F20804C4F2020440F22310C4F267504D
:1025C000206048F6AB12CCF6EF5222601B6813F481
:1025D000007F40D048F6B871C0F601010C6842F2A5
:1025E0001000C4F20200046042F20802C4F20202C7
:1025F00040F22313C4F26753136048F6AB11CCF6D4
:10260000EF511160046814F4007F24D04FF60003EA
:10261000C1F6FF7303F11000834213D24FF0100490
:102620004FF00001184642F20C02C4F202023DF8DB
:1026300001300B52136813F0010FFBD101F10201BD
:10264000A142F4D142F21004C4F202044FF000019E
:102650002160FFF71DFE4FF0000442F21000C4F2AB
:10266000020004602846FEF79BFB204601E04FF085
:10267000020005B030BD00BF40F2B423C2F2000337
:102680001868704770B48568C668446806FB0540E2
:102690004118196040F2B420C2F200000068814283
:1026A0000CD2521890420CD340F2B820C2F2000073
:1026B0000268891819604FF0010004E04FF0000033
:1026C00001E04FF0000070BC704700BF2DE9F04101
:1026D0000546FFF775FA4FF01E0440F2BC26C2F221
:1026E00000064FF000084FF0010733689869042D89
:1026F00017D8DFE805F0030609101300C0F3400205
:1027000010E0C0F380120DE000F01102012A14BFA6
:102710000022012206E0C0F3800203E0C0F3401271
:1027200000E04246AAB9C0F3072111F0010F14D10D
:1027300000F01003D8B2A0B901F00202D1B2A1B9E1
:10274000384605F023FA013CCFD14FF00000BDE838
:10275000F0814FF00100BDE8F0814FF00000BDE8CE
:10276000F0814FF00000BDE8F0814FF00000BDE8BF
:10277000F08100BFF8B540F2BC24C2F20004256825
:102780004FF0FF36EE61FF2B34BF1E46FF264FF0A1
:1027900000044FF0A00767F3090461F38A2466F38D
:1027A0001744FF2B94BF0023012363F3186462F3E3
:1027B00059646C6060F34D346C60002914BF0320D1
:1027C0000020FFF783FF002814BF30460020F8BD2B
:1027D0002DE9F04180460F4616461D46FFF7CAFF19
:1027E0000446002874D14FF0050003F093FA4046E8
:1027F000394632462B46FFF7BDFF0446002867D115
:102800004FF0050003F086FA4046394632462B4623
:10281000FFF7B0FF044600285AD14FF0050003F03F
:1028200079FA4046394632462B46FFF7A3FF044665
:1028300000284DD14FF0050003F06CFA40463946B0
:1028400032462B46FFF796FF0446002840D14FF052
:10285000050003F05FFA4046394632462B46FFF743
:1028600089FF0446002833D14FF0050003F052FAE7
:102870004046394632462B46FFF77CFF044638BBBC
:102880004FF0050003F046FA4046394632462B46E3
:10289000FFF770FF0446D8B94FF0050003F03AFA8D
:1028A0004046394632462B46FFF764FF044678B966
:1028B0004FF0050003F02EFA4046394632462B46CB
:1028C000FFF758FF044618B94FF0050003F022FA4D
:1028D0002046BDE8F08100BF2DE9F04184B01446E8
:1028E0001D460B2900F2A4800B2A00F2A48001EB04
:1028F000810248F6E073C0F6010303EB8202137C09
:10290000002B40F09B8004EB840248F6E073C0F695
:10291000010303EB8202137C012B40F0928048F606
:10292000E073C0F6010301EB810653F8262004EBA7
:10293000840653F826309A4240F0868040F2C02741
:10294000C2F200073870012A02D0022A23D111E016
:1029500041F21C00C4F20200066846F40012026054
:1029600040F2BC23C2F2000345F20047C4F2000764
:102970001F6010E041F21C00C4F20200066846F439
:102980008002026040F2BC23C2F2000345F6000759
:10299000C4F200071F6048F6E078C0F6010801EBBA
:1029A000810108EB8102107991684FF000060096D2
:1029B0004FF001070197D36802934FF003023346AB
:1029C000FEF770FE04EB840408EB84042079A16810
:1029D00000960197E26802924FF003023B46FEF731
:1029E00061FE40F2BC20C2F2000001680E6048F6B1
:1029F000D073C0F601031A680A6145B340F2B820EB
:102A0000C2F200000A99016040F2B422C2F2000250
:102A10000B9B136040F2C420C2F2000048F6D47150
:102A2000C0F601012A46334606F0B2FD384610E0F2
:102A30004FF000000DE04FF000000AE04FF0000002
:102A400007E04FF0000004E04FF0000001E04FF01D
:102A5000010004B0BDE8F0812DE9F04F83B091464C
:102A60000D46002900F09C8040F2BC23C2F2000316
:102A700019680A6842F001040C60044640F2C02A5A
:102A8000C2F2000A49F2D00BC0F6010B40F2BC279B
:102A9000C2F200079AF800005BF8206006F1FF33ED
:102AA00009EA0301731A00F1FF3202F0FF00012866
:102AB0008CBF012602264FF001004FF000010246B4
:102AC000AB4294BFF3187319FFF782FE0646002845
:102AD00052D09AF8001001F1FF33DAB2012A0BD874
:102AE0003868C9F30721816206F1FF364FF0020012
:102AF000FFF7ECFD002842D03B685FFA89F29A624A
:102B0000013E26D04FF0020806F1FF3000F001012F
:102B100001914046FFF7DAFD002846D132E04046F9
:102B2000FFF7D4FD70B334B1386814F8012B6FEAA5
:102B30000201816203E039684FF0FF038B6206F106
:102B4000FF3605F1FF354046FFF7C0FD002855D19F
:102B500018E09AF800005BF820108944C1F10002E7
:102B600009EA02094FF00400FFF7B0FD68B1002D3B
:102B700090D14FF001000AE04FF0000007E04FF065
:102B8000000004E04FF0000001E04FF0000040F2D0
:102B9000BC23C2F2000319684FF000020A6001E092
:102BA0004FF0010003B0BDE8F08F24B93B684FF04F
:102BB000FF029A6205E0386814F8011B6FEA01030E
:102BC000836205F1FF35013EC3D0019A002AA6D0E9
:102BD0004046FFF77BFD0028D4D024B938684FF079
:102BE000FF01816205E03B6814F8012B6FEA0200E7
:102BF000986205F1FF35013E91D1AAE724B93B68FF
:102C00004FF0FF00986205E0396814F8012B6FEA75
:102C100002038B6205F1FF35013E80D199E700BFC9
:102C200030B583B015461C461A4601ABFFF72AFDA6
:102C300048B128462146019AFFF70EFF00280CBF35
:102C40001820002001E04FF01F0003B030BD00BF8E
:102C50002DE9F04F83B0044689461646002A00F05D
:102C60009E8040F2C023C2F20003187800F1FF31C9
:102C700001F0FF0340F2BC22C2F2000211680868B2
:102C800040F001020A604FF001004FF000010A46D7
:102C900083428CBF03460223FFF79AFD002864D0CD
:102CA00040F2C023C2F20003197801F1FF30C2B232
:102CB000012A0DD840F2BC23C2F200031968C4F304
:102CC000072088624FF00200FFF700FD00284FD078
:102CD00040F2BC22C2F200021368E4B29C624FF0E0
:102CE0000100FFF7F3FC002845D04FF001004FF042
:102CF000030740F2BC28C2F2000800E02E464FF065
:102D000001010A463346FFF735FD8246002835D0DB
:102D1000CB46354600F1FF3101F001000190384605
:102D2000FFF7D4FC00283FD12BE03846FFF7CEFC5C
:102D300038B3D8F80020536A6FEA0301A14609F8B6
:102D4000011B05F1FF353846FFF7C0FC002854D1C0
:102D500017E04FF00400FFF7B9FCA8B14FF00000F6
:102D6000002DCBD14FF0010010E04FF000000DE03E
:102D70004FF000000AE04FF0000007E04FF00000C5
:102D800004E04FF0000001E04FF0000040F2BC22F0
:102D9000C2F2000213684FF00001196001E04FF029
:102DA000010003B0BDE8F08FD8F80040626A6FEA16
:102DB000020389F8003009F10104A14606F1FF354C
:102DC0000AEB0501B142C4D001980028ADD03846C5
:102DD000FFF77CFC0028D4D0D8F80020536A6FEAB3
:102DE00003018BF8011004F10104A14605F1FF3540
:102DF0000AEB0500B04298D1ABE7D8F80000426A70
:102E00006FEA0203637009F10104A14605F1FF3581
:102E10000AEB0501B14288D19BE700BF30B583B012
:102E200015461C461A4601ABFFF72CFC48B1019829
:102E300029462246FFF70CFF00280CBF182000206F
:102E400001E04FF01F0003B030BD00BF08B545F6EC
:102E50009C10C2F2000045F69C42C2F20002131A16
:102E60004FF0FF314FEAA302FDF74AFF01F03EFFAA
:102E7000FEF714FB4FF0000008BD00BFBFF36F8FDB
:102E8000704700BF49F2C413C0F60103185C00EBA1
:102E9000400149F28822C0F6010252F821305B6AF3
:102EA000704700BF38B549F2C413C0F601031B5C7C
:102EB00003EBC30440F2D422C2F2000202EB84020C
:102EC00082F8211014693CB140F2D425C2F2000509
:102ED0001346D2699B69A04738BD00BFF8B50646C6
:102EE0000F4649F2C413C0F601031D5C05EBC50093
:102EF00040F2D424C2F2000404EB8004D4F810C0E1
:102F0000BCF1000F07D0E2698A4204D030464FF08E
:102F10000001A369E047E76163695BB105EBC500A8
:102F200040F2D422C2F2000202EB8002304639465F
:102F30009269984794F8201079B127696FB105EB31
:102F4000C50540F2D423C2F2000303EB85053046E9
:102F500094F82110E269AB69B847F8BD49F2C4138F
:102F6000C0F60103185C00EB400149F28822C0F66C
:102F7000010252F82130186840F080011960704752
:102F800049F2C413C0F60103185C00EB400149F29A
:102F90008822C0F6010252F82130986940F00201FF
:102FA00099611A6842F0800018607047F8B50446CD
:102FB00000EB400249F28823C0F6010353F8226077
:102FC000F569356205F0010215F0020F1CBF42F0F1
:102FD0000202D2B215F0040F18BF42F0080215F039
:102FE000080F18BF42F0040215F4807F05D0706806
:102FF00010F4804F18BF42F0100215F0200F00D1DE
:10300000E2B104EBC40140F2D427C2F2000707EB9F
:1030100081039F688FB1716A04EBC40040F2D4232E
:10302000C2F2000303EB800349F26820C0F60100FE
:10303000005DC9B29B69B84700E0736A326812F05C
:10304000800F1CD015F0800F19D031686FF3C711B5
:10305000316004EBC40040F2D423C2F2000353F801
:10306000203063B140F2D422C2F2000202EB8002AF
:1030700049F26820C0F60100005D9169984715F09B
:10308000400F17D004EBC40140F2D423C2F2000376
:1030900003EB810253686BB1084640F2D421C2F2BF
:1030A000000101EB800249F26820C0F60100005DDA
:1030B00091699847F8BD00BF684620F007018D462A
:1030C00001B54FF00300FFF771FFBDE801408546F1
:1030D000704700BF684620F007018D4601B54FF0EC
:1030E0000200FFF763FFBDE801408546704700BF5F
:1030F000684620F007018D4601B54FF00100FFF74B
:1031000055FFBDE801408546704700BF10B582B04D
:103110008DF8071049F2C413C0F60103185C00EBE8
:10312000400249F28821C0F6010151F82240E369CA
:1031300013F0800FFBD002A911F8012DA26200EB61
:10314000C00040F2D424C2F2000404EB8004608C7E
:103150004FF0010204F032FD608404F1200402B05B
:1031600010BD00BF70B582B08DF8071049F2C413CE
:10317000C0F60103185C00EB400149F28822C0F65A
:10318000010252F82140E56915F0800F1DBF9DF83E
:103190000750A5620126002600EBC00340F2D420B0
:1031A000C2F2000000EB8305688C0DF107014FF0BF
:1031B000010204F003FD688405F12005216841F057
:1031C00080022260304602B070BD00BF2DE9F0439E
:1031D00085B016461F4649F2C413C0F601031C5CB5
:1031E00004EB440249F28825C0F6010555F8224057
:1031F00049F28423C0F60103185C00EB400249F257
:103200007C15C0F6010505EBC2058846002956D09D
:10321000002E57D0287B29699DF8342000924FF06A
:10322000010301936A6902924FF003023B46FEF7E5
:1032300039FA40F2CC73C2F2000353E8002F02F1D6
:10324000010243E800210129F7D021684FF0000076
:103250002060012E14BF00260126626866F3CF327B
:10326000626049F28020C0F601000268B8F1010FE7
:1032700014BF4FF000084FF0010868F3C302A260CA
:10328000216053E8002FA2F1010243E80024012C41
:10329000F7D053E8002FB2F1004F0DD14FF00002EC
:1032A00043E80024012CF4D04EF60450CEF2000086
:1032B000016841F080510160BFF32F8F17E04FF09C
:1032C000010901E04FF00009287869689DF8303065
:1032D00000934FF001020192AB6802934FF003029A
:1032E0003B46FEF7DFF9B9F1000FA2D092E705B037
:1032F000BDE8F0832DE9F84F81468B4690461E4687
:103300009DF828A049F2C413C0F601031D5C05EB2B
:10331000450249F28820C0F6010050F822409DF88D
:103320002C70012F14BF00270127082E06D0072E6E
:1033300002D1B8F1000F01D1FDF780FC0AF1FF3195
:10334000CBB2012B01D9FDF779FC49F2B822C0F6C6
:10335000010252F82500B0FBFBF1E1604FF02002C2
:1033600067F38612BAF1010F04D0002F0CBF0223BD
:10337000002301E04FF0000363F30D3267F38E3258
:103380006068C0F3C03363F3CF3262604FF06D0109
:10339000B8F1020F14BF0023012363F3492118F190
:1033A000000818BF4FF0010868F38A21082E18BFE3
:1033B0004FF0000868F30C3121604846FFF762FDCA
:1033C000BDE8F88F2DE9F843054649F2C413C0F66D
:1033D0000103185C00EBC00240F2D424C2F20004E6
:1033E00004EB820449F28821C0F6010100EB40069B
:1033F0004FEA860301EB030851F80390FDF7C6FC82
:10340000064694F82000B8B14FF00007C9F80070E4
:103410003846394698F90420FDF72AFD28463946F2
:10342000FFF740FDE3681BB12846E169A2699847B0
:103430004FF0000284F820203046FDF7B1FCBDE8D3
:10344000F88300BF2DE9F04F85B005468B469246C4
:10345000994649F2C413C0F601031E5C40F2D42819
:10346000C2F2000806EBC6074FEA870708EB07041D
:1034700006EB460049F28821C0F6010101EB800607
:10348000FDF784FC039041F21C03C4F202031868A8
:1034900049F2D011C0F601010A6820EA020E49F291
:1034A000C812C0F6010210684EEA0000186041F22E
:1034B0001803C4F202031868496820EA0100526840
:1034C0001043186049F26C21C0F6010105EB850339
:1034D000C818C95C4278837890F803C0CDF800C062
:1034E000007901902846FFF771FE9DF83820009280
:1034F0009DF83C1001912846594652464B46FFF72D
:10350000F9FE109B48F807301298A060119A62608B
:103510001399E160149BA361B0684FF00F0196F915
:103520000420FDF7A5FC4FF0010084F8200003986B
:10353000FDF736FC05B0BDE8F08F00BF49F2C413BB
:10354000C0F60103185C00EBC00340F2D420C2F2C5
:10355000000000EB830319615A61704749F284232C
:10356000C0F60103185C00EB400149F2D812C0F626
:10357000010202EB01107047032812D849F2C4136C
:10358000C0F60103185C00EBC00140F2D422C2F285
:10359000000202EB81034FF6FF7058844FF00100E8
:1035A00070474FF00000704703280ED849F2C4134B
:1035B000C0F60103185C00EBC00140F2D422C2F255
:1035C000000202EB8103588C70474FF000007047F7
:1035D000F8B54FF04C0404FB00F440F6C821C2F2E9
:1035E0000001621846F20003C4F2000303EB00136B
:1035F00045F60045C4F2000505EB80006558002D36
:1036000074D094680CB1968801E04FF000061F68F2
:1036100066F30F071F6059686FF309015960D1689D
:1036200019B15668A719BFB201E04FF000079E68B4
:1036300067F30F069E603E2994BF00270127DE68CE
:1036400067F3CF36DE60DE6816F4004F1DBF4F090A
:1036500007F1FF3707F01F07C1F34407DE6867F380
:103660008E26DE600368166A66F303032E7A49F23B
:10367000D025C0F6010555F8265065F34A236FF3AF
:103680000823C3F30115002C14BF022400246C404E
:1036900064F30513C3F30134002914BF032100218F
:1036A000614061F30D336FF3CF336FF3C7130360E2
:1036B00040F6C950C2F200000378191F18BF01215B
:1036C00051624FF0010090624FF00003D362136328
:1036D000536340F27A30C2F20000018801F1010127
:1036E0008BB2038002F1100000F050FDF8BD00BF66
:1036F000F8B545F64443C4F200031C6840F27C3040
:10370000C2F20000028802F1010291B2018014F4B9
:10371000004F00F0948045F64445C4F200052E6841
:1037200006F00F0340F6C827C2F200074FF04C0026
:1037300000FB037545F60042C4F2000202EB83076A
:1037400040F27E31C2F200010E8806F10106B0B2ED
:10375000088052F82360C6F3C032EB6A1343EB6271
:10376000C6F3C021286B08432863C6F3C0126B6BF5
:1037700013436B63C6F3072101F00800C2B25AB1CC
:103780004FF00003EB6340F28A31C2F20001088877
:1037900000F1010082B20A80EB6B93B126F07F0149
:1037A000C8B270B140F28033C2F200031A8802F14D
:1037B000010291B219804FF000016963286A03F099
:1037C0003BFCE86A18B96B6B0BB92A6B7AB340F211
:1037D0008231C2F20001088800F1010083B20B803F
:1037E00005F1100000F0D2FC08BB40F28E32C2F2AC
:1037F0000002108840F27C31C2F200010B8840F2D6
:103800006432C2F2000222F8103000F1010080B2EE
:10381000092805D840F28E31C2F20001088006E086
:1038200040F28E33C2F200034FF000021A8049F2D8
:10383000C820C0F60100016826EA01063E6014F4C3
:10384000806F16D040F28433C2F200031A8802F16E
:10385000010290B2188040F6A551C2F200014FF06B
:1038600001030B7040F69C52C2F20002106802F095
:10387000BBF814F4006F25D040F28630C2F200008D
:10388000018801F101018BB2038045F64040C4F28A
:103890000000026842F00801016040F62853C2F2BD
:1038A00000034FF00100187040F6C851C2F2000149
:1038B0004FF000020A7040F69C53C2F200031868F1
:1038C00002F092F814F4805F25D040F28830C2F202
:1038D0000000018801F101018AB2028045F64043EF
:1038E000C4F2000318686FF3C300186040F6285153
:1038F000C2F200014FF000020A7040F6C853C2F253
:1039000000034FF00100187040F69C51C2F2000114
:10391000086802F069F86FEA040445F64442C4F20C
:1039200000021460F8BD00BF684620F007018D4614
:1039300089B500AFFFF7DCFEBD46BDE8894085468E
:10394000704700BF45F64043C4F200031A6860F3B5
:10395000CF321A60704700BF40F6CC53C2F200036A
:103960001A5C45F60040C4F2000049B150F822004C
:10397000C0F3011149F2E823C0F60103585C704717
:1039800050F82210C1F3013349F2E822C0F60102D7
:10399000D05C704740F6CC53C2F200031A7845F66B
:1039A0000043C4F2000353F8221049F2EC20C0F6A1
:1039B0000100006821EA000181F0100141F48070EB
:1039C00043F8220040F28C33C2F200031A8802F15D
:1039D000010291B2198070472DE9F00340F6CC53F3
:1039E000C2F20003185C45F6004CC4F2000C0CEB6C
:1039F000800C4FEA001346F20007C4F2000703EB05
:103A00000708D85983B207EB4307012A31D901F1DE
:103A10000204A2F102094FEA590901F1040606EB7A
:103A20004906351BA5F10205C5F3400534F8024CE3
:103A3000384620F8044B01F10403B34238D10FE0BB
:103A400033F8025C044624F8045B03F1020333F804
:103A5000025C858004F1040003F10203B342EFD15C
:103A600002F0010009F1010901EB490107EB8907A7
:103A700000E0104608B109783980D8F8040062F3F4
:103A80000900C8F80400DCF8003049F2F022C0F662
:103A90000102116823EA01000346C0F3011282F01B
:103AA000030161F30513CCF80030BDE8F003704763
:103AB000002DC5D033F8024C20F8044B03F102036B
:103AC000B342BDD1CCE700BF2DE9F00140F6CC53A5
:103AD000C2F200031C5C45F6004CC4F2000C0CEB77
:103AE000840C46F20000C4F2000000EB0414A3684A
:103AF0009BB200EB4300E3684FEA83534FEA9353D2
:103B0000934204D2E2684FEA82534FEA9352012A69
:103B100031D901F10203A2F102084FEA580801F17C
:103B2000040707EB4807FD1AA5F10205C5F3400697
:103B3000044634F8045B23F8025C01F10403BB4241
:103B400034D10FE0254635F8046B23F8026C03F1FD
:103B50000203A48823F8024C05F1040403F10203D4
:103B6000BB42EFD102F0010308F1010801EB48016B
:103B700000EB880000E013460BB103880B70DCF803
:103B8000000049F2E421C0F601010B6820EA0300BD
:103B90000346C0F3013181F0030060F30D339BB2A3
:103BA000CCF800301046BDE8F0017047002EC9D0B7
:103BB00034F8045B23F8025C03F10203BB42C1D179
:103BC000D0E700BF08B545F64043C4F200031A68C9
:103BD0006FF3C3021A604FF00000FFF7F9FC4FF0DB
:103BE0000100FFF7F5FC4FF00200FFF7F1FC4FF08A
:103BF0000300FFF7EDFC4FF00400FFF7E9FC4FF086
:103C00000500FFF7E5FC4FF00600FFF7E1FC4FF081
:103C10000700FFF7DDFC49F2E020C0F60100016873
:103C200045F64C43C4F20003196008BD2DE9F0418C
:103C3000074640F6C823C2F200031868002800F0C7
:103C4000118140F6C821C2F200014A683F2A08D912
:103C500040F6C824C2F20004A5685619E368F518B6
:103C600001E04FF0400540F6C820C2F20000C16CF0
:103C7000002900F0008140F6C822C2F20002146D53
:103C8000A54207D840F6C826C2F20006756D601935
:103C9000B36DC51840F6C821C2F20001D1F89820D2
:103CA000002A00F0EC8040F6C824C2F20004D4F8E8
:103CB0009C60B54209D840F6C820C2F20000D0F896
:103CC000A0507119D0F8A430CD1840F6C822C2F225
:103CD0000002D2F8E440002C00F0D58040F6C8265F
:103CE000C2F20006D6F8E800854209D840F6C8219D
:103CF000C2F20001D1F8EC504219D1F8F030D518D9
:103D000040F6C824C2F20004D4F83061002E00F05E
:103D1000BE8040F6C820C2F20000D0F834118D42B7
:103D200009D840F6C822C2F20002D2F838514C1924
:103D3000D2F83C31E51840F6C826C2F20006D6F8A3
:103D40007C01002800F0A78040F6C821C2F20001E3
:103D5000D1F88021954209D840F6C824C2F2000467
:103D6000D4F884515619D4F88831F51840F6C82093
:103D7000C2F20000D0F8C811002900F0908040F68F
:103D8000C822C2F20002D2F8CC41A54209D840F6BE
:103D9000C826C2F20006D6F8D0516019D6F8D43140
:103DA000C51840F6C821C2F20001D1F81422002A39
:103DB00079D040F6C824C2F20004D4F81862B542A3
:103DC00009D840F6C820C2F20000D0F81C52711980
:103DD000D0F82032CD1840F6C822C2F20002D2F844
:103DE0006042002C63D0454E4FF00808FCF726FFD8
:103DF000387A88B140F27831C2F200010A8812F0B4
:103E0000020F0CD04FF0010404F1010442FA04F354
:103E100013F0010FF8D104E04FF0000401E04FF07F
:103E2000010440F27830C2F200004FF0010202FAC1
:103E300004F201880A4302807889B060BB89F3608C
:103E40003F2B99BF013323F001031F3323F01F03DE
:103E5000F360F26881184819B0F5E07F2ED9FCF7BD
:103E6000EDFE2BE040F6C826C2F200064FF0000837
:103E70004FF040051EE0224E4FF001081AE0214E9F
:103E80004FF0020816E0204E4FF0030812E01F4EDC
:103E90004FF004080EE01E4E4FF005080AE01D4EDC
:103EA0004FF0060806E01C4E4FF0070802E0134EE4
:103EB0004FF00808B8F1070F9AD997E740F6CC53AE
:103EC000C2F2000303F804803760756006F1200534
:103ED00028464FF000014FF01C0212F053FB3462F1
:103EE0007A68B26306F110004FF006013A682B467B
:103EF00000F02CF92046BDE8F08100BF280D00201D
:103F0000140B0020600B0020AC0B0020F80B0020ED
:103F1000440C0020900C0020DC0C0020032907D169
:103F200045F64C43C4F200031A6860F306021A60B7
:103F3000704700BFF0B585B00646002842D041F278
:103F40001C01C4F202010C6844F400050D604FF03E
:103F5000000400944FF0030501954FF00E070297FF
:103F600020464FF00B012A462346FDF79BFB0094A9
:103F70000195029720464FF00C012A462346FDF793
:103F800091FB49F2CC23C0F601031A6845F640477D
:103F9000C4F200073A60284603F0F8FD3C6043F69F
:103FA0002910C0F600004FF00F014FF04B02FCF754
:103FB0005FFF45F64440C4F2000004604FF41C412A
:103FC000396011E04FF000004FF00F014FF04B024D
:103FD000FCF74EFF49F2F423C0F601031A6845F6D8
:103FE0004040C4F2000002603046FCF713FE05B00A
:103FF000F0BD00BF2DE9F04182B049F2F827C0F6CC
:10400000010744F2D506C0F6000640F2BC15C2F224
:1040100000054FF00408CDF8008038464FF08001CD
:1040200032462B4601F02CFE40F2C034C2F20004AE
:104030002060CDF8008038464FF08101324605EB14
:10404000080301F01DFE6060CDF8008038464FF097
:104050008201324605F1080301F012FEA060CDF89E
:10406000008038464FF08301324605F10C0301F021
:1040700007FEE060CDF8008038464FF084013246FC
:1040800005F1100301F0FCFD2061CDF800803846F9
:104090004FF08501324605F1140301F0F1FD606136
:1040A000CDF8008038464FF08601324605F11803FE
:1040B00001F0E6FDA061CDF8008038464FF08701A1
:1040C000324605F11C0301F0DBFDE06102B0BDE802
:1040D000F08100BF80B505464FF0000640F29839E8
:1040E000C2F2000940F2E038C2F2000840F2943710
:1040F000C2F200071FE0FCF749FE2C6861682960E6
:104100004FF000026260237B062B0ED1216849F834
:104110002610092E9CBF0136F6B2012E03D93A882B
:1041200002F101023A8088F80060FCF739FE23684A
:104130000BB1A06898472B6803F1FF3010F1030F13
:10414000D9D901F01FFC4FF00006F4E70260B3F18B
:10415000FF3F18BF8360FF290ED145F69813C2F2C6
:1041600000031A6822B192F829304FEA530101E0A6
:104170004FF007010173704701F07F010173704731
:1041800010B14FF000020260704700BF38B504461E
:10419000FCF7FCFD054640F2E233C2F200031A8848
:1041A00002F101021A80002C35D06368EBB940F2AD
:1041B000E430C2F20000028802F101020280207B9A
:1041C00040F2BC13C2F2000353F82010616043F8C0
:1041D0002040247B40F2C032C2F2000252F8240098
:1041E00001F002FC4FF0010422E040F29030C2F2F4
:1041F0000000028802F101020280247B062C15D106
:1042000040F29631C2F200010B8803F101030B80EA
:104210004FF000040CE040F29230C2F2000001883E
:1042200001F1010101804FF0000401E04FF00004B2
:104230002846FCF7B5FD204638BD00BF10B5044642
:1042400040F2A050C2F200004FF000014FF01802FF
:1042500012F098F9D4B140F21840C2F200004FF0C9
:1042600000014FF0300212F08DF940F28040C2F2AE
:1042700000004FF000014FF0180212F083F940F2F5
:104280007843C2F200034FF002021A7010BD00BF63
:1042900038B549F21C33C0F6010353F8205040F200
:1042A0005041C2F2000151F8204049F24C32C0F6B0
:1042B0000102105CFDF78CFA2840A04214BF0020D8
:1042C000012038BD49F24C33C0F601031A5C40F2BC
:1042D0008041C2F2000151F8222049F21C33C0F69D
:1042E000010353F8200002420CBF00200120704758
:1042F00070B440F2CC73C2F2000353E8002F02F115
:10430000010243E800210129F7D049F24C32C0F6FE
:104310000102155C40F2A051C2F2000151F82540A3
:1043200049F21C36C0F6010656F8202024EA0200A5
:1043300041F8250053E8005FA5F1010543E8005668
:10434000012EF7D053E8005FB5F1004F0DD14FF0CB
:10435000000543E80056012EF4D04EF60450CEF28C
:104360000000016841F080510160BFF32F8F1442BB
:104370000CBF0020012070BC704700BF49F25833C9
:10438000C0F60103185C704710B50446FDF720FA2B
:1043900040F2DC13C2F2000353F82410484010BD71
:1043A00010B504464FF00100FFF748FF49F26433AF
:1043B000C0F6010353F8342040F27C41C2F2000100
:1043C0000A6003EBC404606840F29843C2F2000341
:1043D000186010BD00B585B04FF00000FFF7E0FF9A
:1043E0004FF00003009340F29C42C2F2000201929F
:1043F0004FF04000029049F24030C0F601004FF00B
:10440000020144F2A942C0F6000201F025FB40F28D
:104410009C53C2F20003186005B000BD2DE9F00105
:10442000804600283CD04FF000034FEA8302086822
:1044300050F823404D6855F8236086EA04078868E1
:1044400050F8235084EA050C4CEA07076FEA070C82
:10445000C86850F8235026EA050707EA0C0705EA62
:104460000C0C66EA0C06354040F82350CD6855F830
:104470002300384345F823000D6955F823003843DD
:1044800045F823004D690DB145F8237048688558FB
:10449000886885504868845003F101034345C4D1BE
:1044A000BDE8F001704700BF2DE9F84340F27C48B9
:1044B000C2F2000840F24846C2F2000640F2E83478
:1044C000C2F200044FF0000540F29847C2F2000724
:1044D000D8F8000000EB800001F01CFC3368002BD2
:1044E00040F05381204629464FF0180212F04AF856
:1044F0004BE14FF0060049F20431C0F60101FFF72D
:104500008DFF40F27841C2F200010A785AB102F1FF
:10451000FF3040F27843C2F20003187040F2A0511D
:10452000C2F200010D6040F27442C2F20002106853
:10453000E8B940F27443C2F200031D6040F24C41FE
:10454000C2F200010A784AB940F27442C2F2000293
:10455000106860B128460BF017FE08E040F2744086
:10456000C2F20000036843F000610160ECE740F232
:104570007843C2F20003197859B101F1FF3040F2DB
:104580007842C2F20002107040F2A053C2F200035F
:104590005D6040F27441C2F200010868E8B940F27F
:1045A0007442C2F20002156040F24C43C2F20003B2
:1045B000197849B940F27441C2F20001086860B14B
:1045C00028460BF0E1FD08E040F27440C2F2000022
:1045D000026842F000630360ECE740F27842C2F206
:1045E000000213785BB103F1FF3140F27840C2F270
:1045F0000000017040F2A052C2F20002956040F249
:104600007443C2F200031968E9B940F27440C2F27F
:104610000000056040F24C42C2F2000213784BB930
:1046200040F27443C2F20003196861B128460BF0EE
:10463000ABFD08E040F27441C2F20001086840F0AE
:1046400000620A60ECE740F27840C2F200000278B3
:104650005AB102F1FF3340F27841C2F200010B700F
:1046600040F2A050C2F20000C56040F27442C2F2B3
:1046700000021368EBB940F27441C2F200010D6010
:1046800040F24C40C2F2000002784AB940F2744253
:10469000C2F20002136863B128460BF075FD08E012
:1046A00040F27443C2F20003196841F000601860E0
:1046B000ECE740F27841C2F20001087858B100F10D
:1046C000FF3340F27842C2F20002137040F2A05170
:1046D000C2F200010D6140F27440C2F200000368B2
:1046E000EBB940F27442C2F20002156040F24C4154
:1046F000C2F20001087848B940F27440C2F20000EA
:10470000036863B128460BF03FFD08E040F27443B4
:10471000C2F200031A6842F000611960ECE740F24F
:104720007842C2F20002117859B101F1FF3040F233
:104730007843C2F20003187040F2A052C2F20002A5
:10474000556140F27441C2F200010868D8B940F2E4
:104750007443C2F200031D6040F24C42C2F20002F8
:10476000117839B140F27440C2F20000036843F09E
:104770000062026040F27441C2F20001086810B1A8
:1047800028460BF001FD3560A2E6D4F800902846DB
:10479000FFF7FAFD40EA09012160D4F804904FF0D8
:1047A0000100FFF7F1FD40EA09026260D4F80890C9
:1047B0004FF00200FFF7E8FD40EA0900A060D4F8DE
:1047C0000C904FF00300FFF7DFFD40EA0903E360C0
:1047D000D4F810904FF00400FFF7D6FD40EA09012D
:1047E0002161D4F814904FF00500FFF7CDFD40EAA9
:1047F00009026261306800F1010030603B68984254
:10480000FFF466AE75E600BF00B585B04FF000035B
:10481000009340F2E452C2F2000201924FF04000D5
:10482000029049F28440C0F601004FF0060144F6C0
:104830004902C0F6000201F00FF940F2B853C2F28B
:104840000003186005B000BD2DE9F04F85B040F2BF
:1048500030731F46C2F2000740F200700646C2F2F3
:10486000000640F2CC51C2F20001029101F08AF838
:104870003A68002AFAD014E1A359002B51D02846F7
:10488000FFF782FD029962586050904349D0A359C6
:1048900010EA030245D0039991F800E049F28C49EF
:1048A000C0F601094FEA451840F2BC51C2F20001BE
:1048B0004FF6FF7C49F2843AC0F6010A40F2E86BF9
:1048C000C2F2000B204674468646C2F10003134034
:1048D00022EA03021CB95EF80B0003421ED1180E37
:1048E00004D01AF8003003F118030DE0180C04D0BE
:1048F0001AF8003003F1100306E0180A1ABF1AF87C
:10490000003008331AF80330434419F8033031F803
:10491000130060451CBF013021F81300002AD4D1D8
:10492000744605F1010504F10404062DA4D1019D8E
:104930006A1E019240F0AC8003990C7804F10104E6
:10494000E3B20B700B2B03D14FF000050D7002E0AA
:10495000002B40F09A8040F21872C2F200021168F7
:1049600091B16FEA010433682340336040F2E8609C
:10497000C2F2000005682C40046040F21871C2F2D7
:1049800000014FF000020A6040F21874C2F2000405
:10499000636893B16FEA030075680540756040F283
:1049A000E862C2F2000251680840506040F2187498
:1049B000C2F200044FF00003636040F21870C2F2CC
:1049C0000000856895B16FEA0504B2682240B260C4
:1049D00040F2E863C2F2000399680C409C6040F228
:1049E0001870C2F200004FF00005856040F21874A4
:1049F000C2F20004E26892B16FEA0203F168194062
:104A0000F16040F2E860C2F20000C5682B40C3606C
:104A100040F21874C2F200044FF00002E26040F26B
:104A20001873C2F20003196991B16FEA0100356988
:104A30000540356140F2E864C2F20004226910408A
:104A4000206140F21873C2F200034FF000011961B7
:104A500040F21870C2F20000456995B16FEA050492
:104A600072692240726140F2E863C2F20003596940
:104A70000C405C6140F21870C2F200004FF000057B
:104A800045614FF4FA74019402E04FF4FA7001901A
:104A90004FF0010001F03EF93A68002A3FF4E6AE1B
:104AA00007E04FF4FA74019440F2E465C2F20005A5
:104AB00003954FF000042546DEE600BF10B54FF029
:104AC000000440F23073C2F200031C6040F2E86060
:104AD000C2F2000021464FF00602FCF711F940F245
:104AE0000070C2F2000021464FF00602FCF708F900
:104AF00040F21870C2F2000021464FF00602FCF7A7
:104B0000FFF840F2CC50C2F2000021464FF00602FE
:104B1000FCF7F6F840F2BC50C2F2000021464FF01C
:104B2000100211F02FFD40F2E460C2F200000470A8
:104B300010BD00BF70B549F24C33C0F601031B5CD9
:104B400049F21C32C0F6010252F8202040F23070C7
:104B5000C2F20000046840F20075C2F2000555F888
:104B60002300104206D104F1010640F23075C2F272
:104B700000052E6049B140F2E861C2F2000151F82F
:104B80002350154341F8235009E040F2E861C2F296
:104B9000000151F8235025EA020541F82350104343
:104BA00040F20071C2F2000141F8230040F2187196
:104BB000C2F2000151F8230020EA020241F823204A
:104BC00034B940F2B853C2F20003186800F00CFF89
:104BD00070BD00BF30B449F24C33C0F601031B5C1A
:104BE00049F21C32C0F6010252F8202040F2007057
:104BF000C2F2000050F82300104229D040F2307475
:104C0000C2F20004256805F10105256071B140F28A
:104C10001871C2F2000151F82340144341F82340B7
:104C200040F2E461C2F20001097889B96FEA020238
:104C300040F2E861C2F2000151F82340144041F80B
:104C40002340024040F20070C2F2000040F82320EE
:104C500030BC704730B4034640F2CC72C2F200025E
:104C600052E8000F00F1010042E80004012CF7D0E7
:104C700040F2BC50C2F2000030F8132039B140F2CB
:104C8000BC51C2F200014FF0000421F8134040F281
:104C9000CC73C2F2000353E8004FA4F1010443E8CF
:104CA0000045012DF7D053E8004FB4F1004F0DD16E
:104CB0004FF0000443E80045012DF4D04EF60450B7
:104CC000CEF20000016841F080510160BFF32F8FE8
:104CD000104630BC704700BF40F2E463C2F20003EC
:104CE0001878D0F1010038BF002070472DE9F84F47
:104CF000DFF834814B4FC8EB07004FEAD00707F1CC
:104D000001074FF0000540F2982AC0F6000A40F271
:104D10005839C0F6000931E044464FF000066FEA0A
:104D2000060B0BEB070101F0010B58F8043CAB42FA
:104D300029D135E054F8043CAB4205D154F8080CB5
:104D40008047FCF73DFF0BE0FF2B09D9FF2D07D172
:104D500054F8040C4FF0070154F8082C00F09CFFA5
:104D600006F1010604F1080454F8041CA94240D1DC
:104D70004CE005F10105B5F5807F02D0CA45CBD3E3
:104D8000F7E7BDE8F88FFF2B0FD9FF2D0DD158F8AD
:104D9000040C4FF0070158F8082C00F07DFF04E0E8
:104DA00058F8082C9047FCF70BFF06F1010604F1B8
:104DB0000804BE42DDD0BBF1000FBBD054F8040C98
:104DC000A8420AD0FF280DD9FF2D0BD14FF00701C3
:104DD00054F8082C00F060FF04E054F8081C8847E1
:104DE000FCF7EEFE06F1010604F10804BE42A1D173
:104DF000BFE7FF290FD9FF2D0DD154F8040C4FF058
:104E0000070154F8082C00F047FF04E054F8082C80
:104E10009047FCF7D5FE06F1010604F10804BE42F6
:104E200088D1A6E75F030008A0020008027840F2DC
:104E30009973C2F200031B789A4206D34FF0000226
:104E40000270087800F1010008700A7840F29A7345
:104E5000C2F200031878824224BF00200870704715
:104E600010B5A0F10803052B3DD8DFE803F01F3C87
:104E70002C3C038340F23870C2F200004FF0200156
:104E80004FF0540211F07EFB40F28C70C2F2000031
:104E90004FF0FF314FF00C0211F074FB40F2A070A4
:104EA000C2F20000026802F1010202604FF000014C
:104EB00040F23473C2F20003197040F23570C2F24E
:104EC0000000017056E040F23471C2F200014FF070
:104ED00000030B7040F23570C2F20000027802F15C
:104EE000010202703CE040F23472C2F20002127819
:104EF00040F23571C2F200010B7840F29971C2F2B2
:104F00000001097801FB032340F23871C2F200016D
:104F1000C95C81421DD040F23874C2F20004E054F2
:104F20004FEA531040F28C71C2F2000103F01F03EC
:104F30004FF0010404FA03F351F820401C4341F8F8
:104F4000204040F2A070C2F20000016801F10101AE
:104F5000016002F1010240F23473C2F200031A70E0
:104F600040F23470C2F2000040F23571C2F200012A
:104F7000FFF75CFF4FF0000010BD00BF70B4039D51
:104F8000049C064628B140F29C70C2F200000078F2
:104F9000307029B140F2A470C2F2000000780870AD
:104FA0002AB140F29871C2F20001087810702BB15A
:104FB00040F2A572C2F20002117819702DB140F2D0
:104FC0003473C2F20003187828702CB140F23572A5
:104FD000C2F200021178217070BC704706281DD8FB
:104FE000002808BF052040F29C73C2F2000318702D
:104FF00049F24C53C0F6010313F8101040F29972B5
:10500000C2F20002117003EB4000417840F29A7343
:10501000C2F2000319704FF0010070474FF000001A
:10502000704700BF08B540F2A473C2F200034FF00E
:1050300001021A704FF00500FFF7D0FF4FF00C008F
:105040004FF00001FFF70CFF08BD00BF08B540F2AC
:105050003472C2F20002107040F23573C2F20003E3
:10506000197010461946FFF7E1FE08BD034628B146
:1050700040F29970C2F200000078187029B140F235
:105080009A73C2F20003187808702AB140F2A07136
:10509000C2F200010B68136040F23870C2F20000E7
:1050A000704700BF2DE9F00140F23877C2F20007E7
:1050B0003F1853284BD8002A49D03B4607F1010737
:1050C00002F1FF3257FA82F74FF0000640F28C747B
:1050D000C2F200044FF001056FEA030C0CEB07026B
:1050E00002EA050C13F8018B01F1FF3111F8012FD1
:1050F00090452FD13DE013F801CB01F10100497833
:105100008C450ED003F8011C4FEA521102F01F0625
:1051100005FA06FC54F821604CEA060644F82160C2
:105120002E4602F10102D2B2542A07D013F801CB65
:1051300000F101014078844542D150E03EB140F297
:10514000A073C2F20003196801F101011960BDE802
:10515000F001704703F8012C4FEA501600F01F08C9
:1051600005FA08F854F8262048EA020244F82620F6
:105170002E4600F10100C2B2542ADFD0BB42DDD07E
:10518000BCF1000FB7D013F801CB11F8010F844523
:105190000ED003F8010C4FEA521002F01F0605FA78
:1051A00006FC54F820604CEA060644F820602E46BF
:1051B00002F10102D2B2542AC0D0BB429BD1BDE75A
:1051C00003F8010C4FEA521002F01F0605FA06FC24
:1051D00054F820604CEA060644F820602E4602F19E
:1051E0000102D2B2542AA9D0BB4284D1A6E700BFA3
:1051F000003018BF012040F2A473C2F200031870FF
:10520000003118BF012140F29870C2F20000017015
:10521000003218BF012240F2A573C2F200031A70D7
:10522000704700BF40F29B73C2F200034FF00002D0
:105230001A7070474FF05400704700BF40F29B73E4
:10524000C2F200034FF001021A707047034628B102
:105250000868834214BF0020012070474FF000000F
:10526000704700BF10B440F2CC73C2F2000353E8A1
:10527000002F02F1010243E800210129F7D0046860
:10528000C4B16268824202D19268626002E04368FF
:10529000816899602368834202D15B68236002E0E1
:1052A000826841685160A26802F1FF31A1604FF04D
:1052B0000004046040F2CC73C2F2000353E8002FF4
:1052C000A2F1010243E80024012CF7D053E8002F9B
:1052D000B2F1004F0DD14FF0000243E80024012C41
:1052E000F4D04EF60450CEF20000016841F0805137
:1052F0000160BFF32F8F10BC704700BF38B5044664
:105300000D464FF000014FF0100211F03BF9E5603F
:1053100038BD00BFF8B504460F46C6688D1929464A
:10532000FFF794FF00283CD140F2CC73C2F2000397
:1053300053E8002F02F1010243E800210129F7D0D0
:105340004FF0000068606168A96001B14D6022689B
:1053500002B925606560BC51A36803F10103A36035
:1053600040F2CC73C2F2000353E8002FA2F1010215
:1053700043E80024012CF7D053E8002FB2F1004F8E
:105380000DD14FF0000243E80024012CF4D04EF67A
:105390000450CEF20000016841F080510160BFF37B
:1053A0002F8FF8BD2DE9F04104468846C6688D1957
:1053B0009719C2B940F2CC73C2F2000353E8002F30
:1053C00002F1010243E800210129F7D002686A6076
:1053D00005604FF00000A860616809B9656020E0D1
:1053E0006B689D601DE03946FFF730FF00283FD015
:1053F0002846FFF737FF40F2CC73C2F2000353E8B0
:10540000002F02F1010243E800210129F7D0B8681A
:10541000A8606F60BD602168B9420EBF2560A968B1
:105420004D6048F80640A26802F10102A26040F215
:10543000CC73C2F2000353E8002FA2F1010243E84B
:105440000024012CF7D053E8002FB2F1004F0DD10A
:105450004FF0000243E80024012CF4D04EF6045033
:10546000CEF20000016841F080510160BFF32F8F40
:10547000BDE8F081C368C918486808B1C01A704710
:105480004FF00000704700BF036813B1C068181ADE
:1054900070474FF00000704708B5C368C918FFF7A0
:1054A000D5FE08BD08B5C0680818FFF7DBFE08BDCB
:1054B00008B540F2A870C2F200004FF01C01FFF7DF
:1054C0001DFF08BD70B5054600F108063046FFF720
:1054D000DBFF0446686050B130462146FFF7E2FF2B
:1054E0004FF00100A861204600F07EFA70BD4FF039
:1054F0000003AB6170BD00BF38B504460D464FF0E8
:1055000000014FF0280211F03DF8204640F8085BFA
:105510004FF01C01FFF7F2FE40F2A870C2F200004B
:105520002146FFF7F7FE38BD2DE9F04107468846D2
:1055300045F69813C2F200031868002800F0FE80B8
:1055400040F2CC74C2F2000454E8002F02F10102D0
:1055500044E800210129F7D0796831B145F6981265
:10556000C2F20002136899422ED145F69810C2F299
:10557000000004687C60B96901F10101B96140F281
:10558000CC73C2F2000353E8002FA2F1010243E8FA
:105590000024012CF7D053E8002FB2F1004F0DD1B9
:1055A0004FF0000243E80024012CF4D04EF60450E2
:1055B000CEF20000016841F080510160BFF32F8FEF
:1055C0004FF00100BDE8F081B8F1FF3F24D140F277
:1055D000CC73C2F2000353E8002FA2F1010243E8AA
:1055E0000024012CF7D053E8002FB2F1004F0DD169
:1055F0004FF0000243E80024012CF4D04EF6045092
:10560000CEF20000016841F080510160BFF32F8F9E
:105610004FF00000BDE8F08107F108052846FFF7CC
:1056200033FF0246F0B145F69816C2F20006306824
:1056300092F8294090F829108C4208D912E033687A
:1056400092F8290093F82940A04204D90AE045F6CF
:105650009816C2F2000628461146FFF70BFF0246D5
:105660000028ECD1284645F69811C2F200010968DD
:10567000FFF798FE40F2CC76C2F2000656E8002F03
:10568000A2F1010246E80024012CF7D056E8002FD1
:10569000B2F1004F0DD14FF0000246E80024012C7A
:1056A000F4D04EF60450CEF20000016841F0805173
:1056B0000160BFF32F8FB8F1000F04D008EB880012
:1056C00000F028FB01E000F05DF940F2CC74C2F27A
:1056D000000454E8003F03F1010344E80032012ACA
:1056E000F7D045F69816C2F2000628463168FFF753
:1056F000D9FE54E8003FA3F1010344E80032012A37
:10570000F7D054E8003FB3F1004F0DD14FF0000344
:1057100044E80032012AF4D04EF60450CEF20000E4
:10572000016841F080510160BFF32F8F78683268C3
:10573000904214BF00200120BDE8F0814FF001002D
:10574000BDE8F08110B5044645F69813C2F2000397
:105750001868002860D06268904201D0FBF76EFAAA
:1057600040F2CC73C2F2000353E8002F02F10102B1
:1057700043E800210129F7D0A16901F1FF30A061C0
:1057800018B340F2CC73C2F2000353E8002FA2F129
:10579000010243E80024012CF7D053E8002FB2F1B6
:1057A000004F0DD14FF0000243E80024012CF4D04B
:1057B0004EF60450CEF20000016841F080510160C5
:1057C000BFF32F8F4FF0000010BD2046FFF77AFE89
:1057D00040F2CC73C2F2000353E8002FA2F10102A1
:1057E00043E80024012CF7D053E8002FB2F1004F1A
:1057F0000DD14FF0000243E80024012CF4D04EF606
:105800000450CEF20000016841F080510160BFF306
:105810002F8F4FF0010010BD4FF0010010BD00BFF1
:10582000F8B5054640F2CC73C2F2000353E8002FEE
:1058300002F1010243E800210129F7D040F2A870EB
:10584000C2F20000FFF720FE0446E0B140F2A87764
:10585000C2F200076068A84203D12046FFF732FE7B
:105860000AE004F1080630462946FFF715FE18B194
:1058700030462946FFF716FE38462146FFF7FAFD67
:1058800004460028E6D140F2CC73C2F2000353E88C
:10589000002FA2F1010243E80024012CF7D053E8C5
:1058A000002FB2F1004F0DD14FF0000243E8002469
:1058B000012CF4D04EF60450CEF20000016841F005
:1058C00080510160BFF32F8FF8BD00BF08B549F2CA
:1058D0005853C0F60103195C012906D011B1022901
:1058E0000BD105E0FDF73AFE08BD02F00FF908BD47
:1058F000FBF7A4F94FF0000008BD4FF0000008BD11
:105900004EF60453CEF200031A6842F0805018603D
:10591000704700BF4FF0010280F8282040F2C873A2
:10592000C2F2000390F8291002FA01F2188802432B
:105930001A80704710B440F2C473C2F200031A68B0
:10594000C2B1904213D104E088420FD102F1140297
:1059500003E040F2C472C2F2000243691BB19C69C9
:105960008169611899614369136003E00A465169CE
:105970000029E9D14FF0000282614FF0FF3141610F
:1059800010BC704710B5FBF701FA044645F69813B2
:10599000C2F20003186890F82820032A1BD0FBF7F6
:1059A000F5F945F69813C2F2000319684FF00002AA
:1059B00081F8282091F82920096940F6B803C2F23D
:1059C000000343F82210FBF7EBF92046FBF7E8F958
:1059D000FFF796FF10BD4FF0020180F82810204617
:1059E000FBF7DEF910BD00BF38B5044690B303687D
:1059F00083B3FBF7CBF9054694F8280010BB20468B
:105A0000FFF788FF45F69811C2F200010B6843B119
:105A100094F8292093F8290020F00101531A002B53
:105A200015DA40F2CC72C2F20002106838B140F0D0
:105A3000004140F2CC73C2F20003196007E0FFF7A7
:105A40005FFF04E0022804BF032084F828002846F2
:105A5000FBF7A6F938BD00BF2DE9F04F85B006462B
:105A60000F46934698460F9DDDF84090FBF78EF960
:105A7000824640F61003C2F2000319685048814282
:105A80000FD248F20002C2F2000252F82C4C54B17C
:105A90004C4B1C468B4207D953F82C090028F8D1EF
:105AA00002E0474C00E0464CA14206D1A1F12C0196
:105AB00040F61002C2F20002116020464FF00001D1
:105AC0004FF02C0210F05EFD4FF0FF3161611EB906
:105AD00049F25C56C0F601062660B8F1000F08D006
:105AE0000E9B042B08D9184600F103004FEA9006DC
:105AF00004E04FF0000601E04FF000060DBB46F257
:105B00009C49C2F2000940F2B875C2F2000529684A
:105B100045F67570C0F600000090CDF8048002963E
:105B200048464FF000025B46FBF768FC2A68A2601B
:105B3000E0604FEA800153182B60C1EB0900606000
:105B400020E028464FF0FF314A46FBF7D9F84AF2E9
:105B5000ED52CDF6CE622A60E56005EB8905656001
:105B600045F67571C0F600010091CDF804800296EB
:105B7000284629464FF001025B46FBF73FFCA5EBA8
:105B8000800363606FEA0702C2F3C01101EB4707AD
:105B900007F0FF0784F8297040F2D073C2F20003C7
:105BA00053F82700206143F827405046FBF7F8F8E8
:105BB0002046FFF719FF204605B0BDE8F08F00BF73
:105BC000D47F0020A87F002030B585B04FF00001C1
:105BD00045F69813C2F200031960284C48F20005FC
:105BE000C2F200052A1B20464FEAA202FBF788F802
:105BF00040F2B870C2F200000460A5F12C0540F636
:105C00001001C2F200010D6045F69C43C2F2000390
:105C10004FF0B504CBF26B141C6003F14C004FF055
:105C2000FF3243F8042F43F8042F43F8042F834234
:105C3000F9D14FF00004009440F61401C2F20001C3
:105C400001914FF02803029349F26850C0F6010019
:105C50004FF0070145F6F542C0F600022346FFF774
:105C6000FBFE40F6B402C2F20002106040F2D070B7
:105C7000C2F20000C46305B030BD00BFA0640020C4
:105C800010B584B0069C00944FF000040194029477
:105C9000FFF7E2FE04B010BD00B585B04FF0000381
:105CA000009301930293FFF7D7FE05B000BD00BF3C
:105CB00038B545F69813C2F200031868C0B1FBF777
:105CC00065F8054645F69814C2F200042068FFF70F
:105CD00021FE216891F82920086940F6B803C2F234
:105CE000000343F822002846FBF75AF8FFF708FEA6
:105CF00038BD00BF38B545F69815C2F2000540F230
:105D0000D074C2F200042B6822681A61FFF7D0FF3A
:105D1000F9E700BF38B545F69813C2F200031968D9
:105D2000002900F0918020B9FFF7C2FF4FF0010277
:105D30009AE0B0F1FF3F04D1FFF724FE4FF00002DC
:105D400092E040F2CC74C2F2000454E8002F02F159
:105D5000010244E800210129F7D040F2C472C2F2E6
:105D600000021568002D7AD0AB6998426FD3C01A33
:105D700005F114016D691DB1AB698342F7D96AE081
:105D800045F69815C2F200052B68986108685861BD
:105D90001846FAF757FF40F2CC74C2F2000454E8F8
:105DA000003FA3F1010344E80032012AF7D054E890
:105DB000003FB3F1004F0DD14FF0000344E8003233
:105DC000012AF4D04EF60450CEF20000016841F0F2
:105DD00080510160BFF32F8FFFF7D4FD54E8003FDF
:105DE00003F1010344E80032012AF7D02868416931
:105DF000B1F1FF3F04D0FFF79DFD4FF0000201E03D
:105E00004FF0010240F2CC73C2F2000353E8004F9E
:105E1000A4F1010443E80045012DF7D053E8004FF9
:105E2000B4F1004F0DD14FF0000443E80045012DBF
:105E3000F4D04EF60450CEF20000016841F08051DB
:105E40000160BFF32F8F0FE04FF001020CE040F232
:105E5000C471C2F20001AC69221AAA6190E740F253
:105E6000C471C2F200018BE7104638BDF8B5044694
:105E700000287AD0FAF78AFF064640F61003C2F2ED
:105E8000000319683948814211D248F20002C2F277
:105E9000000252F81C5CA54263D0354B1D468B4274
:105EA00005D9A3F12C03D86BA042F7D15AE094F89E
:105EB000293040F2D072C2F2000252F82300A04210
:105EC00006D1016940F2D072C2F2000242F82310FA
:105ED0002046FFF72FFD2046FFF7A2FC94F829008B
:105EE000236940F6B801C2F2000141F8203045F6BE
:105EF0009812C2F200021068A04229D0A06838B3FC
:105F0000E76800EB870540F2B877C2F200073B680C
:105F10005A1B29464FEAA2024FF00003FCF748F94A
:105F2000E1683868A0EB81033B6040F61002C2F2E2
:105F3000000211680D4B99420AD29A68954203D823
:105F4000E068A2EB80029A60A3F12C038B42F4D8A4
:105F50004FF00001216084F828103046FAF720FF46
:105F6000F8BD024D21692961A1E7F8BDD47F002069
:105F7000A87F002000BFF04772B645F69814C2F221
:105F800000042068FFF772FF4FF000032360FBF767
:105F900085FA00BF40F2C473C2F20003196849B128
:105FA000886950B100F1FF328A61D2F1010038BF37
:105FB000002070474FF0000070474FF0000070471E
:105FC00070B540F2C473C2F200031C68A4B1A069AA
:105FD00090B940F2C475C2F200054FF0FF36606917
:105FE0002946FAF72FFE66612046FFF7FDFC2C6874
:105FF00014B1A1690029F2D070BD00BFF0B472B62F
:1060000040F2C873C2F200031C882CB940F6B403F6
:10601000C2F2000318685FE049F2705CC0F6010C40
:1060200040F6B805C2F2000540F2D076C2F2000692
:10603000C4F1000323401A0A1ABF1CF802100831E9
:106040001CF8031011F0010F0AD141F0010055F8BE
:10605000200038B190F82820012A38D81F4602E0E5
:106060001F4600E01F4655F82120B2B192F82830B3
:106070007BB140F2C870C2F20000048010462BE0F1
:1060800090F8283033B140F2C872C2F20002148096
:1060900022E0104600690028F2D156F82100824221
:1060A00007D1BC43C4D140F2C871C2F200010C80D8
:1060B000ACE745F8210011F0010FD4D114EA4703F1
:1060C000D1D04FEA4707BFB241F00101CBE740F220
:1060D000C871C2F200010C8062B6F0BC704700BF0C
:1060E00070B545F69813C2F200031B6883420FD1C6
:1060F00093F82820012A9CBF022283F8282093F8D5
:10610000291040F6B800C2F2000040F8213070BDFE
:1061100040F2BC72C2F20002136045F69811C2F25E
:106120000001086090F8292040F6B803C2F200038D
:1061300043F8220090F8281001299CBF022180F822
:1061400028108268AAB9C1684AF2ED53CDF6CE6331
:106150000868984201D0FAF771FD45F69812C2F22C
:10616000000211684868CB6898427ED2FAF766FD53
:1061700070BD40F2C073C2F200031B68984274D035
:1061800093B3586846F29C44C2F20004251A4FEAC1
:10619000A501D96045F69C42C2F2000290420AD3A2
:1061A0004FF0B503CBF26B1345F69C40C2F20000F2
:1061B00004689C4201D0FAF741FD40F2C075C2F27A
:1061C00000052A6840F2B874C2F2000420685168E1
:1061D000D2684FF00003FBF7EBFF296823688B6060
:1061E000C86803EB8002226045F69811C2F20001F4
:1061F0000B6840F2C070C2F200000360DA68002A47
:1062000033D0586899684FF00103FBF7D1FF45F68A
:106210009816C2F200063568A868EC6800EB8404A2
:1062200040F2B876C2F200063268131B21464FEAEC
:10623000A3024FF00003FBF7BBFFE9683068A0EB57
:106240008102326040F61003C2F200031968074B66
:1062500099420AD29A68944203D8E868A2EB800275
:106260009A60A3F12C038B42F4D870BDD47F002038
:1062700000B585B040F65420C2F200004FF0000196
:10628000FFF73CF840F6FC00C2F200004FF00001BE
:10629000FFF734F84FF00003009340F61412C2F2F7
:1062A000000201924FF05000029049F27060C0F677
:1062B0000100194646F2C552C0F60002FFF7CCFBBA
:1062C00040F6F803C2F20003186005B000BD00BF3D
:1062D00008B5FFF7D9F8034648B1C06850B100F1DE
:1062E000FF31D960D1F1010038BF002008BD4FF067
:1062F000000008BD4FF0000008BD00BF70B50546A6
:106300000E46144640F2CC73C2F2000353E8002F4D
:1063100002F1010243E800210129F7D0FFF7B4F8A8
:106320000246002839D0C06884422DD3241A28465A
:106330001146FFF79FF8024600282ED0C068A04201
:10634000F4D921E040F2CC73C2F2000353E8002FED
:10635000A2F1010243E80024012CF7D053E8002FFA
:10636000B2F1004F0DD14FF0000243E80024012CA0
:10637000F4D04EF60450CEF20000016841F0805196
:106380000160BFF32F8F70BDF460D1680B1BD36029
:1063900028463146FFF706F8D4E7F4602846314630
:1063A000FEF7B8FFCEE700BFF8B50646FFF76CF87A
:1063B0000446F8B1C368EBB930462146FFF75AF8F6
:1063C0000546FAF7E3FC074630462146FFF76AF830
:1063D0003846FAF7E5FC22691AB130462146FFF744
:1063E0008DFF04F11400FDF7D1FE1DB12C46E868C5
:1063F0000028E1D0F8BD00BF08B540F61013C2F286
:1064000000031A6802F101021A6040F6FC00C2F2B1
:106410000000FFF75DFF28B140F6FC00C2F200006B
:10642000FFF7C2FF08BD00BF08B5014640F6542083
:10643000C2F20000FFF730F820B140F65420C2F25B
:10644000000008BD40F6FC00C2F2000008BD00BF1D
:1064500070B5044640F2CC73C2F2000353E8002F3B
:1064600002F1010243E800210129F7D0FFF7DCFF28
:1064700005462146FFF710F8002845D040F2CC70C1
:10648000C2F2000050E8002F02F1010240E80021B2
:106490000129F7D028462146FEF7ECFF18B1C16864
:1064A000E2688B18C360FAF771FC0646284621465D
:1064B000FEF7F8FF3046FAF773FC4FF0FF35E56062
:1064C00040F2CC73C2F2000353E8002FA2F10102A4
:1064D00043E80025012DF7D053E8002FB2F1004F1B
:1064E0000DD14FF0000243E80025012DF4D04EF607
:1064F0000450CEF20000016841F080510160BFF30A
:106500002F8F4FF0010501E04FF0000504F114005A
:10651000FDF736FE40F2CC73C2F2000353E8002FC1
:10652000A2F1010243E80024012CF7D053E8002F28
:10653000B2F1004F0DD14FF0000243E80024012CCE
:10654000F4D04EF60450CEF20000016841F08051C4
:106550000160BFF32F8F284670BD00BF2DE9F041C9
:1065600005460F4614469846FFF772FF064694B15B
:106570009DF82030002B14BF20460020286105F133
:1065800014004146069A079BFDF7E0FD3846294670
:106590002246FFF7B3FE3046BDE8F08170B584B007
:1065A0000E4615460093089C01949DF824300293F2
:1065B00040F65421C2F2000132462B46FFF7CEFFCF
:1065C00004B070BD00B583B04FF0000300934FF0EE
:1065D0000100019040F66420C2F2000041F28831CF
:1065E0004FF0FF0246F2F933C0F60003FFF7D6FF83
:1065F00040F65424C2F20004FFF7E2FC2046FFF705
:10660000D3FEFFF7BFF9F7E740F60C13C2F2000321
:1066100018681A689042FBD1704700BF10B540F669
:106620000C13C2F200031A6802F101021A60FFF7AC
:10663000B1FC044640F65420C2F20000FFF748FEC9
:10664000204310F0FF0F06D040F6F800C2F2000021
:106650000068FFF7C9F910BD08B549F27C60C0F6C3
:1066600001004FF0060146F69522C0F60002FFF742
:1066700013FB40F69C53C2F20003186008BD00BF34
:1066800038B504460D4640F6C823C2F20003586AE6
:10669000A0420AD040F6C821C2F200014C620A684A
:1066A0001AB115B14948FDF771FD40F6C823C2F291
:1066B0000003186F84420AD040F6C821C2F20001DC
:1066C0000C67CA6C1AB115B14148FDF75FFD40F681
:1066D000C823C2F20003D3F8BC0084420CD040F6B9
:1066E000C821C2F20001C1F8BC40D1F898201AB10B
:1066F00015B13848FDF74AFD40F6C823C2F2000341
:10670000D3F8080184420CD040F6C821C2F200013F
:10671000C1F80841D1F8E4201AB115B12E48FDF7AF
:1067200035FD40F6C823C2F20003D3F85401844279
:106730000CD040F6C821C2F20001C1F85441D1F892
:1067400030211AB115B12548FDF720FD40F6C823C8
:10675000C2F20003D3F8A00184420CD040F6C82155
:10676000C2F20001C1F8A041D1F87C211AB115B1E3
:106770001B48FDF70BFD40F6C823C2F20003D3F817
:10678000EC0184420CD040F6C821C2F20001C1F8ED
:10679000EC41D1F8C8211AB115B11248FDF7F6FC49
:1067A00040F6C823C2F20003D3F83802A0420CD04E
:1067B00040F6C821C2F20001C1F83842D1F81422D3
:1067C0001AB115B10848FDF7E1FC38BDD80A002020
:1067D000240B0020700B0020BC0B0020080C0020B4
:1067E000540C0020A00C0020EC0C00202DE9F047F8
:1067F00007460D4691460898DDF828800C683E68EB
:10680000D8F800108A19944202D80219964203D38C
:1068100004192C60BDE8F087341B061BB14234BF5D
:106820008A46B246099931B1D9F8000008181919F9
:1068300052460FF083FED8F80030CAEB0302C8F8C6
:1068400000203E6806EB0A013960D9F8000000EB31
:106850000A03C9F800302E68A41954442C60BDE81E
:10686000F08700BF70B584B09CF81960157A947BEE
:106870004FF007038CF810304FF005028CF8112010
:1068800006F00F0260F3C7128CF812204FF00000E0
:1068900065F301008CF813004FF0000261F30A0267
:1068A000ACF814208CF81640DCF80C100093DCF8DF
:1068B00004300193CDF808C001F104000CF1080286
:1068C0000CF11003FFF792FF04B070BD2DE9F04FFB
:1068D0008FB00746059114464FF0000307931360ED
:1068E00012896068131A8B4238BF059305990029F5
:1068F00000F0AA8040F6A055C2F200052D6815B33D
:106900004FEAC5054FF000024FF0FF01134640F675
:10691000A850C2F20000A5F10806C6F3C00E165832
:10692000F6798E4240F0958096E01658F6798E42C0
:106930001CBF0133314602F108028658F6798E42B7
:1069400040F09F80A0E04FF0000303EB43024FEACA
:10695000C20000F1100008904FF48071ADF82410CF
:106960004FF00402ADF826208DF828300DF12900F3
:106970004FF000014FF007020FF004FE04F1040B8A
:1069800004944FF010030093019705A80290584615
:10699000214607AA08ABFFF729FF0599002951D026
:1069A0004FF001028DF821200DF132004FF000016F
:1069B0004FF006020FF0E6FD40F6A053C2F20003CE
:1069C000186800283ED04FF0FF014FF0000440F659
:1069D000A859C2F2000949F2A068C0F6010840F6C1
:1069E000A05AC2F2000A59F83450ED798D4223D0F2
:1069F0008DF820404FEA05160DF1220008EB060144
:106A00004FF008020FF09AFD06F108010DF12A007F
:106A100041444FF008020FF091FD4FF01802009230
:106A2000019705AB02935846049907AA08ABFFF7F4
:106A3000DDFE059830B1294604F10104DAF80020A2
:106A4000A242D0D8079801E04FF0FF300FB0BDE868
:106A5000F08F03F10103314602F10802AA423FF42C
:106A600074AFBEF1000F3FF460AF1658F6798E4256
:106A70001CBF0133314602F10802AA427FF455AF30
:106A800063E703F10103314602F10802AA427FF4F1
:106A90004CAF5AE72DE9F0414FF00100FDF74AFAFB
:106AA00049F28C60C0F60100FDF7C0F840F6C9530A
:106AB000C2F200034FF001021A7040F69850C2F281
:106AC0000000016841B940F69854C2F20004FEF794
:106AD00059FF2568002DFAD040F6A557C2F20007ED
:106AE00040F6C954C2F2000440F62856C2F200062D
:106AF00040F6C855C2F2000540F69458C2F20008AC
:106B00003B783BB14FF000023A704FF0020020702A
:106B1000FDF758F8317859B14FF0000333702278FF
:106B200062F07F0020704FF001000146FFF7A8FDE2
:106B3000297851B14FF000002870237803F07F02CC
:106B400022704FF00101FFF79BFD98F8000010B98B
:106B5000FEF718FFD4E740F6C951C2F200014FF02A
:106B600002030B704FF00000FDF7E4F9BDE8F0817F
:106B700008B540F69853C2F20003186040F69C50E6
:106B8000C2F200000068FEF72FFF08BD70B5054691
:106B90000E4640F6E053C2F200031868032801D9FC
:106BA000FAF74CF840F6E052C2F20002116840F6E3
:106BB0006C54C2F2000444F8316004EBC104656017
:106BC00001F10101116070BD70B505460C46164615
:106BD000032801D9FAF732F840F6A853C2F20003AD
:106BE00053F8350008B1FAF729F840F6A851C2F277
:106BF000000141F8354001EBC5056E6040F6A05339
:106C0000C2F200031A6802F101021A60206930B171
:106C1000FDF70CF804F1040420690028F8D170BDD8
:106C200008B540F6C823C2F20003196881425AD061
:106C300040F6C822C2F20002D36C834234D040F640
:106C4000C821C2F20001D1F8982082422FD040F62C
:106C5000C823C2F20003D3F8E41081422AD040F6E0
:106C6000C822C2F20002D2F83031834225D040F669
:106C7000C821C2F20001D1F87C21824220D040F626
:106C8000C823C2F20003D3F8C81181421BD040F6DA
:106C9000C822C2F20002D2F81432834216D0F9F7A9
:106CA000CDFF4FF0080013E04FF0010010E04FF06F
:106CB00002000DE04FF003000AE04FF0040007E08F
:106CC0004FF0050004E04FF0060001E04FF0070030
:106CD00040F6C821C2F200014FF04C0202FB001046
:106CE00090F8200008BD4FF00000F1E72DE9F04FCB
:106CF0008FB0089007910A924FF000030993136038
:106D0000546813891B1B8B4238BF079307990029CE
:106D100000F04A81082C69D840F6A054C2F2000461
:106D2000D4F800E040F6E055C2F200052E680EEB04
:106D3000CE0707EBC60404F109044FF0000140F64A
:106D4000A857C2F20007CB598BB1DD68641903F173
:106D500010051B695BB15E890EB104F107049B89C4
:106D60000BB104F1070455F8043F002BF3D101F1F6
:106D700008012029E7D140F69851C2F200010D68C0
:106D80002F7E6E7EEB8A03F10103C3F347054FF0BC
:106D900000010C914FF009038DF82C304FF00201E7
:106DA0008DF82D10ADF82E408DF830E04FF0010138
:106DB0008DF831104FF0000167F3451166F386112D
:106DC00061F07F018DF833108DF8345000930190FD
:106DD00007A8029002F10400114609AA0BABFFF7C5
:106DE00005FD079A002A00F0DD80E0E04FF0090081
:106DF0001060DCE05BF83640002C00F0CE80059D92
:106E0000286800284BD07A68B2420CD04FF00003BB
:106E100010F0010F3ED1DFE007EBC3025268B2422F
:106E200040F0E38001E04FF0000357F83300D2B2A6
:106E300090F8048090F805C090F806E0C5790168E4
:106E400019B143F01000C3B201E04FF000034FF05E
:106E500008008DF82C004FF00B018DF82D108DF8E7
:106E60002E208DF82F808DF830C08DF831E08DF810
:106E700032508DF833300A990090089A019207AB8E
:106E8000029301F1040009AA0BABFFF7AFFC0798CE
:106E900028B987E003F101052B468542BCD104F1F6
:106EA000100523697BB129464FF00002588908B1CB
:106EB00002F101029B890BB102F1010251F8043F7A
:106EC000002BF3D101E04FF000025FFA86FCD2B252
:106ED00094F804E06079A17923681BB146F020039F
:106EE000DBB201E04FF000038DF82CA04FF0040856
:106EF0008DF82D808DF82EC04FF0000C8DF82FC02E
:106F00008DF830208DF831E08DF832008DF8331097
:106F10008DF834300A99CDF800A0089A019207A89C
:106F2000029001EB080009AA0BABFFF75FFC079981
:106F3000002937D0A3686BB10A99E26800920898DB
:106F4000019007AA029201EB080009AAFFF74EFC84
:106F5000079B3BB3246904B34FF001084FF00009CD
:106F60002046FFF75DFE8DF83500618939B10DF1DE
:106F70001C0C40462246FFF775FC079991B1A18988
:106F800039B10DF11C0C48462246FFF76BFC0798FF
:106F900040B155F8044F002CE2D106F10106042E51
:106FA0007FF428AF099814E04FF0FF3011E04FF064
:106FB000000640F6A85BC2F2000B40F6E054C2F2B5
:106FC000000405944FF0090A40F66C57C2F200071E
:106FD00010E70FB0BDE8F08F03F1010307EBC30129
:106FE0004A68B2427FF456AF1FE705F1010307EB91
:106FF000C3014A68B2427FF44DAF16E708B540F6C8
:10700000CC53C2F200031A5C40F6C821C2F2000160
:107010004FF04C0000FB0210436AD3F1010238BF6D
:10702000002242634FF00001C1630164416400F13A
:107030001000FDF7ABF808BD2DE9F84F81468A46F0
:1070400040F6CC53C2F200031A5C40F6C820C2F2EC
:1070500000004FF04C0404FB020404F148064FF01A
:1070600001084FF0000740F6882BC2F2000B3546AE
:1070700040463146F9F7E6FD30B14FF002003146A7
:10708000F9F7E0FDBDE8F88FBAF1000F05D14846E9
:107090004146FCF761FC032827D0256C75B15846A2
:1070A000A168E26BA8470546B0F1FF3F14D06064C9
:1070B000484659462A46FCF78FFC0EE0616CA568ED
:1070C0008D4228BF0D464846E16B2A46FCF784FCFA
:1070D000E36B5A19E26300E03D46606CA1688842A8
:1070E0003CBFE7632764451B656438463146F9F7C2
:1070F000A9FD0228BBD0BDE8F88F00BFF8B5054652
:107100000E46174640F6CC53C2F200031A5C40F616
:10711000C820C2F200004FF04C0404FB02044FF000
:107120000000FCF70FFCE76326644FF00001616488
:1071300028464FF00101FFF77FFF4FF00100FCF7F9
:1071400001FCF8BDF8B505460F46164640F6CC538F
:10715000C2F200031A5C40F6C820C2F200004FF0F1
:107160004C0404FB0204A168B1420DD245F69C43D5
:10717000C2F200039F4207D346F29C42C2F20002D1
:10718000974201D2F9F75AFD4FF00000FCF7DAFB05
:10719000E7634FF000002064666428464FF0010169
:1071A000FFF74AFF4FF00100FCF7CCFBF8BD00BF32
:1071B00008B5FCF789FC08BD70B586B005460C46DD
:1071C000164602A8FAF702FC01462EB102A82A468A
:1071D000234600F0A5FD07E04FF00103009302A84D
:1071E0002A46234600F04EFE06B070BD70B58AB048
:1071F0000378212B00F0938004D86BB1012B40F071
:10720000D88186E0A12B00F0A781C02B00F0B481CB
:10721000802B40F0CE8195E04178052903D00929E3
:1072200040F0CA8146E0408840F6C952C2F20002EE
:107230001378022B02D0032B33D118E000F1FF3179
:107240008AB27E2A30D8C0B240F6DC53C2F20003C4
:1072500018704FF00201FCF761FE40F6C950C2F20F
:1072600000004FF0030101704FF00100C3E170B95D
:1072700040F6DC52C2F20002107040F6C950C2F271
:1072800000004FF0020303704FF00100B3E17F28CC
:107290000DD840F6DC51C2F2000108704FF0010039
:1072A000A9E14FF00200A6E14FF00200A3E14FF088
:1072B0000200A0E1827840F6C953C2F200031978B7
:1072C000022923D972B940F6C953C2F200034FF024
:1072D000030119704FF001000146FFF7D1F94FF09B
:1072E000010088E1012A18BF022040F0848140F6A5
:1072F000C950C2F200004FF0040202704FF00000CB
:107300000146FFF7BDF94FF0010074E14FF00200B4
:1073100071E140780B280CBF012002206BE18388CB
:10732000032B00F24C8140F6A854C2F2000404EB97
:10733000C3035B68002B00F045819847002808BF15
:10734000022058E142781AB1062A40F03E8121E03D
:10735000C18802291BD14FF00000ADF8040040F6AF
:107360009852C2F2000212680346517E61F3000394
:10737000ADF80430127E62F341030AA921F8243DDE
:107380004FF00202FFF7DEFE4FF0030033E14FF053
:10739000020030E18278C1888CB2C378022B2ED0F3
:1073A000032B3DD0012B40F0D48040F62C55C2F287
:1073B0000005284649F22071C0F601014FF0120283
:1073C0000FF0BCF840F69850C2F2000001688A89BC
:1073D0002A81CB896B81088AA8818A7C2A71CB7C1F
:1073E0006B71097DA9714FF000002946122C34BF42
:1073F00022461222FFF7A6FE4FF00300FBE040F604
:10740000E452C2F2000211814FF00000506046F6D3
:10741000ED41C0F60001FFF771FE4FF00300EAE016
:10742000D2B940F62C54C2F2000404F1020049F231
:107430009C61C0F601014FF002020FF07FF84FF09F
:10744000040222704FF0030565704FF000002146E2
:10745000FFF778FE2846CEE0012A06D140F6985381
:10746000C2F20003196809682FE0022A06D140F62B
:107470009852C2F200021068416826E0032A06D141
:1074800040F69853C2F20003196889681DE002F0C3
:107490000F0022F00F03102B08D15A4B19688842B5
:1074A0000EDA594A52F8300001680EE0202B07D15D
:1074B000032805D8554951F8300008B1016804E0A7
:1074C000EE2A04D04FF0020095E009B93EE05049A1
:1074D000B1F1FF3F40F0888001A84FF020014FF04C
:1074E0000102FFF769FE0AAD2A184FF0000002F80A
:1074F000240C01A978E000F10206428003F10102A8
:10750000134611F8015F5DB100F10400758002F1CE
:10751000010311F8012F002A6FD101E04FF00003A1
:1075200040F62C51C2F200014FF003054D7003F1FB
:1075300001034FEA4303DAB20A704FF00000A2429F
:1075400028BF2246FFF7FEFD284654E04FF0020018
:1075500051E04FF002004EE08388032B38D840F60C
:10756000A854C2F2000404EBC3035B689BB39847C2
:10757000002808BF02203EE04378212B2ED1C1888D
:1075800040F6E453C2F2000319814FF000025A6042
:107590008088042825D1104646F6CD01C0F60001AA
:1075A00040F6E452C2F20002FFF7A8FD4FF00300DC
:1075B00021E04FF002001EE04FF002001BE04FF010
:1075C000020018E04FF0020015E04FF0020012E058
:1075D0004FF002000FE04FF002000CE04FF002000D
:1075E00009E04FF0020006E00A78002A96D0094828
:1075F0004FF000037FE70AB070BD1E2B7FF47BAF16
:107600008EE700BFE00D00206C0D0020A80D0020CB
:10761000809601082C0D002010B50446436993B1F3
:107620004FF00000606140F6C951C2F200010A78D3
:10763000032A08D140F6DC53C2F2000318784FF059
:107640000301FCF76BFC206958B34FF00000206188
:10765000E06040F6A451C2F20001087040F68C517F
:10766000C2F200014FF00802FFF7A2FD082853D133
:1076700040F68C52C2F20002137813F0800F06D14C
:1076800040F68C50C2F20000C188002944D140F677
:107690008C50C2F200004FF000010A46FFF7A6FD31
:1076A0002DE0E168002937D04FF00000E06040F69F
:1076B000A452C2F20002137840F62C51C2F200012B
:1076C000C3F14002FFF774FD034628B340F6A4500F
:1076D000C2F2000001785A18D2B2027040F68C5300
:1076E000C2F20003D888904216D140F68C50C2F204
:1076F000000040F62C51C2F20001FFF777FD01288F
:1077000004D0022808D1FCF745F910BD4FF0000065
:1077100001460246FFF716FD10BD00BF08B540F652
:10772000F053C2F200031B693BB14FF0000140F679
:10773000F052C2F200025269984740F6F050C2F28D
:1077400000004FF00001017041608160C160016183
:10775000416108BD40F6F050C2F20000816149F27B
:10776000CC71C0F601018A5C42778377037F6FF3A7
:10777000070303774FF000014162704730B583B0D3
:1077800040F6F054C2F200042070089D6560099D27
:10779000A5600A9DE5600B9D25610C9D65619DF8C6
:1077A000184000949DF81C400194FFF7D3FF03B0EC
:1077B00030BD00BF40F6F053C2F200035B6AB3F184
:1077C000FF3F09D140F6F051C2F200014FF0000333
:1077D0004B624FF0010070473F2B0BD840F6F05240
:1077E000C2F20002106AC15403F1010353624FF068
:1077F000010070474FF00000704700BF704700BFA6
:1078000070B540F6F054C2F2000404F1180049F2D9
:107810004471C0F601014FF007020EF08FFE4FF0E9
:10782000000049F2D071C0F60101FFF7AFF947F649
:107830007526C0F600064FF0000049F27C71C0F6D4
:1078400001013246FFF7C0F949F2E875C0F60105BB
:107850004FF0010029463246FFF7B6F92869FFF7D5
:10786000DFF984F8280040F65C60C2F200004FF0B7
:10787000070147F68502C0F600024FF00003FCF74F
:1078800065FC70BD38B540F69063C2F200034FF05E
:1078900001021A7040F6F054C2F2000494F8280075
:1078A0004FF000010A46FFF74DFC606868B140F6F2
:1078B000F054C2F200044FF0FF356562636820782F
:1078C00061699847616A0029F7D040F6F050C2F22A
:1078D00000004FF000024262836833B140F6F0517D
:1078E000C2F2000108784969984738BD2DE9F04F88
:1078F00083B0804643680BB9806828B14FF000011F
:10790000C8F80810FFF7BEFFD8F80C20002A45D0B1
:107910004FF00003C8F80C30D8F8000040F61C61A6
:10792000C2F200014FF04002FFF742FC814640F6F0
:10793000F050C2F20000C16800292FD0B9F1000F49
:107940002CD040F6F054C2F2000440F61C66C2F29D
:1079500000064FF0000509F1FF3B0BF0010B20780A
:10796000715D2A466369E768B84705F1010AD145A8
:1079700070D113E0207816F80A102A466369E76888
:10798000B8470AF1010A207816F80A102A466369F6
:10799000E768B8470AF1010AD145EBD1D8F81420BD
:1079A000002A54D04FF0000440F69063C2F2000366
:1079B0001C70C8F8144040F66C60C2F20000FEF77C
:1079C00047FD40F6F050C2F20000446241680029D1
:1079D00036D040F6F055C2F2000540F69464C2F28B
:1079E00000042C622C46656A6268207861699047C1
:1079F000636A9D42F7D11DB3D8F8000040F6946148
:107A0000C2F200012A46FFF79DFB4FF000000090F4
:107A1000019040F66C60C2F200004FF04B014FF055
:107A2000FF0247F68503C0F60003FEF7B7FD0EE040
:107A300040F6F052C2F2000210785169984706E011
:107A400040F6F051C2F200018B68002BF0D103B078
:107A5000BDE8F08FBBF1000F8CD0207816F80A102B
:107A60002A466369E768B8470AF1010AD14581D11E
:107A700094E700BF10B544780378212B02D0A12BE6
:107A80001BD10EE0202C04D0222C14BF002001209A
:107A900010BD072A14D10D480EF050FD4FF0010023
:107AA00010BD212C0FD14FF0000008494FF0070204
:107AB000FFF748FB4FF0030010BD4FF0000010BD72
:107AC0004FF0020010BD4FF0000010BD080E002066
:107AD00008B540F69063C2F20003187870B940F61A
:107AE000F051C2F200014A6A72B940F6F053C2F294
:107AF000000393F82800FFF781FA08BD40F65C60A8
:107B0000C2F20000FCF742FB08BD00BF49F24C7016
:107B1000C0F60100704700BF70B4037801298CBF24
:107B20004478002402298CBF85780025DCF8000009
:107B300048B34FEA930649F61400C0F60100365CDC
:107B400016704FEA031343EA141303F03F031B5C60
:107B50005370012907D94FEA840444EA951303F0CE
:107B60003F04205C01E04FF03D009070022907D9EE
:107B700005F03F0549F61403C0F60103E95C01E096
:107B80004FF03D01D17070BC704700BF82B04FF024
:107B900009010CE00191019B03F1FF32019233B125
:107BA00000BF019B03F1FF320192002BF8D100F1DD
:107BB000FF30B0F1FF3FEDD102B0704770B4C4B2F6
:107BC0004FEA102049F6A806C0F6010649F6A815A6
:107BD000C0F6010511F8013B1AB94BB944EA00207F
:107BE0000BE06340F45C4440E85C013AF2D1F5E715
:107BF0006340F45C4440E85CECE770BC704700BF55
:107C000010B444F6FB43C0F2861311F8014B02B9DD
:107C1000ACB380EA04404FEA400010F0807F18BF08
:107C200058404FEA400010F0807F18BF58404FEA9C
:107C3000400010F0807F18BF58404FEA400010F01D
:107C4000807F18BF58404FEA400010F0807F18BF77
:107C500058404FEA400010F0807F18BF58404FEA6C
:107C6000400010F0807F18BF58404FEA400010F0ED
:107C7000807F18BF5840002AC7D0013AC5D120F0F4
:107C80007F4010BC704700BF82B001909DF8063065
:107C90004FF0000063F307009DF8052062F30F200A
:107CA0009DF8042062F317409DF8072012F0800F22
:107CB00014BF63F07F0103F07F0161F307004FEA17
:107CC0004201CAB262F31F6013F0800F18BF42F086
:107CD000010262F31F6002B0704700BF84B0C0F3BE
:107CE00007438DF80C30C0F307228DF80D20C3B286
:107CF0004FEA10604FEA500210F0010F14BF63F01A
:107D00007F0103F07F018DF80E1013F0800F18BF74
:107D100062F07F028DF80F20039804B0704700BF17
:107D20002DE9F04F83B005460F4614461E460192DA
:107D300001F1FF3313F1050F44D8032E43D9A6F107
:107D40000400C0F380080DF1040C2846FFF7E4FEA0
:107D500005F10305A7F1030104F10404A6F10406EB
:107D6000A7F1040717F1050F67D92CE00DF1040CFA
:107D7000284639462246FFF7CFFE05F1030B5D4644
:107D8000A7F1030104F1040A5446A6F104094E4682
:107D9000A7F1040717F1050F15D80F460DF1040CD4
:107DA00058465246FFF7B8FE0BF10305A7F1030151
:107DB0000AF10404A9F10406A7F1040818F1050F5B
:107DC00059D900E0FFE799B396B30DF1040C2846AA
:107DD0006A46FFF7A1FE022E11D0032E02D0012E1B
:107DE00026D11AE0019929B19DF8002022704FF0A8
:107DF000010301E04FF0000304F1010401E04FF042
:107E00000003019830B102A9CA1812F8080C2070BA
:107E100003F1010304F1010401E04FF000030199B3
:107E200021B102AAD31813F8080C207004F1010440
:107E30000199601A03B0BDE8F08F0F46032EC2D936
:107E4000B8F1000F92D00DF1040C28462246FFF73E
:107E500063FE05F10305A7F1030104F10404A6F193
:107E60000406A7F1040717F1050FACD80F46032E3F
:107E70003FF67CAFA7E7A7F10307032E3FF676AFE7
:107E8000A1E700BFF0B49DF81040ECB14FEA410704
:107E90009F421CD2DD1B1DD056194FF030046FEAF3
:107EA0000203F31803F0010302F8014BB24240F061
:107EB000928007E0134603F8014B547003F101026E
:107EC000B242F7D13B4607E04FF0000504E04FF027
:107ED000000501E04FF0000500293CD003F1FF341C
:107EE000002B3AD000F1010341182846521B04F13F
:107EF000FF3515F0020F10D032E0A4F1020603F1B5
:107F000001031F46012C29D03446B44613F8016CF6
:107F10004FEA1616092E42D944E01E4613F8015CBA
:107F20004FEA1515092D8CBF37353035155414B966
:107F300000F1010012E013F8016C06F00F05092DA5
:107F40008CBF373530351618757000F1020528469C
:107F50008B42D2D102E0284600E02846F0BC7047B0
:107F60001E4613F8015C4FEA1515092D94BF3035F4
:107F700037351554002CDBD013F8016C06F00F05D3
:107F8000092D94BF303537351618757000F1020091
:107F90008B42E3D003F10103A4F10204BDE706F133
:107FA000300601E006F137065655BCF1000FBFD090
:107FB00013F8016C06F00F06092E94BF30363736E1
:107FC0001018467005F102008F42C7D003F101037B
:107FD000A4F10204A1E7002B3FF46CAF02F8014BBF
:107FE000B2427FF467AF6DE7DCF8143093F84520B8
:107FF00083F84420DCF8141091F8463081F84530BD
:10800000DCF8141091F8472081F84620DCF8143091
:1080100083F84700704700BFDCF8143093F847003E
:1080200093F8462083F84720DCF8141091F8453087
:1080300081F84630DCF8141091F8442081F845208E
:10804000704700BF45F29442C2F2000213684CF63A
:108050000001C0F60101C85CC918497803F10203A8
:10806000136041EA00207047DCF80430DCF8082097
:1080700002EBD300CCF8080003F007014FF0010336
:1080800003FA01F2CCF80420704700BF2DE9F04F4D
:1080900083B004468A4693461E46CDF804C04FF08E
:1080A0000007B846B9463DE025463046D04703466E
:1080B00000283DD0B9F1000F0CD1202829D0092883
:1080C00029D00A2829D00D2829D0022D4FF00109E6
:1080D00088BF0225A3F13002D1B2092910D9A3F13A
:1080E0004100C1B2052903D8A3F13703D9B207E093
:1080F000A3F16102D0B205281AD8A3F15703D9B26F
:108100004FEA0717FCB241EA040708F101082C46C0
:1081100006E02C4604E02C4602E02C4600E02C460B
:108120003046D847FF2CBFD004F1FF35002CBCD11E
:10813000DDF804C03846FFF757FF019B5A69D8F1B4
:10814000010838BF4FF0000882F8508003B0BDE846
:10815000F08F00BF42F6B403C2F200031B684B630A
:108160004BB19A68824209D0DB684B631BB19A68B5
:108170008242F9D102E04FF01E0070474FF000003C
:10818000704700BF884204D8884234BF02200020D4
:1081900070474FF001007047D0F80431D0F800214B
:1081A000934214BFC05C0020704700BFD0F8043178
:1081B000FF2B14BF01330023C0F80431704700BF08
:1081C00010B4DCF81420D16C0B46044658B14FEAC9
:1081D000016343EA116301F47F4043EA002301F4A1
:1081E0007F0143EA1123DCF8040030B199B24FEA71
:1081F000134060F30F0361F31F435CB94FEA03615F
:1082000041EA136103F47F4041EA002103F47F0354
:1082100041EA1323D36410BC704700BFDCF8003080
:10822000FA2B05D840F6D862C2F20002D05C704743
:108230004FF00000704700BFDCF8003003F101038D
:10824000CCF80030DCF8140090F8512002F1010263
:1082500080F85120704700BF70B404460846A1B1B1
:1082600099188C4211D22518AA420ED294423ABFD4
:10827000C4EB0206F6B20026A94205D20019821A02
:10828000D31AF118C8B200E0304670BC704700BF86
:10829000F0B583B042F6BC03C2F200034FF008020F
:1082A0001A7042F6A400C2F2000004683CB31546FE
:1082B00042F6BC07C2F200074FF0000621680B68C7
:1082C00073B10DF107000DF1060198479DF8070005
:1082D0009DF8061032463B78FFF7BEFF4519EDB218
:1082E0006468002CEAD142F6BC02C2F200021078A7
:1082F000A84204D242F6BC01C2F200010D7042F65F
:10830000BC03C2F200034FF007025A7042F6D804D1
:10831000C2F2000424683CB3154642F6BC07C2F220
:1083200000074FF000062068036873B10DF10700E5
:108330000DF1060198479DF807009DF8061032469A
:108340007B78FFF789FF4519EDB26468002CEAD10C
:1083500042F6BC01C2F200014A78AA4204D242F6B7
:10836000BC00C2F20000457042F6BC03C2F200033A
:108370004FF00001997045F29044C2F20004246865
:1083800034B30D4642F6BC07C2F200070E4622681F
:10839000136873B10DF107000DF1060198479DF8C0
:1083A00007009DF806103246BB78FFF755FF4519C8
:1083B000EDB26468002CEAD142F6BC00C2F20000C3
:1083C0008178A94204D242F6BC02C2F20002957042
:1083D00042F6BC03C2F200034FF00000D87045F231
:1083E0009C44C2F20004246834B3054642F6BC073C
:1083F000C2F20007064621680A6872B10DF1070053
:108400000DF1060190479DF807009DF806103246D1
:10841000FB78FFF721FF4519EDB26468002CEAD123
:1084200042F6BC03C2F20003D878A84204D242F656
:10843000BC01C2F20001CD7003B0F0BD45F28C4327
:10844000C2F2000319684CF60000C0F60200401AA0
:10845000704700BF034610B182688A4218D042F6C6
:10846000B803C2F20003186860B182688A4203D17F
:108470000BE083688B420AD040680028F9D14FF0A6
:10848000000305E04FF0000302E0034600E003466E
:108490001846704710B541F61874C2F200044FF444
:1084A000117303FB0044D4F80811B1F1FF3F03D06E
:1084B000D4F8042191420DD123689A6A4FF0FF014C
:1084C0009047002834D0D4F8080100F10100C4F826
:1084D000080110BD91422BD86318197945F29842D2
:1084E000C2F2000213787BB9FD290FD923689A6A7A
:1084F0004FF0FE019047D8B145F29840C2F200001B
:108500004FF00101017010BD6FEA01012268936A0A
:10851000C9B2984760B1D4F8080100F10100C4F86D
:10852000080145F29841C2F200014FF000020A70C2
:1085300010BD00BF70B5064641F61875C2F20005C1
:108540004FF4117404FB00F42B194FF00101C3F830
:108550000C112A59936998472859016A304688476F
:1085600070BD00BF38B541F61871C2F200014FF47A
:10857000117202FB00F28C18D4F80831D4F80451BF
:10858000AB420DD08958E3188A6A1979904738B1FF
:10859000D4F80801FF2814BF01300020C4F80801F6
:1085A00038BD00BF38B541F61874C2F200044FF46C
:1085B000117202FB00F2A318D3F80451D3F808118A
:1085C0008D4206D14FF00001C3F80C11A2589369F7
:1085D000984738BD10B441F61873C2F200034FF447
:1085E000117202FB003000F58870D0F80031FF2BCB
:1085F00014BF5A1C0022D0F80441A2421CBFC1542F
:10860000C0F8002110BC7047F8B545F28C44C2F2A6
:10861000000424688568C768466807FB056045183C
:10862000611911D2CE180B48864210D8012B04D103
:10863000635D13704FF00000F8BD10461A460DF050
:108640007DFF4FF00000F8BD4FF01F00F8BD4FF068
:108650001F00F8BD01C8020810B542F6A803C2F217
:1086600000031A8841F61870C2F200004FF411742A
:1086700004FB0204F8F78AFB4FF0FF31C4F8101234
:108680004FF00003C4F8183204F58874F8F788FB3B
:1086900010BD00BFF8B506464FF0020303704BF65D
:1086A0000000C0F60100C28B4FF6FF718A4221D054
:1086B0003F4C404BA34222D203F110033E4DEF1A30
:1086C0004FEA17124FF6FF7502F1010002F00107A1
:1086D0001C46D98BA9424FD115E01C46D98BA94223
:1086E00011D002F1010203F110031C46D98BA942FB
:1086F00057D108E04BF60004C0F6010403E04BF646
:108700000004C0F601044FF6FF7021464FF00D0241
:10871000FFF754FA4FF6FF73984208BF0020E28932
:1087200082421BD0A4F110054BF60000C0F60100F8
:1087300085421AD34FF6FF7029464FF00D02FFF71E
:108740003DFA4FF6FF71884208BF002034F8024C12
:1087500084420AD12C464FF0010201E04FF00002A2
:10876000607BFF2806D1327004E04FF002033370C3
:108770004FF000042046F8BD4FF0000202F1010264
:1087800003F110038242BED0002FA6D01C46D98B25
:10879000A942B8D002F1010203F1100382429CD138
:1087A000B1E702F1010203F11003824295D1AAE779
:1087B00000C0010800B801080FC0010870B5C0B0C2
:1087C00005460E4620F0FF04684621464FF0400261
:1087D000F8F744FA00AB53FA85F031464FF0100237
:1087E0000DF0ACFE684621464FF48072F9F7DEFDCD
:1087F00040B070BD38B5054641F61874C2F20004A9
:108800004FF4117303FB0044D4F81C02FDF72EFB58
:1088100042F6A800C2F200000188A94206D142F641
:10882000A803C2F200034FF6FF721A804FF0000057
:10883000C4F81C0238BD00BF10B54FF00000FBF7B4
:10884000FDFC42F6A403C2F200031C6834B12068A8
:10885000016901B188476468002CF8D110BD00BFE0
:1088600010B50446072822D8032894BF4FF4FA73A2
:10887000322303FB01F142F66003C2F2000303EB73
:10888000C000416059B1FDF7BFFE002808BF0120BC
:1088900042F66003C2F2000343F8340010BD42F612
:1088A0006001C2F200014FF0000241F8342010BD17
:1088B00038B5044607284BD842F66003C2F20003DD
:1088C00003EBC00045680DB342F66001C2F200013F
:1088D00051F83420D2B1FDF797FE002808BF0120DF
:1088E00042F66003C2F2000353F83410401A854286
:1088F0000BD242F66003C2F2000303EBC4024FF056
:108900000005556043F8345000E02D1A05F10405C8
:108910004CF6CD41CCF6CC41A1FB05204FEA9003AB
:10892000032C0AD803F1630348F21F51C5F2EB117F
:10893000A1FB03324FEA521038BD03F109014CF696
:10894000CD42CCF6CC42A2FB01304FEAD00038BD7C
:108950004FF0000038BD00BF70B506466446DCF835
:1089600014305D6AFDF750FE6169CA6A0AB9C862CF
:1089700008E0801A05EB850506FB05F6B04224BF2A
:108980000020C8626369D96AD1F1010038BF0020B4
:1089900070BD00BF10B541F61873C2F200034FF46A
:1089A000117404FB003303F58873D3F80841002CDD
:1089B0005FD15AB14FF0FF31C3F8001140F6D463D4
:1089C000C2F200034FF00000187010BDD3F8002170
:1089D000B2F1FF3F06D1FF294BD14FF00002C3F89F
:1089E000002110BDFF291ED140F6D461C2F2000162
:1089F0004FF000040C70012A10D94FF00102C3F8A7
:108A0000082141F61873C2F200034FF4117101FB03
:108A10000030D0F81C02FCF7E7FF10BD4FF000005B
:108A2000C3F8000110BDFE2907D140F6D463C2F29D
:108A300000034FF00101197010BD40F6D460C2F27E
:108A40000000007848B16FEA0101C9B240F6D46075
:108A5000C2F200004FF000040470FF2A05D89954B8
:108A600002F10102C3F8002110BD4FF0FF32C3F83C
:108A7000002110BD08B541F61873C2F200034FF48F
:108A8000117202FB0030D0F80811D0F8043100F167
:108A9000040099420AD94FF00002C0F8002142F6C2
:108AA0001410C2F200004068FCF79EFF08BD00BF32
:108AB000F8B5654645F2A043C2F200031A7802F009
:108AC0000804E7B227B1DCF8146096F8516007E0BB
:108AD00012F0110F06BFDCF8147097F852600026F0
:108AE00001EB800411F8203003F0070302F02002AC
:108AF000D7B23FB111F8202002F00807FAB20AB14C
:108B00004FEA430311F820704FEA9712012A08D068
:108B1000022A10D111F82000C0F3011101FB0667F1
:108B20000BE06F6997F8517011F82020C2F3011023
:108B300000FB077701E04FF00007042B50D8DFE877
:108B400013F0C60140003B002200050045F29441AD
:108B5000C2F200010B684CF60007C0F60107FA18D4
:108B600092F802E0D0784FEA006040EA0E40527876
:108B700040EA0220FF5C03F104030B603843FFF777
:108B8000ADF868602CE045F29442C2F2000213682E
:108B90004CF60000C0F60100C11891F801C0C05C9D
:108BA0004FEA004040EA0C208978084303F10303B0
:108BB00013603F186F6013E0FFF744FAC2196A6050
:108BC0000EE045F29443C2F2000318684CF600012F
:108BD000C0F601010A5CBF186F6000F10100186067
:108BE000637803F0070345F2A040C2F20000017869
:108BF00001F02002D7B237B1607800F00801CAB2A4
:108C00000AB14FEA430367784FEA9710012807D06B
:108C100002280ED16178C1F3011202FB06670AE057
:108C20006F6997F851006178C1F3011202FB0007E8
:108C300001E04FF00007042B50D8DFE813F04801A3
:108C400040003B002200050045F29441C2F20001C1
:108C50000B684CF60007C0F60107FA1892F802E01C
:108C6000D0784FEA006040EA0E40527840EA022095
:108C7000FF5C03F104030B603843FFF72FF8A86093
:108C80002CE045F29442C2F2000213684CF6000058
:108C9000C0F60100C11891F801C0C05C4FEA004065
:108CA00040EA0C208978084303F1030313603F185E
:108CB000AF6013E0FFF7C6F9C219AA600EE045F2F3
:108CC0009443C2F2000318684CF60001C0F601019B
:108CD0000A5CBF18AF6000F101001860A37803F0D0
:108CE000070345F2A040C2F20000017801F0200223
:108CF000D7B237B1A07800F00801CAB20AB14FEA82
:108D00004303A7784FEA9710012807D002280ED115
:108D1000A178C1F3011202FB06670AE06F6997F8B8
:108D20005100A178C1F3011202FB000701E04FF0EE
:108D30000007042B50D8DFE813F0CA0040003B00C6
:108D40002200050045F29441C2F200010B684CF686
:108D50000007C0F60107FA1892F802E0D0784FEA4F
:108D6000006040EA0E40527840EA0220FA5C03F1CB
:108D700004030B601043FEF7B1FFE8602CE045F2FE
:108D80009442C2F2000213684CF60000C0F60100E3
:108D9000C11891F801C0C05C4FEA004040EA0C20C5
:108DA0008978084303F1030313603F18EF6013E071
:108DB000FFF748F9C219EA600EE045F29443C2F2A7
:108DC000000318684CF60001C0F601010A5CBF18E8
:108DD000EF6000F101001860E37803F0070345F24B
:108DE000A040C2F20000017801F02002D0B230B100
:108DF000E17801F00802D0B208B14FEA4303E1780C
:108E00004FEA9112012A02D0022A0FD108E06E69BE
:108E100096F85100E278C2F3011101FB000607E069
:108E2000E078C0F3011101FB066601E04FF0000697
:108E3000042B4CD8DFE803F04B031318300045F245
:108E40009443C2F2000318684CF60001C0F6010119
:108E50000A5CB6182E6100F101001860F8BDFFF73A
:108E6000F1F882192A61F8BD45F29442C2F200027B
:108E700013684CF60000C0F60100C1184C78C05CC5
:108E80004FEA004040EA04208978084303F10303D5
:108E9000136036182E61F8BD45F29441C2F200010C
:108EA0000B684CF60004C0F60104E2189678D078FE
:108EB0004FEA006040EA0640527840EA0220E25C55
:108EC00003F104030B601043FEF708FF2861F8BDAF
:108ED00008B503281ED8DFE800F0020910174AF68B
:108EE0004040C0F601000FF01BF908BD4AF64440AF
:108EF000C0F601000FF014F908BD4AF65840C0F65C
:108F000001000FF00DF908BD4AF67040C0F60100EF
:108F10000FF006F908BD00BF2DE9F8430546884665
:108F200016461F4642F6A803C2F20003B3F80090AB
:108F300045F69810C2F20000016842F6A002C2F2A3
:108F400000021368994201D0FFF786FB072D6ED807
:108F50001F2E6CD841F61874C2F200044FF4117041
:108F600000FB094442F61410C2F200004FF0000169
:108F7000FCF7DAFA217965F34711072D14BF0025B4
:108F80000125AA1962F304012171CBB22DB184F835
:108F9000058043444FF0020001E04FF0010006F16C
:108FA000FF3E5FFA8EFE46B302463F1A0EF0010CFA
:108FB0003D5C04F1040635545B1902F101020EF127
:108FC000FF31C9B2FF2934D114E0BD5C04F10406BD
:108FD000B5545B1902F1010201F1FF3101F0FF010B
:108FE000BD5CB5545B1902F1010201F1FF31C9B258
:108FF000FF29EAD100F1010070442218137100F139
:109000000100C4F804014FF0FF33C4F808312168AF
:109010000B6A42F6A800C2F2000000789847FCF7FD
:10902000B1FC42F61410C2F20000FCF78BFBBDE865
:10903000F8834FFA8CF5002DC7D0BD5C04F104060F
:10904000B5545B1902F1010201F1FF31C9B2FF29E8
:10905000BBD1CFE738B5054642F62804C2F200047A
:109060002046FCF76FFBF8F7ABFD2846FCF752FEF5
:1090700020464FF00001FCF757FA38BD10B586B016
:109080000DF10700FFF706FB044618B19DF8073005
:1090900023B90FE04BF60004C0F60104E2894FF655
:1090A000FF7082422BD04CF20001C0F601018C42CD
:1090B00009D32AE0304821464FF00D020CF0E8FDBC
:1090C000002848D0EAE74FF6FF724CF20000C0F6E5
:1090D00001006FEA0403C118C1F3001104F1100488
:1090E000E389934239D10AE004F110031C46D9897F
:1090F000914204D003F11004E389934239D14CF238
:109100000002C0F60102944207D34BF60004C0F6F9
:10911000010420462146F9F7DFF802A816494FF06E
:109120000D020DF00BFA4FF0FF008DF815004FF611
:10913000FF7002A94FF00D02FEF740FD4FF6FF71E0
:10914000884212BFADF816000021ADF81610204677
:1091500002A9FFF733FB06B010BD8442D5D2002927
:10916000C2D004F11004E1899142C8D08442BBD33B
:10917000CBE78442B8D3C8E7DE0E00202DE9F04FDC
:1091800085B0884691461D46E2464FF000042646CB
:109190004FF0020B2DE007462846C047034670B348
:1091A00024B9202822D0092802D11FE0012C05D1A2
:1091B0002B2B0DD02D2B0DD05C4601E0022C01D1C4
:1091C0002E2B09D0A3F13002D0B2092817D805E020
:1091D0005C4603E05C4601E04FF003040E2E05D828
:1091E00004A98A1902F8103C06F101062846C8476E
:1091F0003846FF28CFD000F1FF370028CCD1012C12
:1092000012D98EB104ACA6194FF0000406F8104C28
:10921000684621460CF096FDDAF81410C864DAF8B6
:10922000142082F8504005E0DAF814304FF00100C5
:1092300083F8500005B0BDE8F08F00BF10B586B0D0
:109240004CF60000C0F601003449F9F745F8002853
:109250004BD1334B334A9A421DD24CF60001C0F633
:1092600001010B68B3F1FF3F42D102F104032E4A22
:10927000D01A20F00302991812F0040F3FD11846BB
:109280008B420CD003F104021B68B3F1FF3F3ED0C8
:109290004FF0000031E04CF60000C0F601004CF643
:1092A0000003C0F60203984225D10DF10700FFF735
:1092B000F1F90446B0B19DF80710022912D002A8B6
:1092C00021464FF010020DF039F99DF815006FF3AB
:1092D00007008DF81500204602A9FFF76FFA4FF03E
:1092E00001000AE04FF0010007E04FF0000004E049
:1092F0004FF0000001E04FF0000006B010BD18462E
:1093000003F104030268B2F1FF3FB8D0C0E702F1F5
:1093100004031068B0F1FF3FB1D0B9E7FFC70208FE
:1093200000C8020800C8010803C802082DE9F007B8
:10933000034600284ED040F20022C0F6000292F808
:10934000469092F8470042F6BC04C2F2000494F83A
:10935000018092F848C0257842F60012C2F200025D
:109360001468177A567AD2F804A04FF000021A70E7
:1093700083F801909870DA704FF0FB0018714FF08D
:10938000060983F805909D7183F807804FF0040863
:1093900083F8088083F8098083F80AC0DD721A73A5
:1093A0004FEA14255D739C73DF731E745A744FF07B
:1093B0001D029A744FF00202DA744FF0FE021A7521
:1093C0005A754FEA1A229A7583F817A018764FF04B
:1093D0000F00587629B142F6BC03C2F200031A68A6
:1093E0000A60BDE8F0077047034628B142F6001254
:1093F000C2F200021068186042F60011C2F20001C9
:10940000087A704770B505460E4614464FF00000C6
:109410002946FFF71FF808B1F7F710FC42F6B8032A
:10942000C2F200031A686260A56026601C6070BD0D
:1094300008B539B142F6A403C2F200031A684260CB
:1094400018601EE042F6A403C2F200031B688342C8
:109450000FD1586842F6A401C2F20001086010E082
:1094600042685A6041605A688242F9D013461BB97B
:1094700007E033B14FF000015A688242F0D0134642
:10948000F5E7FEF705FF08BD08B539B142F6D80388
:10949000C2F200031A68426018601EE042F6D80368
:1094A000C2F200031B6883420FD1586842F6D8010C
:1094B000C2F20001086010E042685A6041605A68D8
:1094C0008242F9D013461BB907E033B14FF00001D7
:1094D0005A688242F0D01346F5E7FEF7D9FE08BD80
:1094E00008B539B145F29043C2F200031A684260F0
:1094F00018601EE045F29043C2F200031B688342ED
:109500000FD1586845F29041C2F20001086010E0A6
:1095100042685A6041605A688242F9D013461BB9CA
:1095200007E033B14FF000015A688242F0D0134691
:10953000F5E7FEF7ADFE08BD08B539B145F29C432D
:10954000C2F200031A68426018601EE045F29C43B4
:10955000C2F200031B6883420FD1586845F29C4158
:10956000C2F20001086010E042685A6041605A6827
:109570008242F9D013461BB907E033B14FF0000126
:109580005A688242F0D01346F5E7FEF781FE08BD27
:1095900001604360826042F6B403C2F200031A68BD
:1095A000C2601860704700BF70B582B006464FF0C9
:1095B00000038DF807300D4601B10B7042F6A40090
:1095C000C2F20000046874B121684B6843B13046B0
:1095D0000DF107012A46984710B19DF8070011E0E8
:1095E0006468002CF0D1072E03D83046FAF76AFEE3
:1095F00008E02DB14FF005022A704FF0000001E0A5
:109600004FF0000002B070BD70B582B006464FF05A
:1096100000038DF807300D4601B10B7042F6A4002F
:10962000C2F20000046874B121688B6843B130460F
:109630000DF107012A46984710B19DF8070019E07F
:109640006468002CF0D1072E0BD83046FAF750FE94
:109650008DF8070010B13046FAF790FE9DF807002C
:1096600008E02DB14FF005022A704FF0000001E034
:109670004FF0000002B070BD70B582B006464FF0EA
:1096800000038DF807300D4601B10B7042F6A400BF
:10969000C2F20000046874B12168CB6843B130465F
:1096A0000DF107012A46984710B19DF8070011E017
:1096B0006468002CF0D1072E03D83046FAF7E8FD95
:1096C00008E02DB14FF005022A704FF0000001E0D4
:1096D0004FF0000002B070BD70B582B006464FF08A
:1096E00000038DF807300D4601B10B7042F6D8002B
:1096F000C2F2000004685CB121688B682BB130466F
:109700000DF107012A46984758B96468002CF3D137
:10971000062E0CDC082E0AD83046F8F73FF88DF8F4
:1097200007009DF80700003018BF012008E02DB1A8
:109730004FF006022A704FF0000001E04FF00000E9
:1097400002B070BDF0B583B005460E464FF0000381
:109750008DF8073042F6D800C2F200000468E4B188
:109760004FF000072168CA681AB128463146904771
:10977000F0B923689B6833B128460DF106010DF15D
:109780000702984700E038469DF8071099B96468C9
:1097900014B10028E6D004E018B9062D0DDC082D20
:1097A0000ED82846314606F085FE4FF0000009E04D
:1097B0004FF0000006E0084604E04FF0060001E02C
:1097C0004FF0060003B0F0BD70B582B005460E46FE
:1097D0004FF000038DF8073012B11946FFF7B2FFC2
:1097E00042F6D800C2F2000004686CB121684B68F0
:1097F000284631460DF10702984710B19DF8070041
:1098000012E06468002CF1D1062D08DC082D09D87F
:1098100028463146F7F7E4FF4FF0000004E04FF030
:10982000060001E04FF0060002B070BD08B54FF031
:10983000000001464FF00102FFF7C6FF08BD00BF60
:1098400070B582B005460E464FF000038DF8073024
:1098500045F29040C2F200000468B4B121684B6840
:10986000284669460DF10702984728B10EB10098C5
:1098700030609DF807000DE064684CB19DF807204A
:10988000002AEBD04FF00F0004E04FF00F0001E092
:109890004FF00F0002B070BD70B582B005460E46A5
:1098A0004FF000038DF8073045F29C40C2F20000F3
:1098B00004689CB121684B68284631460DF10702C7
:1098C000984710B19DF807000DE064684CB19DF811
:1098D0000720002AEED04FF00E0004E04FF00E00FB
:1098E00001E04FF00E0002B070BD00BF70B582B055
:1098F00005460E464FF000038DF8073045F29C40B8
:10990000C2F200000468BCB121688B685BB12846D4
:1099100069460DF10702984728B10EB100983060F2
:109920009DF807000DE064684CB19DF80720002AFF
:10993000EAD04FF0060004E04FF0060001E04FF0DF
:10994000060002B070BD00BF2DE9F04F2DED048B75
:109950008BB007461546914259D289464FF0000B0D
:109960004FF000089FED908B9FED919B6FEA0106F1
:10997000B01800F00106CDF804B0022F4CD150E031
:10998000CDF804B0022F05D15FFA89F001A9FFF7E5
:10999000ADFF04E05FFA89F001A9FFF751FF04EB86
:1099A00044060AA88119A1F1200601F8209C01F8BB
:1099B0001F8C01980BF026FC53EC182B0BF0C0FD0C
:1099C00053EC192B0BF078FC0BF0E2FB83B2FF2B6E
:1099D00028BFFF23B37004F101040A2C04D005F161
:1099E000FF324A450AD14CB104EB44044FF0070062
:1099F0003946E2B202ABFFF78FFA444609F101099A
:109A00004E46CDF804B0022F40F089808DE00BB0B7
:109A1000BDEC048BBDE8F08FC8B201A9FFF710FFC1
:109A200003E0C8B201A9FFF761FF0AAC04F8209D6A
:109A300084F8018001980BF0E5FB53EC182B0BF038
:109A40007FFD53EC192B0BF037FC0BF0A1FB81B21F
:109A5000FF2934BF0B46FF23A3704FF0000404F12D
:109A6000010405F1FF324A450DD10AE004EB44043C
:109A70004FF007003946E2B202ABFFF74DFA444619
:109A800001E0002CF2D109F101094D45BFD9002EAA
:109A90003FF476AFCDF804B0022F05D05FFA89F01D
:109AA00001A9FFF7CDFE04E05FFA89F001A9FFF7F5
:109AB0001DFF04EB44060AA8861906F8209D86F8C7
:109AC000018001980BF09EFB53EC182B0BF038FD36
:109AD00053EC192B0BF0F0FB0BF05AFB81B2FF2972
:109AE00034BF0B46FF23B37004F101040A2C0AD1E2
:109AF00004EB44044FF007003946E2B202ABFFF733
:109B00000BFA444605E005F1FF324A4501D1002C2D
:109B1000EED109F101094D453FF632AF77E75FFA23
:109B200089F001A9FFF78CFE04E05FFA89F001A932
:109B3000FFF7DCFE04EB44000AA90B18A3F1200A8E
:109B400003F8206C03F81F8C01980BF05BFB53ECBF
:109B5000182B0BF0F5FC53EC192B0BF0ADFB0BF0B5
:109B600017FB82B2FF2A28BFFF228AF8022004F1E5
:109B700001040A2C0AD104EB44044FF007003946D3
:109B8000E2B202ABFFF7C8F9444605E005F1FF3049
:109B9000B04201D1002CEED109F101094D453FF64B
:109BA000EFAE34E7AFF300800000000000E06F404C
:109BB000000000000000E03F2DE9F04F95B040F6B6
:109BC000C410FCF7A7F84FF002004FF0000142F676
:109BD000BC03C2F20003DA78FFF7B6FE4FF00100D3
:109BE00000904FF0000BDA46D94607464CF6CD41BF
:109BF000CCF6CC4101914FF07D00FCF78BF88DF84D
:109C00002F90C8464E464C4613E045F0800504F1BF
:109C10000804E4B20CA9725CAA4202D00CABF55461
:109C2000B84606F101069DF82F50002D50D1202E88
:109C30004ED020460DF12F01FFF7B6FC051C18BFD2
:109C4000012504F10102D0B20DF12F01FFF7ACFCA8
:109C500010B145F00205EDB204F10203D8B20DF1E6
:109C60002F01FFF7A1FC08B145F0040504F1030042
:109C7000C0B20DF12F01FFF797FC08B145F00805C0
:109C800004F10401C8B20DF12F01FFF78DFC08B1FA
:109C900045F0100504F10502D0B20DF12F01FFF7D8
:109CA00083FC08B145F0200504F10603D8B20DF19C
:109CB0002F01FFF779FC08B145F0400504F10700DA
:109CC000C0B20DF12F01FFF76FFC00289DD19EE778
:109CD000B8F1000F02D1BAF1000F0CD14FF0020021
:109CE0004946F2B20CABFFF717F94FF03200FCF720
:109CF00011F83E4600E04E4642F6BC00C2F20000BB
:109D00008278B2B1019CA4FB0A014FEA111303EB64
:109D10008305BAEB850F0CD138464946FFF714FE90
:109D20004FF03200FBF7F6FFBBF1000F40F0B780B9
:109D300003E0BBF1000F40F09C8003A849464FF0C0
:109D400020020CF01FFC42F6BC00C2F20000847836
:109D5000ACB34B466FEA09010D1905F0010209F099
:109D6000070607FA06F09DF80C1040EA01058DF889
:109D70000C5003F10103A342C0F2B2801FE014AE05
:109D800006EBD30503F0070007FA00F215F8441CB0
:109D900042EA010605F8446C03F1010314A800EB44
:109DA000D30203F0070107FA01F612F8445C46EA11
:109DB000050002F8440C03F10103A342DFDB4FF07E
:109DC00007004FF011014FF01E0203ABFFF7A4F89C
:109DD0004FF03200FBF79EFF03A849464FF02002E8
:109DE0000CF0D0FB42F6BC04C2F20004E678A6B345
:109DF0004B466FEA0902911901F0010509F00700CD
:109E000007FA00F49DF80C2044EA02018DF80C10CA
:109E100003F101039E424FDC1FE014AC04EBD302BC
:109E200003F0070007FA00F512F8441C45EA0104A4
:109E300002F8444C03F1010314AA02EBD30403F02B
:109E4000070007FA00F514F8441C45EA010204F87B
:109E5000442C03F101039E42DFDC4FF007004FF07A
:109E600012014FF01E0203ABFFF756F84FF0060B3E
:109E700015E0A6B9BBF1020F11D1009A7AB942F6EA
:109E8000BC06C2F20006F2784AB14FF00200494621
:109E9000FFF75AFD4FF03200FBF73CFF0097BAF195
:109EA000000F06D10BF1FF3BCDF800904FF0280AD0
:109EB000A1E60AF1FF3A9EE6002DAED014AD05EB07
:109EC000D30403F0070007FA00F214F8441C42EA36
:109ED000010504F8445C03F101039E429DDCBCE7EC
:109EE000002A3FF44CAF14AA02EBD30603F007009C
:109EF00007FA00F516F8441C45EA010206F8442C5E
:109F000003F10103A342FFF63AAF58E72DE9F04F02
:109F10002DED028B87B008EE100A0C4617469946C5
:109F2000129E1399B5EEC08AF1EE10FA54BF0025C7
:109F30000125A84604F1FF33D8B2082807D8092A1A
:109F400005D8A24601F1FF32944205D808E001F19C
:109F5000FF339C4240F2CD8001F1FF34E4B2C8E00F
:109F600018EE100A0BF022FD48B930464FF03F01C1
:109F700022460CF007FB4FF000013155C4E018EE0B
:109F8000100A0BF07FFD06EE900AF2EE047AF4EE72
:109F9000E76AF1EE10FA0DDB4FF00100B0EE677AE0
:109FA00000F1010067EE877AF4EEE76AF1EE10FA4D
:109FB000F6DA03E04FF00100F2EE047A214643198D
:109FC000A34200F39680C0EB040EC5EB0E0202F133
:109FD000FF3E49F6A84AC0F6010ADFED9C4AF6EEBC
:109FE000003AB2EE044AC0EB040CC5EB0C0303F0DC
:109FF000010BBEF1000F00F38F808AE0BEF1000F6D
:10A0000004DDBE45B4BF72463A4601E04FF000029F
:10A010005AF8223003EE103AB8EE430A20EE027AE4
:10A02000B4EEE47AF1EE10FA48BF37EE237ABDEED3
:10A03000C73A13EE10CABCFBF3FB06EE10BAB8EE3B
:10A04000C65AB4EEE75AF1EE10FA0DDB00F1010C3E
:10A0500087EE006A67EE847A0EF1FF3E6046BEF13D
:10A06000000200F3C380BEE013EE105AB5FBF3F418
:10A0700003FB14542CB916EE107A002F08BF4FF0D2
:10A080000008B9F1000F07D0C8EB0103181A002A25
:10A0900018BF0138831A01E04FF0000301F10101FC
:10A0A000B8F1000F04D04AF69447C0F6010703E068
:10A0B00048F2F827C0F6010722B14AF69840C0F6E8
:10A0C000010003E048F2F820C0F601004AF6AC4572
:10A0D000C0F60105009501978DED026A0390049288
:10A0E000059430464AF69C42C0F601020BF014FE7D
:10A0F0000AE03046002D0CBF2B212D2122460CF00A
:10A1000041FA4FF00000305507B0BDEC028BBDE8BE
:10A11000F08F4FF0000203E0BE45B4BF72463A46EE
:10A120005AF8223000EE103AB8EE405A65EE260A90
:10A13000F4EEE40AF1EE10FA48BF70EEA30ABDEEA9
:10A14000E03A13EE10CABCFBF3FC06EE10CAF8EEC0
:10A15000C65AF4EEE75AF1EE10FA85DB00F1010081
:10A1600080EE852A67EE847A0EF1FF3E4219914215
:10A17000BFDBBBF1000F3FF441AFBEF1000F02DCCB
:10A180004FF0000203E0BE45B4BF72463A465AF8AB
:10A19000223001EE103AF8EE411A21EE822AB4EE96
:10A1A000E42AF1EE10FA48BF32EE232ABDEEC23A9D
:10A1B00013EE10BABBFBF3FB06EE10BAF8EEC62A9C
:10A1C000F4EEE72AF1EE10FAFFF64EAF00F10100CF
:10A1D00082EE212A67EE847A0EF1FF3E43199942FE
:10A1E000BFF60CAF85E74FF0000202E0BA42A8BF0D
:10A1F0003A465AF8223006EE903AF8EE660A20EE19
:10A20000861AB4EEE41AF1EE10FA48BF31EE231AC2
:10A21000BDEEC13A13EE10BABBFBF3FB06EE10BA6B
:10A22000F8EEC65AF4EEE75AF1EE10FAFFF61CAF5C
:10A230000CF1010081EE202A67EE847A0EF1FF3ED8
:10A2400042199142BFF6DAAE53E700BF0000004B5F
:10A25000F8B505460F46F6F799FD064641F6187221
:10A26000C2F200024FF4117303FB05F014181158E9
:10A2700011B18A682846904784F820724FF0000593
:10A28000C4F81052C4F81452C4F80451C4F8085168
:10A290003046F6F785FD04F5097029464FF00802AF
:10A2A000F6F72EFDF8BD00BF70B588B0054641F643
:10A2B0001874C2F200044FF4117303FB004494F8C5
:10A2C000200200284AD042F6A801C2F200010A8802
:10A2D0004FF6FF76B24204D0D0B24FF00401FFF740
:10A2E000B7FF28464FF00001FFF7B2FF42F6A8067D
:10A2F000C2F2000635804AF6B840C0F601004FF0C1
:10A3000007014FF62132C0F60002FBF7C5FCC4F886
:10A310001C02246830784FF0010300934FF00002D4
:10A32000019248F29541C0F60001029148F675236A
:10A33000C0F60003039348F69511C0F6000104919E
:10A3400048F2F573C0F600030593069264684FF473
:10A3500016514FF00803A047FEF77EF908B070BD14
:10A3600038B506F09BF842F6C003C2F200034FF086
:10A3700001021A704FF000042546E0B229462A4631
:10A38000FFF722FA60B904F10104E0B229462A4637
:10A39000FFF71AFA00286BD002E04FF0000401E04A
:10A3A0004FF000044FF00005E0B22946FFF774FAC1
:10A3B00010B904F10104F7E745F29C41C2F2000133
:10A3C0000C6834B12368DA6802B190476468002CE5
:10A3D000F8D142F6B800C2F2000004683CB121682E
:10A3E0000B680BB1A06898476468002CF7D1FAF7A6
:10A3F00065FBFEF721FA41F61872C2F2000292F8EC
:10A400002002042806D028B14FF000004FF00401CC
:10A41000FFF71EFF41F61871C2F2000191F8643493
:10A42000042B06D02BB14FF001004FF00401FFF7D1
:10A430000FFF41F61872C2F2000292F8A806042833
:10A4400006D028B14FF002004FF00401FFF700FFE3
:10A4500041F61871C2F2000191F8EC38042B06D0D5
:10A460002BB14FF003004FF00401FFF7F1FE38BDB0
:10A4700004F10104B4F5807F7FF47FAF8DE700BF66
:10A480002DE9F04F2DED048BABB01CAF26AC49F697
:10A49000A825C0F6010595E80F0084E80F00A76025
:10A4A00048F21D23C0F60003E36020462AA9F8F70E
:10A4B000E5FC22AE95E80F0086E80F00B76048F291
:10A4C0003920C0F60000F06030462146F8F7D6FC8F
:10A4D0004FF000041B9442F62800C2F2000021460F
:10A4E000FBF722F842F60011C2F200010C72FFF7EE
:10A4F00037FF0AF041F94FF00200FFF7D5FE45F2B1
:10A500009442C2F2000215680DBB0DF0F9FDF0B9DE
:10A51000F7F756FA10F0C20F19D14FF00300FEF70B
:10A52000D7FC4FF47A744FF032052846FBF7F2FB64
:10A53000F7F746FB04F1FF342846FBF7EBFBF7F790
:10A540003FFB013CF1D14FF00000FEF7C1FC45F2AA
:10A55000A043C2F200034FF000041C604FF0010062
:10A56000187042F63C15C2F200052846214642F614
:10A5700054220CF007F840F6D860C2F200002146E1
:10A580004FF480520BF0FEFF42F66000C2F2000072
:10A5900021464FF040020BF0F5FF45F29030C2F239
:10A5A000000021464FF0FC020BF0ECFF21954FF02C
:10A5B0000A01696220462946FDF7CCFD42F6C40235
:10A5C000C2F20002146042F6B003C2F200031C6043
:10A5D00045F29445C2F200054FF030042C604CF671
:10A5E0000004C0F6010494F82F0000F1010094F873
:10A5F0002E1000EB0122101945F28C43C2F2000329
:10A600001860FCF701F80A902B68E15CFF2930D153
:10A6100042F60012C2F200024FF001011172136003
:10A620002198026A1AB102F1010250F8223042F672
:10A630000011C2F200014B604FF0FF00487242F679
:10A64000AC03C2F200034FF000021A6042F6A80108
:10A65000C2F20001088841F61872C2F200024FF4FB
:10A66000117303FB0021D1F81C02FBF7BDF905F0C3
:10A6700085B905F0F1FE4FF000060996B246344662
:10A6800001E04FF000042CB94FF00000FEF7E2FCAF
:10A690004FF0640404F1FF3445F2A047C2F2000712
:10A6A0003D7805F0E7026FF345123A7045F29440A9
:10A6B000C2F200000368089345F29446C2F2000615
:10A6C0004CF60007C0F6010745F2A048C2F20008A8
:10A6D00049F6D059C0F6010931687D5C01F10101EC
:10A6E000316098F8002012F0010F0ED10AF1010A32
:10A6F00040F2FF30824508D942F60013C2F200034F
:10A700004FF03601197205F0EEB80DF1700C2846C5
:10A710004946FEF7CDF94AF20823C0F6010353F883
:10A7200025204AF62C1BC0F6010B42F00101084718
:10A730003268B85C0B9002F1010232600F2805F21A
:10A74000CA800DF1700C5946FEF7B2F949F6B823EC
:10A75000C0F601030B9953F82120E6E73268B85C94
:10A760000B9002F101023260102802D9054605F073
:10A77000B3B80DF1700C0B984AF6FC31C0F601012C
:10A78000FEF796F94AF21873C0F601030B9953F8D5
:10A790002120CAE73268B85C0B9002F101023260F6
:10A7A0000F2802D9054605F097B80DF1700C0B98EB
:10A7B0004AF6BC31C0F60101FEF77AF94AF66C237D
:10A7C000C0F601030B9953F82120AEE73268B85C5C
:10A7D0000B9002F1010232602F2802D9054605F0E4
:10A7E0007BB80DF1700C0B9849F6F821C0F6010109
:10A7F000FEF75EF94AF25C73C0F601030B9953F859
:10A80000212092E73268B85C0B9002F101023260BD
:10A810003B2802D9054605F05FB80DF1700C0B9886
:10A8200049F6B831C0F60101FEF742F94AF2086371
:10A83000C0F601030B9953F8212076E73268B85C23
:10A840000B9002F1010232603F2802D9054605F063
:10A8500043B80DF1700C0B9849F6D041C0F60101D8
:10A86000FEF726F94AF66C13C0F601030B9953F86C
:10A8700021205AE73268B85C0B9002F10102326085
:10A88000432802D9054605F027B80DF1700C0B9846
:10A890004AF6AC21C0F60101FEF70AF94AF61C039C
:10A8A000C0F601030B9953F821203EE7219E96F84C
:10A8B00046700DF1700CFDF7AFFB219D381895F82F
:10A8C000503003F0010142181C9285F84720FF2AFE
:10A8D00094BF0022012285F85020D4E6219E96F8EC
:10A8E00046700DF1700CFDF797FB3D181C952198F3
:10A8F00080F84750FF2D94BF0025012580F8505067
:10A90000C1E60DF1700CFDF787FB30B1219991F88C
:10A910004720131C18BF012301E04FF00003219EC4
:10A9200086F84730AFE60DF1700CFDF775FB219FFF
:10A9300097F84750284087F84700A4E61D98A0F1F3
:10A94000FB001C9019E11D9BA3F1FB031C93A1E1EB
:10A950001D99A1F1FB011C91D2E11D9AA2F1FB020C
:10A960001C926EE21D98A0F1FB001C904FF00203B8
:10A970001B9306E21D99A1F1FB011C911E9A1B92EB
:10A9800030E21D98A0F1FB001C902AE11D9BA3F171
:10A99000FB031C93ACE21D99A1F1FB011C91E8E2C1
:10A9A0001D9EA6F1FB061C961E9F1B9725E31D9A74
:10A9B000A2F1FB021C921E981B904FF000038DF831
:10A9C0006A30D3E31D99A1F1FB011C911E9A1B92E1
:10A9D0004FF001008DF86A00C8E31D9BA3F1FB0353
:10A9E0001C9300F060BC1D9DA5F1FB051C9500F0BB
:10A9F000B5BC9DF874004FF00101FEF7A3FE8DF881
:10AA00006B0000283FF43FAE42F60014C2F200048F
:10AA1000207204F068BF1D9E1C964FF001008DF857
:10AA20006A000646219991F84720104205D09DF80A
:10AA300070003146FEF786FE68B99DF86A004FEA5D
:10AA400040038DF86A301C9901F101011C9113F04B
:10AA5000FE00E7D10CE09DF86A20012A08D19DF89C
:10AA60006B4042F60013C2F200031C7204F03BBFBD
:10AA70000DF1700CFDF7D0FA05E69DF8740005F0B5
:10AA8000DDFC00E60DF1700CFDF7C6FA1C9045F2F6
:10AA90009443C2F2000318681C9900EB41021A604B
:10AAA000FDF7D0FA1C9001F0D1BE45F2A041C2F2F0
:10AAB0000001087810F0280F06D01D9AB2F5805FCB
:10AAC00034BF0022012204E01D9AFA2A94BF00221A
:10AAD000012242B142F60014C2F200044FF0130208
:10AAE000227204F000BF40F6D861C2F200011D9B43
:10AAF000C85C1C90CBE7219991F852301C93C6E7B3
:10AB0000219890F850201C92C1E74FF0000ABAE556
:10AB10000DF1700CFDF780FA1C90219F97F84710FB
:10AB20001B91FDF72FFB87F84700ACE5219D95F8B9
:10AB3000470095F84610FDF725FB85F85000A2E583
:10AB40000DF1700CFDF790FA1E9E40F6D863C2F22C
:10AB50000003985D1D9920EA01029A5593E545F29C
:10AB60009030C2F200004FF000014FF0FB020BF0FA
:10AB700009FD88E54FF000061C960DF1A80C1CF8A5
:10AB8000386DFDF749FA0146304608F007FA8DF8AE
:10AB90006B0000283FF477AD42F60014C2F20004C7
:10ABA000207204F0A0BE06F07DFD6CE506F082FD8B
:10ABB0008DF86B0000283FF466AD42F60013C2F238
:10ABC0000003187204F08FBE45F28C47C2F20007F2
:10ABD0003D681D98281806F059FD54E54FF0000116
:10ABE0001C911C9B41F61872C2F200024FF41170C6
:10ABF00000FB032191F82022032A3FD141F6187669
:10AC0000C2F2000600FB03F303F58877F119F3188D
:10AC100003F104034FF00000D1F80021FE2A94BF95
:10AC2000551C0025D1F80461B54214BF002501254B
:10AC300065F30000B24214BF0022012262F341001A
:10AC4000D3F80051FE2D94BF013500250DF1A80C5D
:10AC50004CF8385DD3F80471BD4214BF00250125BE
:10AC600065F38200D3F80811D1F1010338BF002346
:10AC700063F3C300C0B2FDF7B7F904E542F6001470
:10AC8000C2F200044FF04803237204F02CBE4FF0D0
:10AC900000001C901C9B41F61872C2F200024FF497
:10ACA000117101FB032090F82022032A1CD141F6E8
:10ACB0001876C2F2000601FB0365D5F81072D5F8CC
:10ACC0001412781AB0F5807F88BF00F580701C9050
:10ACD0001C9AFF2A84BFFF221C920DF1A80C1CF8BD
:10ACE000380DFDF781F9CEE442F60014C2F20004FB
:10ACF0004FF04803237204F0F6BD4FF000031C939D
:10AD00001C9841F61872C2F200024FF4117101FB57
:10AD1000002393F82022032A24D141F61876C2F2A8
:10AD2000000601FB006505F58877D7F80011D7F814
:10AD30000431CA1AB2F5807F88BF02F580721C9276
:10AD40000DF1700CFDF768F98DF86A001C9EB04299
:10AD500038BF1C90D7F804011C9D2918CBB2C7F846
:10AD6000043190E442F60014C2F200044FF04800AF
:10AD7000207204F0B8BD4FF000021C924FF00200A8
:10AD80001B901C9B41F61872C2F200024FF4117125
:10AD900001FB032090F82022032A15D141F61877F1
:10ADA000C2F2000701FB03760DF1700C1B9848F20C
:10ADB0009911C0F6000148F2AD12C0F6000206F586
:10ADC0008873FDF763F95EE442F60014C2F20004F2
:10ADD0004FF04803237204F086BD4FF000011C9130
:10ADE0001D981B901C9B41F61872C2F200024FF492
:10ADF000117101FB032090F82022032A15D141F69E
:10AE00001875C2F2000501FB03570DF1700C1B9879
:10AE100048F29911C0F6000148F2AD12C0F60002E6
:10AE200007F58873FEF7AAF92DE442F60014C2F282
:10AE300000044FF04803237204F055BD4FF00001A9
:10AE40001C911C9841F61872C2F200024FF4117363
:10AE500003FB002191F82022032A3DD141F6187608
:10AE6000C2F2000603FB006505F588750DF1700C54
:10AE7000FDF7D2F88DF86A00D5F804111C914FF057
:10AE800000071B97D5F800710B468F4207D06A5C0C
:10AE9000824219D04FF001024FF0000E0CE04FF04B
:10AEA000FF001B9010E002F10106E95C814202D133
:10AEB0001C931B9208E03246FF2B14BF01337346EC
:10AEC0009F42F0D11C93EAE70DF1700C9DF86C00E5
:10AED000FDF78AF8FFF7D7BB42F60014C2F2000470
:10AEE0004FF04800207204F0FEBC4FF000031C93AA
:10AEF0001C9841F61872C2F200024FF4117101FB66
:10AF0000002393F82022032A27D141F61875C2F2B4
:10AF1000000501FB005707F58875D7F81462D7F8CC
:10AF200010128E4212D00DF1700CFDF775F88019D9
:10AF3000C7B21C970DF1700CE85DFDF755F84FF0A6
:10AF40000005219E86F85050FFF79DBB4FF001028F
:10AF5000219B83F85020FFF796BB42F60014C2F203
:10AF600000044FF04800207204F0BDBC4FF0000117
:10AF70001C911C9B41F61872C2F200024FF4117032
:10AF800000FB032191F82022032A28D141F61877EB
:10AF9000C2F2000700FB037505F58876D6F80401B8
:10AFA000D6F80011884213D00DF1700C305CFDF71B
:10AFB0001BF8D6F80471FF2F14BF01370027C6F81D
:10AFC00004714FF00005219E86F85050FFF75BBBDF
:10AFD0004FF00102219B83F85020FFF754BB42F64B
:10AFE0000014C2F200044FF04803237204F07BBC4B
:10AFF0004FF000001C901D991B9145F28C42C2F24B
:10B000000002D2F800801B9F08EB07064CF60003F5
:10B01000C0F602039E4208D942F60014C2F20004B0
:10B020004FF01F02227204F05EBC1C98032808D95E
:10B0300042F60010C2F200004FF03703037204F032
:10B0400052BCF1780D2908D942F60014C2F200046E
:10B050004FF03701217204F046BC41F61875C2F278
:10B0600000054FF4117202FB005393F8200238B12F
:10B0700018F8071021B10FE04846FDF7EBFF05E097
:10B080004CF24F354FF09609DDF828B0FBF7BCFACB
:10B09000CBEB0002AA42EFD918F80770032F3FF656
:10B0A000F2AADFE807F002080F169DF87000FFF71C
:10B0B000FBF8FFF7E8BA9DF87000314607F090FF03
:10B0C000FFF7E1BA9DF87000314606F047FAFFF746
:10B0D000DABA9DF87050B77828464FF00301FFF7B1
:10B0E000B7F84FF4117303FB05F041F61871C2F283
:10B0F0000001085800283FF4C6AA4AF20473C0F6BB
:10B10000010307EB470703EB0708F6784AF2D01272
:10B11000C0F6010252F82610DA5D98F8013098F86E
:10B12000027000974FF00006019648F26557C0F68E
:10B130000007029748F2A557C0F60007039748F2A8
:10B14000D557C0F60007049748F2F577C0F6000718
:10B150000597069646682846B047FFF794BA4FF021
:10B1600000011C911D981B908DF86A101C9841F6E7
:10B170001873C2F200034FF4117101FB003292F810
:10B180002032032B79D141F61875C2F2000501FB7C
:10B19000005707F5887945F28C46C2F200063168FF
:10B1A000219A936B01EB030BCB5CFF2B5CD0D84651
:10B1B0004FF001054FF0000B0894CDF82CA0AA46E3
:10B1C00098F8014004EB032745F28C46C2F20006D2
:10B1D0003268D319D9F804111C919DF86A0018B18E
:10B1E000D75D03F1010300E05F4603F1FF349DF8F2
:10B1F0006A502DB177B9089C5046DDF82CA005E0C7
:10B2000066783EB9089C5046DDF82CA01C9AC9F817
:10B2100004212BE01C9BD9F800219A4218D014F885
:10B22000016F19F803501B9939B930460AF018FD1F
:10B23000C6B228460AF014FDC5B2AE4208D11C9829
:10B24000FF2814BF013058461C9007F1FF37CEE7A6
:10B250000AF1010A18F8023FFF2BB1D1089CDDF872
:10B260002CA04FF0000001E04FF000000DF1700C39
:10B27000C0B2FCF7B9FEFFF706BA42F60014C2F2FC
:10B2800000044FF04800207204F02DBB4FF0000383
:10B290001C931E9A1B924FF001018DF86A1065E70E
:10B2A0004FF000011C911C9841F61873C2F2000384
:10B2B0004FF4117101FB003292F82032032B31D18F
:10B2C00041F61876C2F2000601FB006505F58877A5
:10B2D0000DF1700CFCF7A0FE8DF86A004FF0000134
:10B2E0001C91D7F80431D7F80051AB4212D0FA5C68
:10B2F00082420FD14FF00006FF2B14BF01333346BB
:10B300009D4202D1C7F8043104E0F95C8142F3D0D8
:10B31000C7F804310DF1700C4FF00000FCF764FE2B
:10B32000FFF7B1B942F60014C2F200044FF0480032
:10B33000207204F0D8BAFBF767F90A9FC01B0DF121
:10B34000700C4CF24F3398428CBF00200120FCF768
:10B350004BFEFFF798B94FF000001C901C9D41F682
:10B360001872C2F200024FF4117606FB052191F823
:10B370002072032F7FF487A941F61873C2F20003ED
:10B3800006FB053000F10405D0F80861D5F800216E
:10B3900002F10102964238BF06F58076B11AFF2904
:10B3A00034BF0F46FF270DF1700CF8B2FCF71CFEFE
:10B3B000FFF769B91D9B40F6D860C2F20000C55C7A
:10B3C00005F1FF36C654FFF75EB945F2A042C2F25E
:10B3D0000002117811F0280F06D01D9BB3F5805F95
:10B3E00034BF0023012304E01D9BFA2B94BF0023EC
:10B3F000012343B142F60014C2F200044FF01302DD
:10B40000227204F070BA1D9840F6D862C2F20002AF
:10B41000115C01F1FF33D9B2115400293FF433A973
:10B420001E981C9001F012BA45F2A043C2F200032C
:10B43000197811F0280F06D01D98B0F5805F34BF41
:10B440000020012004E01D98FA2894BF002001206C
:10B4500040B142F60014C2F200044FF0130222720F
:10B4600004F041BA1D9A40F6D861C2F200018B5C2B
:10B4700003F1FF30C3B28B54002B42F00087FFF77B
:10B4800002B945F2A041C2F20001087810F0280F7D
:10B4900006D01D9BB3F5805F34BF0023012304E079
:10B4A0001D9BFA2B94BF0023012343B142F60014E5
:10B4B000C2F200044FF01302227204F014BA1D9A73
:10B4C00040F6D861C2F20001885C00F1FF33D8B2C7
:10B4D0008854002802F0D386FFF7D5B8219F97F84B
:10B4E000515005F1FF3687F85160FFF7CCB821992C
:10B4F00091F8473003F1FF3081F84700FFF7C3B8F8
:10B50000219AD06C0AF0BEFA219FF864FFF7BBB80D
:10B51000219D95ED137AD5ED127A37EE270A85ED48
:10B52000130A219AD06C0AF021FA30B14FF00202CE
:10B53000219B83F85020FFF7A6B82198C06C0AF031
:10B5400025FA30B14FF00106219981F85060FFF7DC
:10B550009AB84FF00007219D85F85070FFF793B817
:10B560009DF87400219901F14C01FEF769F98DF8FD
:10B570006B0000283FF487A842F60014C2F20004D2
:10B58000207204F0B0B99DF874002199C96CFEF7DF
:10B5900083F98DF86B0000283FF475A842F600137C
:10B5A000C2F20003187204F09EB9219EF06C0AF0FA
:10B5B000EDF920B92198806C0AF0E8F930B14FF02C
:10B5C0000306219880F85060FFF75DB8219AD2ED0C
:10B5D000138A92ED128A78EEC80A10EE900A0AF0E9
:10B5E00051FA09EE100A18EE900A18EE101A0AF035
:10B5F000E3F901464FF07E500AF0DEF99FEDCF1AD5
:10B6000001EE900A21EE812AB4EEC29AF1EE10FA10
:10B6100006D84FF00001219B83F85010FFF733B894
:10B62000219FD7ED132A97ED123AF4EEC32AF1EEDB
:10B6300010FA05DD4FF0010587F85050FFF723B8E9
:10B64000F4EEC32AF1EE10FA4CBF0222032287F86F
:10B650005020FFF718B8219AD2ED133AB7EE004AFE
:10B6600073EEC44AC2ED134A2198C06C0AF08EF9F9
:10B6700030B14FF00305219F87F85050FFF703B812
:10B68000219BD3ED138A9FEDAE8A38EEC89A19EE4E
:10B69000100A0AF0F7F909EE100A18EE900A18EEEF
:10B6A000101A0AF089F901464FF07E500AF084F929
:10B6B000DFEDA23A04EE100A64EE234AB4EEE49AF7
:10B6C000F1EE10FA22D9219E96ED138ADFED9C8AC5
:10B6D00038EE285A15EE100A0AF0D4F908EE900A4E
:10B6E00018EE100A6FF052510AF066F901464FF059
:10B6F0007E500AF061F9DFED915A06EE100A66EE0F
:10B70000256AF4EEE68AF1EE10FA06D84FF0040648
:10B71000219981F85060FEF7B6BF2199CD6C28467B
:10B720000AF0B0F908EE100A28464FF000010AF0BE
:10B7300043F901464FF07E500AF03EF9DFED7F7A83
:10B7400007EE100A27EE270AB4EEC08AF1EE10FACF
:10B7500006D84FF00000219B83F85000FEF793BFFE
:10B76000219FD7ED130AF5EEC00AF1EE10FA05DDC0
:10B770004FF0010287F85020FEF785BFF5EEC00AB2
:10B78000F1EE10FA4CBF0222032287F85020FEF798
:10B790007ABF219F97ED125AD7ED135A85EE256A8D
:10B7A00087ED136ABDE62199C86C0AF0DBF8002822
:10B7B00041F04A80FEF767BF219BDE6C30460AF0FD
:10B7C00061F908EE100A30464FF000010AF0F4F873
:10B7D00001464FF07E500AF0EFF8DFED586A07EEB1
:10B7E000100A67EE267AB4EEE78AF1EE10FA01F35A
:10B7F0002B80FEF748BF2198C06C0AF0B3F80028F0
:10B8000001F02280FEF73FBF219A92ED130AD2ED9C
:10B81000120AB4EEE00AF1EE10FA81F21580FEF79A
:10B8200032BF219991ED131AD1ED121AB4EEE11A3B
:10B83000F1EE10FA01F30880FEF725BF219B93ED8E
:10B84000132AD3ED122AB4EEE22AF1EE10FA40F2F6
:10B85000FB87FEF718BF219890ED133AD0ED123A0E
:10B86000B4EEE33AF1EE10FA00F1EE87FEF70BBF0B
:10B87000219EF66C30460AF005F908EE100A3046B3
:10B880004FF000010AF098F801464FF07E500AF0A0
:10B8900093F89FED2A4A04EE900A24EE845AB4EEFF
:10B8A000C58AF1EE10FA40F2CF87FEF7ECBE219D7B
:10B8B000E86CFCF7E9F9E8640DF1700C4FF000005A
:10B8C000FCF77EFCFEF7DFBE1D9AF62A08D942F689
:10B8D0000014C2F200044FF01202227204F003B806
:10B8E000219FF86C0AF03EF838B9219B93ED136A5A
:10B8F000F6EE006A36EE268A06E0219991ED138A6B
:10B90000F6EE005A38EE658A18EE100A0AF02AF8A8
:10B9100000BB9FED0C7AB4EEC78AF1EE10FA04DC9E
:10B9200018EE100A0AF022F8A0B14FF00100219E93
:10B9300086F850006FF000403BE000BF000000348C
:10B94000FFFF7F4BFEFFFF4AFEFFFFCA0000804360
:10B95000000080C318EE100A0AF004F898B15FEDF9
:10B96000067AB4EEE78AF1EE10FA04D418EE100A63
:10B9700009F0FCFF38B14FF00101219B83F8501012
:10B980004FF0004015E018EE100A09F0FFFF38B143
:10B990004FF00202219F87F850204FF0000008E08E
:10B9A000BDEEC88A18EE100A4FF00006219D85F8FA
:10B9B00050604FEA006545EA106200F47F4742EAB2
:10B9C000072100F47F0341EA132045F29036C2F2CA
:10B9D00000061D9D7051FEF756BE1D99F62908D927
:10B9E00042F60014C2F200044FF01201217203F07B
:10B9F0007ABF45F29037C2F2000778584FEA0063E9
:10BA000043EA106600F47F4546EA052100F47F0210
:10BA100041EA122700EE107AF8EEC00A2198C0ED34
:10BA2000130A1FED381AF4EEC10AF1EE10FA06DC23
:10BA30005FED3B1AF4EEE10AF1EE10FA05D54FF096
:10BA4000010680F85060FEF71EBE4FF0000380F83C
:10BA50005030FEF718BE0DF1700C4FF00100FCF7EE
:10BA6000AFFB219DE86CFCF739F9219AD064FEF711
:10BA70000ABE219F97ED132AF7EE002A32EE223AF2
:10BA800087ED133AF0E5219AD06C09F07FFF50B1B1
:10BA9000219D4FF0000785F847704FF0040285F8AC
:10BAA0005020FEF7F0BD219890ED131AB5EEC01AA4
:10BAB000F1EE10FA23DB1FED5B3AB4EEC31AF1EEA0
:10BAC00010FA0FD5FCEEC13A13EE906A0DF1700C2E
:10BAD000F0B2FCF789FA4FF00001219B83F8501077
:10BAE000FEF7D1BD0DF1700C4FF0FF00FCF77CFAB2
:10BAF0004FF00202219880F85020FEF7C4BDB5EE49
:10BB0000C01AF1EE10FA7EF5BEAD5FED6F1AB4EE1D
:10BB1000E11AF1EE10FA11DDB1EE412AFCEEC22A73
:10BB200012EE901A0DF1700CC8B2FCF75DFA4FF0EE
:10BB30000105219F87F85050FEF7A5BD0DF1700C4F
:10BB40004FF0FF00FCF750FA4FF00306219B83F8FB
:10BB50005060FEF798BD45F2A040C2F200000178A7
:10BB600011F0280F08D01D9B03F10103B3F5805F8E
:10BB700034BF0023012306E01D9B03F10103FA2BD0
:10BB800094BF0023012343B142F60014C2F2000423
:10BB90004FF01302227203F0A6BE219E96ED134AC7
:10BBA000FDEEC44A14EE905A2FB21C97BAB2C5F3F8
:10BBB000072040EA022140F6D866C2F200061D9B2B
:10BBC000F152FEF760BD45F2A040C2F200000178DC
:10BBD00011F0280F08D01D9B03F10103B3F5805F1E
:10BBE00034BF0023012306E01D9B03F10103FA2B60
:10BBF00094BF0023012343B142F60014C2F20004B3
:10BC00004FF01302227203F06EBE219D95ED135A80
:10BC1000FCEEC55A15EE907ABEB21C964FEA16227B
:10BC200042EA062040F6D861C2F200011D9BC852CC
:10BC3000FEF729BD1D9D219FBD64FEF724BD1D9EFD
:10BC40002198C664FEF71FBD0DF1700CFCF7E4F9F6
:10BC500006EE100AF8EE466A2199C1ED136AFEF766
:10BC600012BD45F2A043C2F200031A7812F0280F69
:10BC700008D01D9800F10100B0F5805F34BF0020AE
:10BC8000012006E01D9800F10100FA2894BF002071
:10BC9000012040B142F60014C2F200044FF013013B
:10BCA000217203F020BE40F6D865C2F200051D9F48
:10BCB000EE5B4FEA162141EA06239AB207EE902A7C
:10BCC000B8EE670A219880ED130A9FEDC97AB4EEA9
:10BCD000C70AF1EE10FAFEF6D6ACDFEDC60A30EE7A
:10BCE000601A80ED131AFEF7CEBC45F2A043C2F2F3
:10BCF00000031A7812F0280F08D01D9800F10100F7
:10BD0000B0F5805F34BF0020012006E01D9800F1EF
:10BD10000100FA2894BF0020012040B142F600142F
:10BD2000C2F200044FF01301217203F0DCBD40F6B3
:10BD3000D865C2F200051D9FEE5B4FEA162141EA6D
:10BD400006239AB201EE902AB8EE612A219880ED7E
:10BD5000132AFEF798BC1D98072808D942F600134D
:10BD6000C2F200034FF008021A7203F0BCBDFCF7E8
:10BD70009FFD02EE900AB8EE623A219D85ED133ADE
:10BD8000FEF781BC219FD7ED133A97ED124A63EE7F
:10BD9000844AC7ED134AFFF7C4BB219E96ED135AA0
:10BDA000F1EE455AC6ED135AFEF76DBC4FF0000098
:10BDB0004FF001010A46FDF707FD219890ED136A47
:10BDC000F1EE046A66EE267A4FF0000100910191CF
:10BDD00042F6DC00C2F20000BCEEE70A10EE101AD8
:10BDE0004FF0FF0249F62D03C0F60003FAF7D6FB29
:10BDF000FEF749BC45F2A043C2F200031A7812F0E4
:10BE0000280F08D01D9800F10300B0F5805F34BF03
:10BE10000020012006E01D9800F10300FA2894BFDD
:10BE20000020012040B142F60014C2F200044FF09D
:10BE30001301217203F057BD40F6D865C2F2000528
:10BE40001D9FE859FBF74AFF219EB064FEF71BBC1B
:10BE500045F2A043C2F200031A7812F0280F08D06E
:10BE60001D9800F10300B0F5805F34BF0020012071
:10BE700006E01D9800F10300FA2894BF002001207D
:10BE800040B142F60014C2F200044FF013012172D7
:10BE900003F029BD40F6D865C2F200051D9FE859A0
:10BEA000FBF71CFF219EF064FEF7EDBB1D9B072BEB
:10BEB00008D942F60014C2F200044FF008002072C4
:10BEC00003F011BD2198D0ED130AF5EEC00AF1EE92
:10BED00010FA0FDB9FED487AF4EEC70AF1EE10FA84
:10BEE00008D8FCEEE01ACDED1C1A4FF0000580F8E2
:10BEF000505021E09FED401AF4EEC10AF1EE10FA25
:10BF000007DD6FF07F431C934FF0010280F8502053
:10BF100012E04FF000021C9210EE900A09F022FD90
:10BF200028B14FF00206219981F8506004E04FF0EB
:10BF30000305219F87F850501D981C99FCF790FC31
:10BF4000FEF7A1BB219FF86C09F020FD00287EF4CC
:10BF50009AAB219E96ED132AB5EEC02AF1EE10FAA7
:10BF600004DD4FF07E53F364FEF78DBBB5EEC02ABF
:10BF7000F1EE10FA7EF587AB4FF00001CBF6807141
:10BF8000F164FEF780BB219DAA6ACAB1FAF73CFBB7
:10BF9000219FBE6AC6F104010B184CF6CD45CCF6C4
:10BFA000CC45A5FB03124FEA92007E6AB0FBF6F186
:10BFB00002EE901AB8EE623A87ED133AFEF763BBD1
:10BFC0004FF6FF70C7F67F70E864FEF75CBB45F282
:10BFD000A043C2F200031A7812F0280F10D01D9867
:10BFE00000F10300B0F5805F34BF002001200EE0B7
:10BFF0000000004700008047FFFF7F4B0000003437
:10C000001D9800F10300FA2894BF0020012040B1E0
:10C0100042F60014C2F200044FF01301217203F043
:10C0200062BC1D9F219DE86CFBF72EFE40F6D86692
:10C03000C2F20006F051FEF726BB219BD3ED123A67
:10C0400093ED134A73EEC44AC3ED134AFFF769BA7E
:10C050002198C76C1C97856CC5648764FEF713BB79
:10C06000219EF06C09F092FC30B14FF00307219B48
:10C0700083F85070FEF707BB2199C86C09F076FC75
:10C0800030B14FF00401219A82F85010FEF7FBBA4C
:10C09000219AD76C384609F0F5FC08EE100A3846AC
:10C0A0004FF0000109F088FC01464FF07E5009F086
:10C0B00083FC1FED2E5A05EE900A25EE856AB4EE3C
:10C0C000C68AF1EE10FA06D84FF00005219E86F8D8
:10C0D0005050FEF7D8BA219BD3ED136AF5EEC06A33
:10C0E000F1EE10FA05DD4FF0010083F85000FEF785
:10C0F000CABAF5EEC06AF1EE10FA4CBF0222032272
:10C1000083F85020FEF7BFBA2198D0ED138A90ED46
:10C11000128A38EEC89A19EE100A09F0B3FC09EE3B
:10C12000100A18EE900A18EE101A09F045FC0146A4
:10C130004FF07E5009F040FC5FED507A00EE100A9F
:10C1400060EE270AB4EEE09AF1EE10FA0DF1700CF1
:10C150008CBF00200120FBF747FFFEF794BA219D1A
:10C16000EE6C304609F08EFC08EE100A30464FF0B7
:10C17000000109F021FC01464FF07E5009F01CFC43
:10C180001FED621A07EE100A67EE011AB4EEE18A9B
:10C19000F1EE10FA0DF1700C8CBF00200120FBF7BE
:10C1A00023FFFEF770BA219991ED132AD1ED122ADF
:10C1B000B4EEE22AF1EE10FA0DF1700CB4BF0020DB
:10C1C0000120FBF711FFFEF75EBA219A92ED133AB8
:10C1D000B5EEC03AF1EE10FA0DF1700CB4BF0020CC
:10C1E0000120FBF701FFFEF74EBA219FD7ED133A6E
:10C1F00097ED124AF4EEC43AF1EE10FA0DF1700C1C
:10C20000D4BF00200120FBF7EFFEFEF73CBA219BD4
:10C21000D3ED134A93ED125AF4EEC54AF1EE10FA3B
:10C220000DF1700C8CBF00200120FBF7DDFEFEF746
:10C230002ABA2198D0ED135A90ED126AF4EEC65A3C
:10C24000F1EE10FA0DF1700C54BF00200120FBF745
:10C25000CBFEFEF718BA219DD5ED136AF5EEC06A44
:10C26000F1EE10FA0DF1700C54BF00200120FBF725
:10C27000BBFEFEF708BA219ED6ED138A96ED128A10
:10C2800038EEC89A19EE100A09F0FCFB09EE100A04
:10C2900018EE900A18EE101A09F08EFB01464FF0C6
:10C2A0007E5009F089FB5FEDAB7A00EE100A60EE7C
:10C2B000270AB4EEE09AF1EE10FA0DF1700CD4BF3B
:10C2C00000200120FBF790FEFEF7DDB92199CF6C2D
:10C2D000384609F0D7FB08EE100A38464FF0000147
:10C2E00009F06AFB01464FF07E5009F065FB1FED37
:10C2F000BD1A07EE100A67EE011AB4EEE18AF1EEFC
:10C3000010FA0DF1700CD4BF00200120FBF76CFE79
:10C31000FEF7B9B945F2A042C2F20002137813F059
:10C32000280F08D01D9800F10200B0F5805F34BFDF
:10C330000020012006E01D9800F10200FA2894BFB9
:10C340000020012040B142F60014C2F200044FF078
:10C350001300207203F0C7BAFAF756F9219F00F1D3
:10C3600004004CF6CD45CCF6CC45A5FB00164FEAB3
:10C3700096017A6AB1FBF2F31D9D40F6D860C2F2D5
:10C38000000041194E78425D4FEA024545EA062019
:10C39000897840EA01061B969B1B23F07F421C9282
:10C3A00002EE102AF8EE422AC7ED132AFEF76BB907
:10C3B000219FFD6CBD64FEF766B9219991F851305B
:10C3C000002B40F04182FEF75EB9219A92F85100AD
:10C3D000002800F03982FEF756B945F2A041C2F2BA
:10C3E00000010B7813F0280F06D01D9AB2F5805F7C
:10C3F00034BF0022012204E01D9AFA2A94BF0022D1
:10C40000012242B142F60014C2F200044FF01300C0
:10C41000207203F068BA40F6D860C2F200001D999D
:10C42000435C002B7EF42FA91E9A1C920EE245F26B
:10C43000A041C2F200010B7813F0280F06D01D9A1C
:10C44000B2F5805F34BF0022012204E01D9AFA2A6F
:10C4500094BF0022012242B142F60014C2F200044D
:10C460004FF01300207203F03EBA40F6D860C2F2DB
:10C4700000001D99435C002B3EF405A91E9A1C92F6
:10C48000E4E142F60011C2F200014FF001030B7229
:10C4900003F029BA1D98F92808D942F60014C2F20F
:10C4A00000044FF01202227203F01DBA45F29032DE
:10C4B000C2F20002115C1E9B19427EF4E4A81F9890
:10C4C0001C90C3E11D99F92908D942F60014C2F263
:10C4D00000044FF01203237203F005BA45F29033C3
:10C4E000C2F20003585C1E9A10423EF4CCA81F9979
:10C4F0001C91ABE145F2A040C2F20000027812F0BC
:10C50000280F06D01D99B1F5805F34BF00210121AD
:10C5100004E01D99FA2994BF0021012141B142F69E
:10C520000014C2F200044FF01300207203F0DBB9D4
:10C5300040F6D860C2F200001D9BC25C002A7EF467
:10C54000A2A81E991C91B2E145F2A043C2F20003D9
:10C550001A7812F0280F06D01D99B1F5805F34BF0C
:10C560000021012104E01D99FA2994BF0021012135
:10C5700041B142F60014C2F200044FF013002072E1
:10C5800003F0B1B940F6D860C2F200001D9BC25C56
:10C59000002A3EF478A81E991C9188E145F2A04338
:10C5A000C2F200031A7812F0280F06D01D99B1F5D7
:10C5B000805F34BF0021012104E01D99FA2994BF56
:10C5C0000021012141B142F60014C2F200044FF0F3
:10C5D0001303237203F087B940F6D860C2F200005B
:10C5E0001D9BC25C1E998A427EF64DA81F981C9026
:10C5F0002CE145F2A042C2F20002117811F0280F9E
:10C6000006D01D98B0F5805F34BF0020012004E003
:10C610001D98FA2894BF0020012040B142F6001472
:10C62000C2F200044FF01303237203F05CB940F62A
:10C63000D862C2F200021D9BD15C1E988142FEF4BA
:10C6400022A81F9A1C9201E145F2A041C2F200010A
:10C65000087810F0280F06D01D9AB2F5805F34BF1D
:10C660000022012204E01D9AFA2A94BF002201222E
:10C6700042B142F60014C2F200044FF013032372D9
:10C6800003F031B940F6D861C2F200011D9BC85CCD
:10C690001E9A90427DF4F7AF1F991C91D6E045F2A7
:10C6A000A040C2F20000027812F0280F06D01D99B7
:10C6B000B1F5805F34BF0021012104E01D99FA2902
:10C6C00094BF0021012141B142F60014C2F20004DE
:10C6D0004FF01303237203F006B940F6D860C2F29C
:10C6E00000001D9BC25C1E998A423DF4CCAF1F988E
:10C6F0001C90ABE045F2A042C2F20002117811F0AA
:10C70000280F06D01D98B0F5805F34BF00200120AF
:10C7100004E01D98FA2894BF0020012040B142F6A1
:10C720000014C2F200044FF01303237203F0DBB8CD
:10C7300040F6D862C2F200021D9BD15C1E98814275
:10C740003DF6A1AF1F9A1C9280E045F2A041C2F2D3
:10C750000001087810F0280F06D01D9AB2F5805F0E
:10C7600034BF0022012204E01D9AFA2A94BF00225D
:10C77000012242B142F60014C2F200044FF013034A
:10C78000237203F0B0B840F6D861C2F200011D9BDD
:10C79000C85C1E9A9042BDF476AF1F991C9155E07B
:10C7A000219890F847201D998A427DF46CAF1E9B1A
:10C7B0001C937CE0219890F847201D998A423DF413
:10C7C00062AF1E9B1C9372E0219890F847201D9940
:10C7D0008A427DF658AF1E9B1C9368E0219890F822
:10C7E00047201D998A42FDF44EAF1E9B1C935EE0CC
:10C7F000219890F847201D998A42BDF444AF1E9BB2
:10C800001C9354E0219890F847201D998A423DF6E8
:10C810003AAF1E9B1C934AE09DF874000DF16B012A
:10C82000FCF7F2FE8DF86A009DF86B1031B142F60C
:10C830000014C2F20004217203F055B800283DF440
:10C8400022AF1E981C9001E01D9A1C921C984CF679
:10C850000003C0F6010393F82E1093F82F2042EA4C
:10C860000123834208D242F60014C2F200044FF0C2
:10C870000900207203F037B845F29445C2F2000572
:10C880002860FDF700BF0DF1700CFBF7C5FB1C9095
:10C890000028D9D0FDF7F7BE0DF1700CFBF7BCFBFB
:10C8A0001C900028D0D1FDF7EEBE1D9B1C93219A51
:10C8B000136A052B08D942F60014C2F200044FF0A7
:10C8C0000A03237203F00FB803F1020045F294410A
:10C8D000C2F20001096842F8201003F10103219A15
:10C8E0001362B3E70DF1700CFBF796FB1C90002868
:10C8F000DBD0FDF7C8BE0DF1700CFBF78DFB1C9073
:10C900000028D2D1FDF7BFBE0DF1700CFBF784FB00
:10C910001C901D9988427DF4B6AE1E981C9095E738
:10C920000DF1700CFBF778FB1C901D9A90423DF4C2
:10C93000AAAE1E9B1C9389E70DF1700CFBF76CFBF4
:10C940001C901D9988427DF69EAE1E981C907DE736
:10C950000DF1700CFBF760FB1C901D9A9042FDF4EA
:10C9600092AE1E9B1C9371E70DF1700CFBF754FB0C
:10C970001C901D998842BDF486AE1E981C9065E7F8
:10C980000DF1700CFBF748FB1C901D9A90423DF690
:10C990007AAE1E9B1C9359E79DF874000DF16B0154
:10C9A000FCF702FE8DF86A009DF86B1031B142F67B
:10C9B0000014C2F20004217202F095BF00283DF479
:10C9C00062AE1E981C9041E79DF874000DF16B015A
:10C9D000FCF7EAFD8DF86A009DF86B3033B142F642
:10C9E0000011C2F200010B7202F07DBF00287DF43D
:10C9F0004AAE1E9A1C9229E70DF1700CFBF734FB2E
:10CA000040F6D860C2F200001E9BC25C1D990A422B
:10CA10003DF439AE1F981C9018E70DF1700CFBF730
:10CA200023FB40F6D862C2F200021E9BD15C1D9827
:10CA300001427DF428AE1F9A1C9207E70DF1700C9D
:10CA4000FBF712FB40F6D861C2F200011E9BC85CE6
:10CA50001D9A10427DF417AE1F991C9127E70DF126
:10CA6000700CFBF701FB40F6D860C2F200001E9B81
:10CA7000C25C1D990A423DF406AE1F981C9016E751
:10CA800098F8005045F0080088F80000FDF724BE33
:10CA90000DF1700CFBF7C0FA8DF86A00219991F83E
:10CAA00051201D9BD1181C9145F2A042C2F20002F8
:10CAB000137813F0280F09D01E9A02F1FF3359188A
:10CAC000B1F5805F34BF0021012107E01E9A02F119
:10CAD000FF335918FA2994BF0021012141B142F6D0
:10CAE0000014C2F200044FF01303237202F0FBBEE5
:10CAF0004FF000061B961E9FEFB11C9940F6D865BB
:10CB0000C2F200056A5C824236D007F1FF3240F67D
:10CB1000D863C2F200035B1840F6D866C2F2000682
:10CB2000C6F10107C1F10101C6EB010E12F0010FC0
:10CB30001AD002F046BF4FF0FF001B901CE013F824
:10CB4000019F02F1FF35484504D11C91CDF86CC01E
:10CB50001E9211E02A46F9180EEB030C13F8016F30
:10CB6000B04242F03B87F0E7F9180EEB030C002AC5
:10CB7000E5D11C911E92DEE70DF1700C9DF86C0062
:10CB8000FBF732FAFDF77FBD0DF1700CFBF744FAAD
:10CB900042F6500BC2F2000B8BF800004FF001017F
:10CBA0001C91CDF830B0BBE0219A92F851001D9B4A
:10CBB000C1181C9145F2A042C2F20002107810F098
:10CBC000280F07D001F10101B1F5805F34BF0021CA
:10CBD000012105E001F10101FA2994BF00210121A1
:10CBE00041B142F60014C2F200044FF01303237265
:10CBF00002F079BE1E981B900DF1700C26AF47F025
:10CC0000010122AD45F001024FF00003FBF73EFAAF
:10CC1000FDF739BD219991F851201D9813181C93E7
:10CC200045F2A041C2F200010A7812F0280F05D0A7
:10CC3000B3F5805F34BF0023012303E0FA2B94BFD8
:10CC40000023012343B142F60014C2F200044FF066
:10CC50001300207202F047BE1F9E1E98B04228BFEC
:10CC600030461B900DF1700C26AF47F0010122AD4C
:10CC700045F001024FF00003FCF780FAFDF703BD19
:10CC80000DF1700CFBF7C8F9034642F6500BC2F2E7
:10CC9000000B58464FF010014AF6C842C0F6010298
:10CCA00009F03AF81C90CDF830B039E01E9B1C9387
:10CCB0001F991B914FF000020C9231E04FF0FF30B2
:10CCC0001C900C902CE0219EF06C9DF878109DF843
:10CCD0007C2042F65006C2F2000600964FF0100388
:10CCE00001934FF00103FDF711F94FF0FF311C9153
:10CCF0000C9615E0219AD06C9DF878109DF87C2058
:10CD000042F65006C2F2000600964FF0100301935F
:10CD10004FF00003FDF7FAF84FF0FF301C900C962F
:10CD20001D9BA3F1FB0291B20B91A3F1FB00032821
:10CD300023D841F61873C2F200034FF411720B9915
:10CD400002FB013090F82032032B08D042F600118C
:10CD5000C2F200014FF04800087202F0C4BD41F673
:10CD60001876C2F200064FF411770B9A07FB0267A0
:10CD700007F104074FF0000605E0219F97F8516086
:10CD8000F6184FF00007DDF870B0BBF1FF3F11D18E
:10CD90004FF0FF0B4FF00009C84645F2A041C2F228
:10CDA00000010D9140F6D860C2F200000E900F9580
:10CDB0000C9D05E0BBF1000FECD14FF000096FE0D6
:10CDC0001D9BA3F1FB03032B10D8D7F80061FF2EA6
:10CDD00014BF01364646D7F80421964206D1404694
:10CDE000FCF738F9D7F804118E42F8D0B5F1FF3FBF
:10CDF00015D1219850F8342F1168D1F800C0494658
:10CE000010AA4FF00103E0478DF86B0080B10F9D31
:10CE100042F60014C2F20004207202F064BD25B193
:10CE200015F809308DF8403002E01B988DF840006D
:10CE30001C98B0F1FF3F02D19DF8403083B31D9A9A
:10CE4000A2F1FB02032A07D8D7F800019DF8403071
:10CE50003B54C7F800611FE00D99087810F0280FC7
:10CE600005D0B6F5805F34BF0020012003E0FA2E24
:10CE700094BF0020012048B10F9D42F60014C2F279
:10CE800000044FF01301217202F02DBD9DF84030D7
:10CE90000E9A935506F1010609F10109D9458FD380
:10CEA0001D9EA6F1FB06032E05D80B9AD0B2FBF708
:10CEB00041FBFDF7E8BB219F97F8515009EB050EA8
:10CEC00087F851E0FDF7DFBB1D9AA2F1FB010329B2
:10CED00058D88FB241F61871C2F200014FF41172A6
:10CEE00002FB071393F82002032808D042F600142F
:10CEF000C2F200044FF04803237202F0F4BC41F682
:10CF00001876C2F200064FF4117505FB076505F1AE
:10CF100004051E9901F1FF321E9271B34FF0000813
:10CF200045F29449C2F200094CF600039B46C0F654
:10CF3000010BD5F80061FF2E14BF01364646D5F827
:10CF40000401864206D14046FCF784F8D5F8041166
:10CF50008E42F8D0D9F80030D5F800211BF8030034
:10CF6000A85403F10103C9F80030C5F800611E9E02
:10CF700006F1FF311E91002EDBD1F8B2FBF7DAFA91
:10CF8000FDF781BB1E9B1C93219991F851008218DB
:10CF90001B9245F2A046C2F20006367816F0280F22
:10CFA00008D003F1FF36B218B2F5805F34BF00221B
:10CFB000012206E003F1FF36B218FA2A94BF0022DC
:10CFC000012242B142F60014C2F200044FF01300F5
:10CFD000207202F088BCC71881F851701C9A02F1C7
:10CFE000FF351C95002A3DF44EAB45F29443C2F246
:10CFF00000031E681B9F40F6D861C2F20001C919E8
:10D000004CF60000C0F6010030184FF0000305F0A8
:10D01000010E10F803C001F803C003F101039342AD
:10D0200042F0C0840DE010F8038001F8038003F1A2
:10D03000010310F803E001F803E003F10103934258
:10D04000F1D1E819A91901F1010145F29442C2F2A6
:10D05000000211604FF0FF331C9300F101001B90A0
:10D06000FDF711BB4FF000028DF86A20219991F86D
:10D0700051201D9BD3181C931E9A1B9245F2A04071
:10D08000C2F20000007810F0280F08D002F1FF3241
:10D09000D018B0F5805F34BF0020012006E002F117
:10D0A000FF32D018FA2894BF0020012040B142F688
:10D0B0000014C2F200044FF01300207202F013BCFF
:10D0C00040F6D867C2F2000707EB03099DF87CB071
:10D0D00045F28C45C2F200052E688B6BF118F75CA7
:10D0E000FF2F52D088464FF0010208920B9498F817
:10D0F000014004EB072745F28C45C2F200052E687B
:10D10000F3194FF000011C919DF86A00002802F00D
:10D110001C84F75D03F1010302F019BC9DF86A203D
:10D1200012B15FB90B9C02E065783DB90B9C219E62
:10D1300096F851209D1886F8515029E014F8015FA7
:10D1400019F803B046B9284608F08AFDC5B258461A
:10D1500008F086FD5FFA80FB5D4508D11C9B03F15A
:10D1600001031C9307F1FF371B999942D6D2B346AE
:10D17000089800F10100089018F8027FFF2FB6D13F
:10D180000B9C4FF00003089302E04FF00000089062
:10D190000DF1700C0899C8B2FAF726FFFDF773BAC3
:10D1A0004FF001008DF86A0060E70DF1700CFAF79E
:10D1B00033FF034642F6500BC2F2000B58464FF0C5
:10D1C00010014AF6D042C0F6010208F0A5FD1C90FD
:10D1D000CDF830B0A4E50DF1700CFAF71DFF034651
:10D1E00042F6500BC2F2000B58464FF010014AF6BF
:10D1F000D842C0F6010208F08FFD1C90CDF830B087
:10D200008EE50DF1700CFAF707FF034642F6500B5E
:10D21000C2F2000B58464FF010014AF6DC42C0F64D
:10D22000010208F079FD1C90CDF830B078E50DF1E1
:10D23000700CFAF7F1FE034642F6500BC2F2000BF7
:10D2400058464FF010014AF6E442C0F6010208F0D9
:10D2500063FD1C90CDF830B062E5219B93F85160DE
:10D2600006F1010683F85160FDF70DBA1D9F40F6E7
:10D27000D865C2F20005EA5D02F10102EA55FDF748
:10D2800002BA219991F8470000F1010081F84700A6
:10D29000FDF7F9B99DF874000DF16B01FCF784F905
:10D2A0000DF1700CFAF7A0FE9DF86B30002B3DF4E9
:10D2B000EAA942F60014C2F20004237202F013BB82
:10D2C0009DF874000DF16B01FCF7D6F90DF1700CAF
:10D2D000FAF78AFE9DF86B1000293DF4D4A942F6B6
:10D2E0000012C2F20002117202F0FDBA1D981C90E9
:10D2F0004FF000031B934FF001018DF86A109DF869
:10D3000070000DF16B01FCF74FF99DF86B309BB984
:10D3100020B19DF86A201B9810431B909DF86A105D
:10D320004FEA41038DF86A301C9A02F101021C9207
:10D3300013F0FE0FE3D10AE09DF86A00012806D140
:10D3400042F60014C2F20004237202F0CCBA0DF1CE
:10D35000700C9DF86C00FAF747FEFDF794B91D9923
:10D360001C914FF000031B934FF001028DF86A20CF
:10D370009DF870000DF16B01FCF77EF99DF86B10C4
:10D3800099B920B19DF86A001B9B03431B939DF83C
:10D390006A204FEA42018DF86A101C9800F10100E2
:10D3A0001C9011F0FE0FE3D10AE09DF86A30012BCA
:10D3B00006D142F60014C2F20004217202F093BAC0
:10D3C0000DF1700C9DF86C00FAF70EFEFDF75BB9DD
:10D3D0009DF874000DF16B01FCF716F98DF86A00E9
:10D3E0009DF86B1031B142F60012C2F200021172C8
:10D3F00002F079BA0DF1700CFAF7F6FDFDF743B9BA
:10D400001D981C904FF000031B934FF001038DF803
:10D410006A30219991F8472013420ED09DF8700090
:10D420000DF16B01FCF7F0F89DF86B309BB920B162
:10D430009DF86A001B9901431B919DF86A204FEAF1
:10D4400042038DF86A301C9800F101001C9013F023
:10D45000FE03DED10AE09DF86A10012906D142F6EA
:10D460000014C2F20004237202F03DBA1B9E219FF9
:10D4700087F84760FDF707B99DF874000DF16B015F
:10D48000FCF72AF90DF1700CFAF7AEFD9DF86B0070
:10D4900000283DF4F8A842F60012C2F20002107211
:10D4A00002F021BA1D9B1C93D8B20DF16B01FCF761
:10D4B00013F91B909DF86B1031B142F60014C2F2C3
:10D4C0000004217202F00FBA4FF001058DF86A5086
:10D4D0001C9E70191C90C0B20DF16B01FCF7FCF89A
:10D4E0009DF86A7000FA07F01B9A02431B9207F13D
:10D4F00001078DF86A701C9800F101001C90FBB2C6
:10D50000072BE8D90DF1700C9DF86C00FAF76CFD53
:10D51000FDF7B9B80DF1700C219991F85100FAF7A7
:10D5200063FDFDF7B0B8FDF7AEB842F6C005C2F234
:10D5300000054FF001062E70FDF7A5B842F6C007B2
:10D54000C2F200074FF000023A70FDF79CB8219834
:10D550004FF000014FF0540209F014F84FF00000B2
:10D56000219042F6C403C2F200031C6804F1FF31AB
:10D57000196002F021B942F6C403C2F2000319682F
:10D580007F2908D942F60014C2F200044FF030029D
:10D59000227202F0A8B94FF001051C9542F63C1624
:10D5A000C2F20006B76D002F42F0DC8105E0D2F830
:10D5B000AC10002949D11C9301E04FF001031D9FDD
:10D5C00042F63C15C2F200054FF0540606FB03F389
:10D5D000EA18EF5057601E9882F852004FF00A0187
:10D5E0005162104600F13400219901F134014FF0ED
:10D5F000100208F0A3FF1C9B06FB035000F144003F
:10D60000219901F144014FF0040208F097FF1C9F9B
:10D6100006FB075000F14800219901F148014FF045
:10D62000080208F08BFF219A92F851001C9906FB22
:10D63000015585F8510042F6C406C2F2000633686F
:10D6400003F101033360FDF71EB803F101052B461A
:10D6500002F15402D2F8AC60002E42F09A81AAE79F
:10D660001C93FDF710B8219A92F852001E9082E7A1
:10D670000DF1700CFAF7D0FC1E907CE71D9F2198ED
:10D6800080F85170FCF7FFBF0DF1700C9DF874002D
:10D69000FAF7AAFCFCF7F7BF21998B6A002B3CF440
:10D6A000F2AFF8F7B1FF21998A6A801A496A1D9B87
:10D6B00001FB03F303EB83029042BCF4E4AF1E983A
:10D6C0001C90FFF7C3B8F8F79FFF219DA862FCF7F5
:10D6D000DABF45F29031C2F2000191F8FB201E9BA7
:10D6E000D018FB2808D942F60013C2F200034FF00D
:10D6F0001200187202F0F7B845F2A041C2F2000120
:10D70000087810F0280F09D01D98111801F1FF3189
:10D71000B1F5805FB4BF0021012107E01D995018C9
:10D7200000F1FF31FA29D4BF0021012141B142F6B5
:10D730000014C2F200044FF01302227202F0D3B8B8
:10D7400045F29036C2F20006F01840F6D867C2F2F1
:10D7500000071D9D791908F0F1FEFCF794BF98F8B9
:10D76000001041F0100588F80050FCF7B5BF219E6D
:10D7700096F84770002F0CBFFF22002286F8472042
:10D78000FCF781BF219B93F847006FEA000183F803
:10D790004710FCF778BF0DF1700CFAF765FC1E9D81
:10D7A00040F6D866C2F20006775D1D9A7A4072553F
:10D7B000FCF769BF219B986B1D990A181C92BDE16B
:10D7C000219BD86B996B42181C92B7E1219B186C76
:10D7D00040B942F60014C2F200044FF02001217259
:10D7E00002F081B800F1FF351D64FCF74CBF219AAF
:10D7F000136C03F101031364002B7CF444AF42F675
:10D800000010C2F200004FF02004047202F06BB866
:10D8100021994A6B1368586840B942F60013C2F266
:10D8200000034FF01E021A7202F05DB80DF1700C89
:10D83000FAF7F2FB1C90219850F8346F31684E686B
:10D840001D991CAA4FF00103B0478DF86B0000280A
:10D850003CF419AF42F60014C2F20004207202F048
:10D8600042B80DF1700CFAF7D7FB1C9054E10DF1A2
:10D87000700CFAF7D1FB219FF863FCF704BF0DF1A0
:10D88000700CFAF7C9FB219D2864FCF7FCBE2198B7
:10D8900050F8346F31680E681D991CAA4FF00103CF
:10D8A000B0478DF86B0030B142F60014C2F20004AC
:10D8B000207202F018B80DF1A80C1CF8380DFAF718
:10D8C00093FBFCF7E0BE2198436B0DF1700C187AC6
:10D8D000FAF78AFBFCF7D7BE0DF1700C219A92F88B
:10D8E0003C00FAF781FBFCF7CEBE2199086CFF28BB
:10D8F00008D942F60014C2F200044FF0200323724C
:10D9000001F0F1BF0DF1700CC0B2FAF76DFBFCF73E
:10D91000BABE219850F8347F3D68AE68B04703EE38
:10D92000100AF8EE433A219AC2ED133AFCF7ABBE67
:10D93000219991ED0E4AF8EE444AC1ED134AFCF7E5
:10D94000A2BE219890ED105AF8EE455AC0ED135A38
:10D95000FCF799BE219B93ED136AFCEEC66ACDEDF0
:10D960001C6AEBE0219AD2ED137A9FEDB40AF4EE33
:10D97000C07AF1EE10FA08DB42F60014C2F200049D
:10D980004FF02001217201F0AEBFFCEEE70AC2EDBC
:10D99000100AFCF778BE219850F8346F33681E687F
:10D9A0001D991CAA4FF00403B0478DF86B0030B1ED
:10D9B00042F60012C2F20002107201F094BF1C98ED
:10D9C000FAF78CF9219FB864FCF75DBE219850F8F6
:10D9D000341F0E6836681D991CAA4FF00403B04727
:10D9E0008DF86B0030B142F60014C2F200042072D0
:10D9F00001F079BF1C98FAF771F9219DE864FCF7F2
:10DA000042BE2198436B1A68516841B942F6001032
:10DA1000C2F200004FF01E02027201F064BFC06C3F
:10DA2000FAF732F91C90219850F8346F33685E6829
:10DA30001D991CAA4FF00403B0478DF86B00002815
:10DA40003CF421AE42F60014C2F20004207201F050
:10DA50004ABF45F2A041C2F200010B7813F0280F33
:10DA60000BD0219AD16B1D9B581800F1FF30B0F5F7
:10DA7000805F34BF0020012009E02198C26B1D990E
:10DA80008B1803F1FF30FA2894BF0020012040B129
:10DA900042F60011C2F200014FF01300087201F0CB
:10DAA00022BF219B184650F8347F3E6836684FF0FD
:10DAB000000140F6D867C2F200071D9ABA18DB6B66
:10DAC000B0478DF86B0000283CF4DDAD42F6001441
:10DAD000C2F20004207201F006BF219850F8343FD2
:10DAE0001E6836681D991BAA4FF00403B0478DF8D5
:10DAF0006B0030B142F60014C2F20004207201F053
:10DB0000F2BE1B998AB2C1F3072040EA022399B200
:10DB10001C9113E01D9A1C921C982199FAF71AFB8C
:10DB20008DF86B0000283CF4AEAD42F60013C2F253
:10DB30000003187201F0D7BE1D981C901C98B0F518
:10DB4000803F08D342F60014C2F200044FF01F02D7
:10DB5000227201F0C8BE219DA863FCF794BD1D9DF3
:10DB6000219FFD63FCF78FBD1D9E21990E64FCF77C
:10DB70008ABD219A906B1D9BC11A1C91DEE71E9AEB
:10DB8000219BD96B8818FB2808D942F60013C2F2F2
:10DB900000034FF012021A7201F0A5BE45F2903751
:10DBA000C2F2000787F8FB10184650F8346F31684E
:10DBB0000E681D99BA18DB6BB0478DF86B00002812
:10DBC0003CF461AD42F60014C2F20004207201F090
:10DBD0008ABE219B586B0668766846B942F60010EB
:10DBE000C2F200004FF01E02027201F07CBE45F24C
:10DBF000A041C2F200010A7812F0280F0AD0DA6BB5
:10DC00001D99881800F1FF30B0F5805F34BF002007
:10DC1000012008E0D86B1D990A1802F1FF30FA289C
:10DC200094BF0020012058B142F60013C2F2000355
:10DC30004FF01301197201F056BE00BF000080477B
:10DC400003F134004FF0000140F6D867C2F200073C
:10DC50001D9ABA18DB6BB0478DF86B0000283CF4B6
:10DC600012AD42F60014C2F20004207201F03BBE75
:10DC7000F7F732F800287CF406AD1D9B1C93FEF7E5
:10DC8000E5BDF7F729F800283CF4FDAC1D991C917F
:10DC9000FEF7DCBD1D98072808D942F60014C2F231
:10DCA00000044FF00502227201F01DBEC0B24FF019
:10DCB0000001F6F7CFFF01EE100AB8EE417A219F7E
:10DCC00087ED137AFCF7DFBC1D9B072B08D942F6C2
:10DCD0000011C2F200014FF00500087201F003BE0E
:10DCE000D8B24FF00101F6F7B5FF01EE900AB8EE99
:10DCF000612A219D85ED132AFCF7C5BC1D9A072AD0
:10DD000008D942F60014C2F200044FF00503237252
:10DD100001F0E9BDD0B24FF00001F6F70BFFFCF7C0
:10DD2000B2BC1D99072908D942F60010C2F20000C2
:10DD30004FF00502027201F0D6BDC8B24FF00101EA
:10DD4000F6F7F8FEFCF79FBC1D9B072B08D942F69F
:10DD50000014C2F200044FF00501217201F0C3BDAE
:10DD6000D8B24FF00001F6F735FFFCF78CBC1D98D8
:10DD7000072808D942F60013C2F200034FF005024B
:10DD80001A7201F0B0BDC0B24FF00101F6F722FFE8
:10DD9000FCF779BC9DF87400F3F73AFD00287CF499
:10DDA00072AC42F60014C2F200044FF02801217256
:10DDB00001F099BD9DF87400219901F14C01F3F730
:10DDC00047FD00287CF45FAC42F60010C2F2000070
:10DDD0004FF02803037201F086BD219AD2ED132A79
:10DDE0009DF87400BCEEE23A13EE101AF3F762FDF0
:10DDF00000287CF448AC42F60014C2F200044FF054
:10DE00002801217201F06FBDFCF73DBC0DF1700CD3
:10DE1000FAF702F930B9219E96F847703D1C18BFF9
:10DE2000012501E04FF00105219880F84750FCF7EB
:10DE30002ABC9DF874600DF1700CFAF7EDF80146FC
:10DE400030464FF00102FBF7BFFC8DF86B00002855
:10DE50003CF419AC42F60013C2F20003187201F050
:10DE600042BD0DF1700CFAF7D7F801468DF86A0043
:10DE70009DF87400FBF766FC8DF86B0000283CF4FD
:10DE800002AC42F60012C2F20002107201F02BBD89
:10DE90001D991C914FF001038DF86A301E462198A0
:10DEA00090F8472013420AD090F846109DF8700071
:10DEB00019403246FBF788FC8DF86B0068B99DF875
:10DEC0006A304FEA43018DF86A101C9800F1010096
:10DED0001C9011F0FE03E2D10AE09DF86A20012AAD
:10DEE00006D142F60014C2F20004207201F0FBBC1D
:10DEF0004FF000068DF86B600DF1700CFAF78CF89E
:10DF00000DF1700CFAF788F8FCF7BDBB9DF87400B2
:10DF10004FF001010A46FBF757FC8DF86B00002813
:10DF20003CF4B1AB42F60011C2F20001087201F0FC
:10DF3000DABC9DF874004FF000014FF00102FBF7CE
:10DF400043FC8DF86B0000283CF49DAB42F60013B7
:10DF5000C2F20003187201F0C6BC0DF1700CFAF7A2
:10DF60005BF8219F97F84750284387F84700FCF754
:10DF70008ABB1D980DF1A80C4CF8380DFAF7ECFC93
:10DF800000287CF480AB45F29440C2F20000089A6D
:10DF9000026001F028BC10A8FAF77CFB014640B1F2
:10DFA0009DF84060022E04D0C2484FF00D0208F0E8
:10DFB000C5FA0DF1700C9DF84000FAF715F8FCF762
:10DFC00062BBFBF75BF8FCF75EBB0DF1700CFAF778
:10DFD00023F8FCF758BB1D9EFA2E08D942F6001410
:10DFE000C2F200044FF01203237201F07CBC0DF169
:10DFF000700CFAF711F845F29031C2F20001885521
:10E00000FCF741BB0DF1700CFAF706F845F29037BA
:10E01000C2F2000787F8FB00FCF735BB0DF1700C6E
:10E02000219D95F84700F9F7DFFFFCF72CBB1D9801
:10E03000FA2808D942F60011C2F200014FF012048A
:10E040000C7201F050BC0DF1700C45F29032C2F22E
:10E050000002105CF9F7C8FFFCF715BB0DF1700C5E
:10E0600045F29036C2F2000696F8FB00F9F7BCFFC5
:10E07000FCF709BB1D9EF62E08D942F60010C2F22D
:10E0800000004FF01202027201F02DBC219B986C2F
:10E09000F9F7FAFD45F29037C2F20007B851FCF7E4
:10E0A000F2BA45F2A041C2F200010B7813F0280F3A
:10E0B00006D01D98B0F5805F34BF0020012004E039
:10E0C0001D98FA2894BF0020012040B142F60014A8
:10E0D000C2F200044FF01302227201F004BC0DF1F1
:10E0E000700C40F6D865C2F200051D9EA85DF9F7D8
:10E0F0007BFFFCF7C8BA0DF1700CF9F7B5FF40F6DD
:10E10000D867C2F200071E99785C1D9B18420DF17A
:10E11000700C0CBF0020FF20F9F766FFFCF7B3BAC4
:10E1200045F2A042C2F20002117811F0280F08D087
:10E130001D9800F10100B0F5805F34BF0020012080
:10E1400006E01D9800F10100FA2894BF002001208C
:10E1500040B142F60011C2F200014FF013020A7200
:10E1600001F0C1BB1D9B40F6D862C2F20002D15C37
:10E17000D018437843EA01221C92002A3CF483AA77
:10E18000FEF764BB45F2A043C2F20003187810F01A
:10E19000280F06D01D99B1F5805F34BF0021012101
:10E1A00004E01D99FA2994BF0021012141B142F6F2
:10E1B0000014C2F200044FF01301217201F093BB6E
:10E1C00040F6D862C2F200021D9BD05C002856D1F6
:10E1D000FCF759BA45F2A042C2F20002137813F0DC
:10E1E000280F06D01D98B0F5805F34BF00200120B5
:10E1F00004E01D98FA2894BF0020012040B142F6A7
:10E200000014C2F200044FF01300207201F06BBB47
:10E2100040F6D861C2F200011D9A8B5C7BB3FCF71B
:10E2200032BA0DF1700CF9F7F7FE1C9038BBFCF711
:10E230002ABA0DF1700CF9F717FF40F6D861C2F257
:10E2400000011E9A885C1D9B184218D0FCF71BBA6F
:10E250000DF1700CF9F708FF40F6D861C2F2000129
:10E260001E9A885C1D9B184209D1FCF70CBA0DF16F
:10E27000700CF9F7D1FE1C9000287CF404AA219BB5
:10E28000186A40B942F60014C2F200044FF00301CC
:10E29000217201F028BB00F1FF351D6200F1010081
:10E2A00053F8207045F29446C2F200063760FCF73E
:10E2B000EAB900BFDE0E002098F8005045F02001BA
:10E2C00088F80010FCF708BA219E96F847704FEACC
:10E2D000D71242EA470086F84700FCF7D4B9219BE1
:10E2E00093F847504FEA550141EAC51683F8476055
:10E2F000FCF7C9B9FAF7A0FAFCF7C5B942F60C1752
:10E30000C2F20007FA784FF0010000FA02F03B7900
:10E3100023EA00033B71FCF7B6B942F60014C2F2DF
:10E3200000044FF00101217201F0DDBA42F60C1534
:10E33000C2F20005EE7846B942F60C10C2F20000B7
:10E340004FF00603C370FCF79EB906F1FF3742F6A3
:10E350000C12C2F20002D770FCF795B942F60C110C
:10E36000C2F200010D7805F1FF36F7B20F700A799D
:10E37000FF2A0BD1632F7CF686A942F60C11C2F25C
:10E3800000014FF063050D70FCF77DB9172F7CF687
:10E390007AA942F60C10C2F200004FF01703037086
:10E3A000FCF771B942F60C16C2F20006777807F155
:10E3B000FF32D0B270703379FF2B0BD100287CF480
:10E3C00062A942F60C16C2F200064FF00C077770F5
:10E3D000FCF759B93B287CF656A942F60C11C2F25B
:10E3E00000014FF03B054D70FCF74DB942F60014AB
:10E3F000C2F200044FF00102227201F074BA42F638
:10E400000010C2F200004FF00103037201F06BBA7A
:10E4100042F60011C2F200014FF001040C7201F04B
:10E4200062BA42F60010C2F200004FF0010202721E
:10E4300001F059BA42F60C15C2F20005EE78052E2D
:10E4400008D942F60C13C2F200034FF00001D97054
:10E45000FCF719B906F1010642F60C17C2F20007E3
:10E46000FE70FCF710B942F60C10C2F20000027800
:10E4700002F10102D5B205700679FF2E0BD1632D92
:10E480007CF601A942F60C11C2F200014FF0000027
:10E490000870FCF7F8B8172D7CF6F5A842F60C17B3
:10E4A000C2F200074FF000033B70FCF7ECB842F6F5
:10E4B0000C12C2F20002557805F10105EEB2567059
:10E4C0001779FF2F0BD10C2E7CF6DDA842F60C102D
:10E4D000C2F200004FF001024270FCF7D4B83B2EAC
:10E4E0007CF6D1A842F60C13C2F200034FF00001F3
:10E4F0005970FCF7C8B842F60014C2F200044FF09D
:10E500000103237201F0EFB942F60C15C2F20005C7
:10E51000EE784FF0010707FA06F7297987EA01003C
:10E520002871FCF7B0B80DF1700CF9F775FD42F6E3
:10E530000C12C2F200021071FCF7A5B80DF1700CBC
:10E54000F9F76AFD062842F60C13C2F2000392BFE7
:10E55000D8700025DD70FCF796B80DF1700CF9F756
:10E560005BFD42F60C16C2F200063070FCF78BB869
:10E570000DF1700CF9F750FD42F60C17C2F20007CE
:10E580007870FCF780B80DF1700CF9F745FD42F694
:10E590000C11C2F200018870FCF775B80DF1700C17
:10E5A00042F60C10C2F200000079F9F71DFDFCF7ED
:10E5B0006AB80DF1700C42F60C12C2F20002D0786B
:10E5C000F9F712FDFCF75FB80DF1700C42F60C1371
:10E5D000C2F200031878F9F707FDFCF754B80DF103
:10E5E000700C42F60C15C2F200056878F9F7FCFCD5
:10E5F000FCF749B80DF1700C42F60C16C2F2000699
:10E60000B078F9F7F1FCFCF73EB842F60014C2F21C
:10E6100000044FF00101217201F065B91D9A0F2A23
:10E6200008D942F60014C2F200044FF0270020720D
:10E6300001F059B941F6D867C2F2000707EB820032
:10E6400042F60C13C2F2000317F822501D704678F0
:10E650005E704FF000019970D97082781A71FCF7E2
:10E6600012B842F60013C2F200034FF00101197212
:10E6700001F039B942F60C17C2F20007FD784FF0ED
:10E68000010606FA05F63A7946EA02003871FBF708
:10E69000FABF42F60014C2F200044FF001032372E5
:10E6A00001F021B942F60011C2F200014FF001025F
:10E6B0000A7201F018B94FF00007139712971197DB
:10E6C000199742F60C15C2F200052E7806F1640681
:10E6D0001696687800F1FF331593A978149111A864
:10E6E00007F052FD179A1AB102F1FF35EFB201E0BF
:10E6F0004FF0060742F60C16C2F20006F770FBF761
:10E70000C2BF1D9A0F2A08D942F60014C2F20004B3
:10E710004FF02702227201F0E6B841F6D860C2F24B
:10E72000000000EB820142F60C13C2F200031F78D6
:10E7300000F822705D784D701E798E70FBF7A3BFD4
:10E7400042F60010C2F200004FF00101017201F028
:10E75000CAB80DF1700C219B93F85000F9F744FCF6
:10E76000FBF791BF45F2A044C2F20004227812F0F8
:10E77000010F08D142F60010C2F200004FF0300144
:10E78000017201F0B0B842F6C400C2F200000168A4
:10E7900041B942F60014C2F200044FF03102227275
:10E7A00001F0A1B845F2A043C2F200031C7804F0C6
:10E7B000FE0242F00400187042F6B001C2F20001FD
:10E7C0004FF000030B6000F0F7BF45F2A043C2F228
:10E7D00000031C7814F0010F08D142F60010C2F2B9
:10E7E00000004FF03002027201F07DB842F6C40220
:10E7F000C2F20002106840B942F60013C2F20003F0
:10E800004FF034041C7201F06EB845F2A041C2F220
:10E8100000010B7803F0FE0444F002020A7042F695
:10E82000B000C2F200004FF00001016000F0C4BF70
:10E83000219F97F846500DF1700CF9F7EDFB219EE2
:10E84000291A96F8503003F001000A1A1C9286F833
:10E850004720FF2A94BF0022012286F85020FBF7B0
:10E8600012BF45F2A041C2F200010B7813F0280F4D
:10E8700006D01D98B0F5805F34BF0020012004E071
:10E880001D98FA2894BF0020012040B142F60014E0
:10E89000C2F200044FF01302227201F024B840F6D5
:10E8A000D867C2F200071E9D1D9EBD55FBF7EBBE4B
:10E8B0004FF000011C911AE04FF001031C9316E089
:10E8C0004FF002001C9012E04FF003071C970EE07F
:10E8D0004FF004051C950AE04FF005061C9606E073
:10E8E0004FF006021C9202E04FF007011C911D99A7
:10E8F0001B911C98F9F7B4FFFBF7C5BE0DF1700C26
:10E90000F9F7B2FB1E9B40F6D867C2F20007F85C2D
:10E910001D9D0543FD54FBF7B6BE1D9BF92B08D981
:10E9200042F60014C2F200044FF01201217200F00E
:10E93000DABF45F29036C2F200061E9AF254FBF797
:10E94000A2BE45F29037C2F200071D9887F8FB007F
:10E95000FBF799BE45F23873C2F200031A6842B958
:10E9600042F60010C2F200004FF00101017200F007
:10E97000BABF56681D981E994FF001020DF16A0347
:10E98000B0478DF86B009DF86A10D1F1010238BFD5
:10E990000022219B83F8502000283BF474AE42F6FD
:10E9A0000014C2F20004207200F09DBF45F23872DC
:10E9B000C2F20002136843B942F60010C2F200002E
:10E9C0004FF00101017200F08EBF1A681D981E9968
:10E9D00090478DF86B0000283BF455AE42F60014CA
:10E9E000C2F20004207200F07EBF45F23873C2F21A
:10E9F00000031A6842B942F60010C2F200004FF05C
:10EA00000101017200F06FBF56681D981E994FF00A
:10EA100000020DF16A03B0478DF86B009DF86A1093
:10EA2000D1F1010238BF0022219B83F85020002839
:10EA30003BF429AE42F60014C2F20004207200F04A
:10EA400052BF09981E99F9F705FD099040B942F6A1
:10EA50000013C2F200034FF01700187200F043BF1A
:10EA6000099A13689B6A43B942F60011C2F2000189
:10EA70004FF015020A7200F036BF099880689DF8C1
:10EA8000741045F29032C2F2000298478DF86B0084
:10EA900000283BF4F8AD42F60014C2F200042072E4
:10EAA00000F021BF09981E99F9F7D4FC099040B9EC
:10EAB00042F60013C2F200034FF01700187200F084
:10EAC00012BF09990A68536943B942F60011C2F2AC
:10EAD00000014FF015020A7200F005BF0998806826
:10EAE0009DF8741045F29032C2F2000298478DF8FA
:10EAF0006B0000283BF4C7AD42F60014C2F20004DC
:10EB0000207200F0F0BE09981E99F9F7A3FC099055
:10EB100040B942F60013C2F200034FF017021A7216
:10EB200000F0E1BE099F39688F6947B942F60010CD
:10EB3000C2F200004FF01501017200F0D4BE45F2A0
:10EB40009036C2F20006099A90689DF87410324619
:10EB50000DF16A03B8478DF86B009DF86A30337089
:10EB600000283BF490AD42F60014C2F2000420727B
:10EB700000F0B9BE09981E99F9F76CFC09901D992F
:10EB80007F2909D1051C18BF012545F29036C2F234
:10EB900000063570FBF777BD099840B942F60013BF
:10EBA000C2F200034FF01700187200F09CBE099BE0
:10EBB0001A68536843B942F60011C2F200014FF0DF
:10EBC00015020A7200F08FBE09988068C9B245F23A
:10EBD0009032C2F2000298478DF86B0000283BF497
:10EBE00052AD42F60014C2F20004207200F07BBE67
:10EBF00009981E99F9F72EFC099040B942F60013C6
:10EC0000C2F200034FF017021A7200F06CBE099FA7
:10EC100039688F6847B942F60010C2F200004FF021
:10EC20001501017200F05FBE45F29036C2F2000697
:10EC3000099A90689DF8741032780DF16A03B8470C
:10EC40008DF86B009DF86A30337000283BF41BADE3
:10EC500042F60014C2F20004207200F044BE09988B
:10EC60001E99F9F7F7FB099040B942F60011C2F27C
:10EC700000014FF017030B7200F035BE099F386892
:10EC8000C76847B942F60010C2F200004FF0150203
:10EC9000027200F028BE45F29036C2F200060999D1
:10ECA00088689DF8741032460DF16A03B8478DF8F4
:10ECB0006B009DF86A30337000283BF4E4AC42F6F8
:10ECC0000014C2F20004207200F00DBE09981E99D3
:10ECD000F9F7C0FB099040B942F60010C2F20000FB
:10ECE0004FF01702027200F0FEBD099F38680769F5
:10ECF00047B942F60011C2F200014FF015030B7242
:10ED000000F0F1BD099ED6F808809DF8749045F298
:10ED10009036C2F200063068F8F7E0FF024640463F
:10ED200049460DF16A03B8478DF86B009DF86A20DB
:10ED3000327000283BF4A7AC42F60014C2F2000483
:10ED4000207200F0D0BD09984FF00001F9F782FB66
:10ED5000099040B942F60013C2F200034FF01700C9
:10ED6000187200F0C0BD09990B68DB6A43B942F61E
:10ED70000011C2F200014FF015020A7200F0B3BD9B
:10ED8000099880689DF8741098478DF86B000028EA
:10ED90003BF479AC42F60014C2F20004207200F099
:10EDA000A2BD09981E99F9F755FB099040B942F6A2
:10EDB0000013C2F200034FF01700187200F093BD69
:10EDC00009990A68D36943B942F60011C2F20001F9
:10EDD0004FF015020A7200F086BD099880689DF810
:10EDE000741045F29032C2F2000298478DF86B0021
:10EDF00000283BF448AC42F60014C2F20004207232
:10EE000000F071BD09981E99F9F724FB099040B9EB
:10EE100042F60013C2F200034FF01700187200F020
:10EE200062BD09990A68136A43B942F60011C2F239
:10EE300000014FF015020A7200F055BD0998806874
:10EE40009DF8741045F29032C2F2000298478DF896
:10EE50006B0000283BF417AC42F60014C2F2000429
:10EE6000207200F040BD09981E99F9F7F3FA099055
:10EE700040B942F60011C2F200014FF017030B72C5
:10EE800000F031BD09990A68536A43B942F600108F
:10EE9000C2F200004FF01502027200F024BD099882
:10EEA00080689DF8741010AA98478DF86B00109830
:10EEB000F8F7EAFE45F29031C2F2000108609DF8D1
:10EEC0006B30002B3BF4DFAB42F60014C2F20004BF
:10EED000237200F008BD09984FF00001F9F7BAFA63
:10EEE000099040B942F60013C2F200034FF0170137
:10EEF000197200F0F8BC09980268136B43B942F626
:10EF00000010C2F200004FF01502027200F0EBBCDC
:10EF1000099988689DF8741045F29032C2F2000297
:10EF200098478DF86B0000283BF4ADAB42F6001417
:10EF3000C2F20004207200F0D6BC1D98072808D940
:10EF400042F60014C2F200044FF00803237200F0EE
:10EF5000CABC42F66005C2F2000555F83070002FB9
:10EF60007BF491ABF7F750FB002808BF012042F675
:10EF70006006C2F200061D9A46F83200FBF783BB1A
:10EF80001D99072908D942F60014C2F200044FF077
:10EF90000801217200F0A7BC42F66000C2F2000036
:10EFA00050F83150002D3BF46EABF7F72DFB1D9F51
:10EFB00042F66006C2F2000656F83720831A1C9308
:10EFC00006EBC701486883428CBF0020C3EB0000FA
:10EFD0001B9042F66005C2F2000505EBC7061B9ABE
:10EFE00072604FF0000345F83730FBF74CBB45F239
:10EFF000A040C2F20000027812F0280F06D01D9B3C
:10F00000B3F5805F34BF0023012304E01D9BFA2B7E
:10F0100094BF0023012343B142F60014C2F200045E
:10F020004FF01301217200F05EBC1D9F0DF1700CBA
:10F03000F8F7F2FF40F6D865C2F20005E855FBF795
:10F0400022BB0DF1700CF9F70FF80DF1700CF8F709
:10F05000E3FF1C9050B11E9D40F6D866C2F2000638
:10F06000725D1D9911437155FBF70DBB1E9E40F655
:10F07000D862C2F20002905D1D9B20EA03079755FB
:10F08000FBF701BB1D9B1E9AD018C1B245F2903010
:10F09000C2F2000080F8FB10FA2908D942F60014E9
:10F0A000C2F200044FF01203237200F01CBC45F2C0
:10F0B0009447C2F200073D6845F29036C2F200065E
:10F0C000F0184CF60003C0F60103E91807F036FA11
:10F0D0003A681E9950183860FBF7D5BA45F2A0423D
:10F0E000C2F20002117811F0280F08D01D9800F12B
:10F0F0000200B0F5805F34BF0020012006E01D98BB
:10F1000000F10200FA2894BF0020012038B142F635
:10F110000014C2F200044FF013022272E3E3F7F787
:10F1200073FA00F104004CF6CD47CCF6CC47A7FBB0
:10F1300000154FEA9506219B5A6AB6FBF2F71C9719
:10F140001D9D40F6D861C2F200014FEA17404855B4
:10F150004E194FEA17237370B770FBF794BA45F254
:10F16000A041C2F20001087810F0280F08D01D9BC2
:10F1700003F10203B3F5805F34BF0023012306E0EF
:10F180001D9B03F10203FA2B94BF002301233BB123
:10F1900042F60014C2F200044FF013022272A2E3FE
:10F1A000F7F732FA00F104004CF6CD47CCF6CC4725
:10F1B000A7FB00254FEA9506219A516AB6FBF1F0AC
:10F1C0001D9B40F6D867C2F20007FE187578FA5CFE
:10F1D0004FEA024141EA0527B37847EA03061B9646
:10F1E000801B20F07F451C950DF1700C1E98854208
:10F1F0002CBF00200120F8F7F7FEFBF744BA219955
:10F2000091F846700DF1700CF8F706FF3E1A1C9647
:10F21000219B83F84760FF2E94BF0026012683F8C8
:10F220005060FBF730BA45F2A040C2F2000002780D
:10F2300012F0280F08D01D9901F10101B1F5805F8E
:10F2400034BF0021012106E01D9901F10101FA29D5
:10F2500094BF0021012139B142F60013C2F200032C
:10F260004FF013021A723EE31D9A45F29443C2F224
:10F2700000031B6840F6D861C2F200014FEA132078
:10F2800088548A185370FEF7FABF219890F84750B7
:10F290001C9590F8467080F8477080F84650FBF750
:10F2A000F2B91D98072807D942F60014C2F20004EB
:10F2B0004FF00801217216E3F9F7FAFA0DF1A80CE4
:10F2C0004CF8380D003018BF0120F8F78DFEFBF721
:10F2D000DAB9219E96F8470096F846300DF1700C89
:10F2E000984214BF00200120F8F77EFEFBF7CBB94F
:10F2F000219A92F8470092F846500DF1700C401B8D
:10F3000018BF0120F8F770FEFBF7BDB9219F97F8F1
:10F31000470097F846100DF1700C88422CBF002072
:10F320000120F8F761FEFBF7AEB9219E96F8470081
:10F3300096F846300DF1700C984294BF00200120E1
:10F34000F8F752FEFBF79FB9219A92F8470092F81E
:10F3500046500DF1700CA8428CBF00200120F8F738
:10F3600043FEFBF790B9219F97F8470097F84610A6
:10F370000DF1700C884234BF00200120F8F734FEF4
:10F38000FBF781B91D98F62807D942F60014C2F29E
:10F3900000044FF012022272A5E245F29036C2F24A
:10F3A00000063058F8F79AFC219BD864FBF76BB93C
:10F3B0001D99F62907D942F60010C2F200004FF05D
:10F3C000120303728FE245F29035C2F200056858CD
:10F3D000F8F784FC219FB864FBF755B945F29032E9
:10F3E000C2F2000292F8FB201D9BD118FB2907D91D
:10F3F00042F60013C2F200034FF01201197272E2DA
:10F4000045F2A040C2F20000017811F0280F09D0A7
:10F410001E99501800F1FF30B0F5805FB4BF002096
:10F42000012007E01E98111801F1FF30FA28D4BF1F
:10F430000020012038B142F60014C2F200044FF05F
:10F44000130222724FE240F6D866C2F200061E9DF9
:10F45000701945F29037C2F20007F91807F06EF8FC
:10F46000FBF711B92198466B326856683EB942F6EF
:10F470000013C2F200034FF01E01197233E21E9A0C
:10F4800045F29033C2F2000393F8FB309918FB2940
:10F4900007D942F60010C2F200004FF012020272C9
:10F4A00021E200F134001D9945F29037C2F20007C5
:10F4B000BA18B0478DF86B0000283BF4E4A842F678
:10F4C0000014C2F2000420720DE242F60014C2F2EF
:10F4D00000044FF00100207205E20DF1700CF8F706
:10F4E000C3FD40F6D865C2F200051E9FEE5D1D9A71
:10F4F00016423BF4C8A845F29443C2F200030899AF
:10F50000196070E10DF1700CF8F7AEFD40F6D860AF
:10F51000C2F200001E9D475D1D9E37427BF4B3A8DA
:10F5200045F29444C2F20004089A22605BE19DF81F
:10F5300074000DF16B01FAF737F88DF86A009DF849
:10F540006B302BB142F60014C2F200042372CAE100
:10F5500000283BF498A845F29440C2F200000899B4
:10F56000016040E19DF874000DF16B01FAF71CF8A1
:10F57000D0F1010238BF00228DF86A209DF86B108F
:10F5800029B142F60012C2F200021172ABE1219DD4
:10F59000EF6A17B98DF86A7002E09DF86A6066B983
:10F5A0000DF1700C1E98F9F7D7F930B945F2944473
:10F5B000C2F200040898206015E10DF1700C9DF86E
:10F5C0006A00F8F711FD4FF00002219BDA62FBF7A9
:10F5D0005AB89DF874000DF16B01F9F7E5FF8DF84D
:10F5E0006A009DF86B302BB142F60010C2F20000A9
:10F5F000037278E100287BF446A845F29445C2F2F4
:10F600000005089F2F60EEE09DF874000DF16B017E
:10F61000F9F7FAFF8DF86A009DF86B1029B142F6F0
:10F620000012C2F2000211725DE100287BF42BA8E7
:10F6300045F29446C2F20006089C3460D3E09DF87F
:10F6400074000DF16B01F9F7DFFF031C18BF0123F4
:10F650008DF86A3092E79DF874000DF16B01F9F7AF
:10F66000A3FF003018BF01208DF86A0086E71D9EB9
:10F67000F62E07D942F60013C2F200034FF012042F
:10F680001C7230E12199C86CF8F7FEFA45F290350A
:10F69000C2F20005A851FAF7F6BF0DF1700CF8F7A9
:10F6A000BBFC219F97F84760D6F1010238BF0022CA
:10F6B000002814BF104682F0010087F84700FAF7CF
:10F6C000E2BF0DF1700CF8F7A7FC219991F84750B3
:10F6D000684081F84700FAF7D6BF0DF1700CF8F7D3
:10F6E0009BFC219B83F85100FAF7CDBF05F0B8FCD5
:10F6F0000DF1A80C4CF8380DFF2828BFFF20C0B230
:10F70000F8F772FCFAF7BFBF05F0A0FC0DF1A80CEA
:10F710004CF8380DFF2828BFFF20C0B2F8F764FC72
:10F72000FAF7B1BF05F0A6FC0DF1A80C4CF8380DA6
:10F73000FF2828BFFF20C0B2F8F756FCFAF7A3BF96
:10F7400005F07AFC0DF1700C00280CBFFF200020A2
:10F75000F8F74AFCFAF797BF45F28C42C2F2000272
:10F7600010681D99401804F0D9FF8DF86B0000282F
:10F770003AF489AF42F60014C2F200042072B2E0FB
:10F780001D9804F089FFFAF77EBF0DF1700CF8F7B1
:10F7900043FC04F07BFFFAF776BF45F28C47C2F2D8
:10F7A00000073E681D9D701904F092FFFAF76BBFC9
:10F7B00004F076FFFAF767BF42F6C403C2F2000313
:10F7C0001A6882B945F2A040C2F20000017801F047
:10F7D0000204E3B23BB142F60014C2F200044FF05F
:10F7E000350323727FE045F2A047C2F200073E785E
:10F7F00016F0010F7AF445AF219D2DB145F29442E8
:10F80000C2F200021068686042F6B001C2F2000164
:10F810000C687F2C00F2A28004F101041B941C945C
:10F8200014B94FF001071B9742F63C16C2F20006CE
:10F830004FF0540545F2A044C2F2000442F6C4075A
:10F84000C2F200071C9B05FB036221929BB9217841
:10F8500001F00400C1B209B9386840B9217841F01B
:10F8600001006FF382002070506840B115E04FF046
:10F8700001021C92E6E7506878B9802B02D003F1B0
:10F88000010301E04FF000031C931B9A9342D9D16E
:10F890004FF00000F9F7DEFBD4E742F6B006C2F203
:10F8A0000006336045F29445C2F2000528604FF02F
:10F8B000000A5446FAF7E7BE219F396A41F000403A
:10F8C0003863FAF7E0BE4FF00006219D2E63FAF789
:10F8D000DABEFAF7D8BE0B9D42F60014C2F200045D
:10F8E0004FF00102227242F60010C2F20000089CA2
:10F8F0000460219B1A6A22B102F1010253F822101E
:10F90000089142F60010C2F20000089C4460457263
:10F91000F2F756F9F2F754F9219D2B6A7BB14FF0BB
:10F9200000021C922199086A48B1F2F749F91C9C1F
:10F9300004F101041C94219D2B6AA342F5D84FF0D9
:10F940000000F9F787FBFAF7D2BD4FF0000703F18B
:10F95000FF344FF000035E46FDF7E0BB4FF00003BD
:10F960001C935EE74FF002031C9342F63C12C2F276
:10F970000002D2F8AC0030B9FDF71DBE2BB0BDECD3
:10F98000048BBDE8F08F03F1010302F15402FDF78F
:10F990000EBE05F1010302F15402812B7DF407AE86
:10F9A000FDF75EBEBEF1000F3DF43DAB10F80390D5
:10F9B00001F8039003F1010393427DF434ABFDF7AA
:10F9C00040BBF9180EEB030C13F8016F02F1FF3581
:10F9D000B0423DF4BAA82A46FDF7C6B805F1FF3299
:10F9E000FDF7C2B838B5054642F6A004C2F20004DD
:10F9F0002068F6F73BFA4FF0000323608DB14AF61A
:10FA0000E840C0F601004FF007014AF28142C0F61B
:10FA10000002F6F741F942F6AC01C2F200010860BB
:10FA200038BD42F6AC04C2F200042068F6F71EFAB4
:10FA30004FF000002060F5F7F5FBFAF791FC04F0B9
:10FA40009BFE42F6A801C2F200010A884FF6FF733E
:10FA50009A4204D0D0B24FF00401FAF7F9FB38BD56
:10FA600070B542F61410C2F200004AF6F841C0F632
:10FA70000101F5F741FD42F6A803C2F200034FF67B
:10FA8000FF721A8041F61874C2F200044FF00406A7
:10FA900084F820624FF00005C4F81C522846F5F7A0
:10FAA00015FF206084F86464C4F860544FF00100CE
:10FAB000F5F70CFFC4F8440284F8A866C4F8A4560D
:10FAC0004FF00200F5F702FFC4F8880484F8EC68F0
:10FAD000C4F8E8584FF00300F5F7F8FEC4F8CC0678
:10FAE00042F62800C2F200004AF60451C0F60101B5
:10FAF000F5F702FD42F6C800C2F200004AF2F861D2
:10FB0000C0F601012A462B46F9F742FDF8F7C0FB83
:10FB10004FF00100FFF766FF70BD00BF000000005E
:10FB20002DE9F04F2DED028B8FB04FF0000842F61B
:10FB3000AC07C2F2000742F6A003C2F2000303932F
:10FB400042F6A80BC2F2000B41F61876C2F200068C
:10FB50009FEDB98B39684FF0FF3041B9F2F730F8BB
:10FB6000386800280CBFFA204FF0FF30FFE7F6F7A7
:10FB7000D1F828B1B8F1320F09D808F1010806E030
:10FB8000B8F1330F0CBF4FF034084FF000083A685B
:10FB9000D2B9F2F715F8B8F1320F0ED1039C2068F4
:10FBA000F6F764F94FF00005039B1D60F5F73AFB8B
:10FBB0004FF00200F9F78CF906E0B8F1340F03D1E9
:10FBC0004FF00100F9F784F9BBF800104FF4117001
:10FBD00000FB0162D2F81842002CBBD04FF4117523
:10FBE00005FB01F303F5887406EB0409315DE02998
:10FBF0000CD199F801000E2808D14FF6FF70494644
:10FC0000D9F80021F7F7DAFF10B392E2325D02F083
:10FC10001F0509EB05035A78294605F0010019F87C
:10FC20000550521B01F1FF33002940F09F820BE089
:10FC300019F80300151A03F1FF3119F80120AA1A67
:10FC400001F1FF330029F3D112F0FF0F40F0718270
:10FC5000335D4FEA5310072800F26382DFE810F0AB
:10FC60000800610261023500A60061028A002601D7
:10FC7000335D09F1010513F01F0000F05A8209F10C
:10FC8000020905F1020500F1FF3255FA82F40294EF
:10FC90004FF000054FF0010A15E019F8011CE8B219
:10FCA00021405246F9F790FD002840F0428205F1CC
:10FCB00001054FEA4404FF2CEFD909F1010902992B
:10FCC000894500F036825446E7E799F801403868E4
:10FCD00070B1F6F7CBF84FF000003860F5F7A2FAF4
:10FCE000FAF73EFB4FF00100F9F7F2F8F1F768FF81
:10FCF00003990B686BB94AF60C50C0F601004FF03F
:10FD0000070149F6B932C0F60002F5F7C5FF039DB9
:10FD1000286005A84FF00001F9F708FB7CB9F6F759
:10FD200073FCC1B201F1FF33DDB2FD2D45F2A440F9
:10FD3000C2F2000092BF01700122027009E045F298
:10FD4000A440C2F20000027802FB04F404EB142485
:10FD5000047045F2A444C2F2000421780EAB03F80B
:10FD6000241D4FF003004FF000014FF01A02F9F785
:10FD7000D3F8EFE60DF11300F8F78CFC01469DF87F
:10FD800013508DF81450012D06D828B10DF115002F
:10FD90004FF00D0206F0D2FB4FF006004FF00001CD
:10FDA0004FF00E0205ABF9F7B7F8D3E6BBF8003019
:10FDB0004FF4117101FB03F499F80100032872D884
:10FDC000DFE800F002263E504FF00100FFF70AFE88
:10FDD0004FF000050EAB03F8255D4FF004002946F7
:10FDE0004FF00102F9F798F84FF0C800F7F7CEFE90
:10FDF00032599BF800004FF0010400940195D2F8AD
:10FE00000CC04FF416512A464FF00803E0478DE12D
:10FE10004FF0000142F60013C2F2000319724FF0D6
:10FE200001040EAB03F8254D4FF004002246F9F70C
:10FE300073F87BE1AFF300800000000000E06F404A
:10FE4000F9F71CF90EAB4FF0020103F8251D4FF036
:10FE500004004FF000014FF00102F9F75DF84FF098
:10FE6000010463E10EAB4FF0120203F8252D4FF0B1
:10FE700004004FF000014FF00102F9F74DF84FF088
:10FE8000C800F7F783FE35599BF800004FF00104D6
:10FE900000944FF000020192ED684FF416414FF0CC
:10FEA0000803A84742E14FF000043FE199F802E05F
:10FEB00099F8035099F80110A1F102010E2900F2FE
:10FEC0003381DFE811F00F00690081003101310159
:10FED0003101310131013101310131013101C20002
:10FEE00031019D00315DC1F30400C5B2012D00F068
:10FEF000208109F1050509F1080400EBC00200EBBF
:10FF0000420303EBC30101F15401C8B200EB40020C
:10FF1000A418C5EB040CACF1030E0EF0010A99F81D
:10FF2000029015F8010C05F0AFF853EC182B05F012
:10FF3000BDFB05F083F901464846F9F7ADFC05F134
:10FF40000305A54240F0F880F3E015F8039C15F88E
:10FF5000010C05F099F853EC182B05F0A7FB05F000
:10FF60006DF901464846F9F797FC05F1030515F8C8
:10FF700003AC15F8010C05F087F853EC182B05F0CD
:10FF800095FB05F05BF901465046F9F785FC05F154
:10FF90000305A542D9D1CCE0305DC0F30402A2F143
:10FFA0000302D2B209F103010EEB0204FF2CC4BF1D
:10FFB000CEF10002D2B240F6D863C2F2000303EBE6
:10FFC0000E0006F0BBFAB4E00EAC04F824ED0DF11F
:10FFD000150040F6D863C2F2000303EB0E01202D9A
:10FFE00034BF2A46202206F0A9FA05F101054FF098
:10FFF00007004FF00301EAB22346F8F78DFFA9E5A9
:020000040801F1
:1000000099F804A005EB0E24A3B24FEA132242EAAA
:1000100003200EAD25F8240D0DF1160040F6D86131
:10002000C2F20001C918BAF11D0F34BF52461D2299
:1000300006F084FA0AF102044FF007004FF01001B5
:10004000E2B22B46F8F768FF84E5BEF1000F16D147
:10005000ADB904F091FB039B1868F5F707FF4FF06B
:100060000000039A1060F5F7DDF84AF61C50C0F660
:10007000010008F055F8F9F7E1F8002848D099F8A0
:10008000025099F803104AF62C50C0F6010041EADC
:10009000052108F045F899F803A0494611F8024FE8
:1000A0004CF60003C0F6010303EB042540F6D864C8
:1000B000C2F2000404EB0A0001F102014FF08002D9
:1000C00006F03CFA4FF68070CFF6FF70CAEB0002E4
:1000D000D1B2601869184FF0800206F02FFA20465E
:1000E00029464FF48072F2F761F9A0B920462946FB
:1000F0004FF4807205F0CCFD80B94FF001004FF055
:1001000000010A460B46F8F707FF4FF001040DE027
:100110004FF000040AE04FF0000407E04FF0000445
:1001200004E04FF0000401E04FF00004002C7FF4E5
:1001300011ADF8F791FA0DE5BAF1000F3FF405AFF4
:1001400015F803AC15F8010C04F09EFF53EC182BC6
:1001500005F0ACFA05F072F801465046F9F79CFB41
:1001600005F10305A5427FF4F0AEE2E700283FF475
:100170005FAD19F80310521A03F1FF33B3F1FF3FDB
:100180007FF456AD60E500BF704700BF704700BF09
:1001900042F6B403C2F200031B684B634BB19A688A
:1001A000824209D0DB684B631BB19A688242F9D165
:1001B00002E04FF01E0070474FF00000704700BF94
:1001C00045F2A643C2F200031A78027045F2A54038
:1001D000C2F2000003780B70704700BF45F2A643DF
:1001E000C2F200031B78834225D845F2A542C2F231
:1001F000000212789A18904220DAC01A4FEA50038F
:100200004FF0010202FA03F310F0010F09D045F29A
:10021000B040C2F20000026813400B704FF00100C2
:10022000704745F2A840C2F20000026813400B700C
:100230004FF0010070474FF0000070474FF0000092
:10024000704700BF10B545F2A643C2F200031B7809
:1002500083427AD845F2A542C2F2000212789A1877
:10026000904275DAC31A03F0FE0445F2B440C2F2BC
:1002700000000278A418E4B24FEA53024FF00100E4
:1002800000FA02F213F0010F12D041B145F2B04072
:10029000C2F20000016842EA010303601AE045F27D
:1002A000B040C2F20000036823EA0203036011E0D9
:1002B00041B145F2A840C2F20000036842EA0301DE
:1002C000016007E045F2A843C2F20003196821EA81
:1002D0000201196045F2A840C2F2000001680A421A
:1002E00024D045F2B043C2F20003186802420ED097
:1002F00020464FF00001F1F773FA04F10102D0B289
:100300004FF00101F1F76CFA4FF0010010BD2046EB
:100310004FF00101F1F764FA04F10101C8B24FF0A6
:100320000001F1F75DFA4FF0010010BD20464FF0DB
:100330000001F1F755FA04F10102D0B24FF00001CB
:10034000F1F74EFA4FF0010010BD4FF0000010BD64
:100350004FF0000010BD00BF08B545F2B443C2F233
:100360000003187045F2AC43C2F20003197045F265
:10037000A643C2F200031A70091A01F10101C8B2C2
:1003800045F2A542C2F200021070412801D9F0F7EF
:1003900055FC40F2F410C2F200004FF00101F9F7F1
:1003A00073F808BD2DE9F84345F2B543C2F20003E6
:1003B00018784FEA400111F0FF0405D045F2B5422C
:1003C000C2F20002147006E045F2B545C2F2000523
:1003D0004FF001062E7045F2D847C2F20007387878
:1003E00045F2B543C2F20003197808420CBF4FF042
:1003F00000094FF001094FF000052C464FF00107AE
:1004000045F2B846C2F20006A84604F01F0207FAF9
:1004100002F0AB59184204D0204649464246F9F74B
:10042000D3F904F10104E4B214F01F0FEDD105F18A
:100430000405202DE9D1BDE8F88300BF45F2D8437B
:10044000C2F20003187045F2B540C2F200004FF04E
:1004500001020270704700BF00B583B045F2B8409A
:10046000C2F200004FF000014FF00802F0F748FC24
:100470004FF0000300934FF00100019045F2DC4083
:10048000C2F200004FF47A714FF0060240F2A53339
:10049000C0F60103F6F782F803B000BD08B545F2D7
:1004A000DC40C2F20000F5F7D3FF4FF0CC00FFF7BD
:1004B000C5FF08BD89B14FEA501245F2B843C2F2F8
:1004C000000300F01F004FF0010101FA00F053F8A3
:1004D0002210084343F8220011E04FEA501245F27F
:1004E000B843C2F2000300F01F004FF0010101FA0F
:1004F00000F053F8221021EA000143F822104FF0D7
:100500000000704708B54FF440404AF64C51C0F621
:10051000010145F20052C2F20002F8F773FF08BD74
:1005200010B584B0144649BB0DF10D0300930DF1D5
:100530000E0001904FF0000001460DF10A020DF18E
:100540000B03F4F71BFD4FF000018DF80C109DF824
:100550000B201AB14FF001038DF80C309DF80A0002
:1005600028B19DF80C1041F002028DF80C204FF0DC
:1005700000008DF80F00039B236001E04FF0140092
:1005800004B010BD70B514468AB199B94FF000009F
:1005900001460246F4F76AFD06462578F4F74AFE5E
:1005A00085420AD2735D23704FF0000070BD4FF09A
:1005B000160070BD4FF0140070BD4FF0160070BDF6
:1005C000F8B515461F464FF000033B70A9B992F8E5
:1005D000FB0060B14FF000042646285D3146F4F779
:1005E0003FFC04F1010495F8FB20A242F5D84FF03E
:1005F000010139704FF00000F8BD4FF01400F8BD54
:1006000010B586B04FF001041C70F1B945F20C53DF
:10061000C2F20003197845F20D50C2F200000378CF
:1006200002AC00944FF01000019010461A464FF0B3
:100630000103F9F76BFC4AF64850C0F60100214669
:1006400007F06EFD4FF0000004E04FF000021A705A
:100650004FF0140006B010BD2DE9F04115461C46C0
:100660004FF00103237004297CD8DFE801F0030B6D
:100670007B1B640068782978F4F7E8FC4FF00000F1
:10068000BDE8F081287845F20C51C2F200010870F3
:100690006A7845F20D53C2F200031A704FF0000061
:1006A000BDE8F0812C786D7805F1040546F26761AC
:1006B000C6F2666181FB05234FEA630202EB82000A
:1006C00010F0FF0555D04FF00007A5F1050808F020
:1006D0000108042C94BF2646052630463946F4F717
:1006E000BFFBA41BE4B2A5F1050515F0FF0544D13D
:1006F0001DE0042C94BF2646052630463946F4F703
:10070000AFFBA31BA5F1050505F0FF0503F0FF04F2
:10071000042C94BF2646052630463946F4F7A0FB44
:10072000A21BD4B2A5F1050515F0FF05E1D14FF0EC
:100730000000BDE8F0812E78F4F77CFD864206D3F8
:100740004FF0000020704FF01600BDE8F0813046F9
:1007500005F101014FF00102F4F7A4FC4FF0000095
:10076000BDE8F0814FF0000020704FF01400BDE8AC
:10077000F0814FF00000BDE8F0814FFA88F6002EBE
:10078000B7D0042C94BF2646052630463946F4F7E8
:1007900067FBA11BCCB2A5F1050515F0FF05A8D19B
:1007A000C5E700BF10B51C464FF0010323700529B3
:1007B00041D8DFE801F0030E18222C361046F4F77A
:1007C0000DFC00283DD14FF0000020704FF01600C6
:1007D00010BD4AF6E440C0F60100114607F0A0FC47
:1007E0004FF0000010BD4AF6DC40C0F60100114693
:1007F00007F096FC4FF0000010BD4AF6D840C0F656
:100800000100114607F08CFC4FF0000010BD4AF6C5
:10081000D040C0F60100114607F082FC4FF0000006
:1008200010BD4AF6C840C0F60100114607F078FC3A
:100830004FF0000010BD4FF0000121704FF0140088
:1008400010BD4FF0000010BD08B5012805D00228EA
:1008500014BF00220122114603E04FF000024FF0C6
:1008600001014FF00100F4F7C3FC08BD08B54FF0DB
:100870000103137001F1FF31032921D8DFE801F0F2
:10088000020B12194AF64040C0F6010007F048FC7E
:100890004FF0000008BD4FF00000FFF7D5FF4FF00C
:1008A000000008BD4FF00100FFF7CEFF4FF0000041
:1008B00008BD4FF00200FFF7C7FF4FF0000008BD72
:1008C0004FF0000010704FF0140008BD08B5F4F7A9
:1008D000A9FC4FF001004FF000010A46F4F788FC34
:1008E000F4F7ACFC4FF00C004FF00001F4F7B8FA4D
:1008F000F4F798FC08BD00BF037B13B9437B13B921
:100900000EE0994208D301F1FF318A18437B9A42E5
:100910008CBF0020012001E04FF00000C0B2704702
:100920004FF00100704700BF70B4447A24B14FF01B
:10093000320606FB04F610E0C5784AF2D014C0F681
:10094000010454F82550B5F5964F9DBF49F26466F1
:10095000B6FBF5F606EB86060826847A24B14FF03E
:10096000320505FB04F501E041F28835C07A18B183
:10097000FF2808BF012001E04FF0010001B10E6027
:1009800002B1156003B1186070BC704741F618736E
:10099000C2F200034FF4117202FB00304FF000016D
:1009A000C0F810124FF6FF73C0F82C32C0F81812BE
:1009B000704700BFF8B505460E4641F61874C2F2FE
:1009C00000044FF4117303FB0044D4F8240200EB3D
:1009D0005007F5F719FED4F82812421A974202D9A7
:1009E000B81AF5F797F923689A6928464FF001017C
:1009F000904741F61870C2F200004FF4117101FBEC
:100A000005014FF6FF7001F104013246F7F7D6F801
:100A1000A31918714FEA10225A7106F10206C4F8A0
:100A200004614FF00000C4F8080121680B6A2846F1
:100A30009847F4F7A7FF2846FFF7A8FFF8BD00BFC7
:100A400030B583B041F61874C2F200044FF411754A
:100A500005FB0040D0F83002B1F57A7F1BD3A1F539
:100A60007A7163B1837B13B9C37B13B907E09942F1
:100A700024D38A1802F1FF32C07B824221D8C8B247
:100A80000DF10701F8F728FE9DF80710D1F10100DC
:100A900038BF00201AE04FEAD10402F107024FEA02
:100AA000D20523B121462A46FFF726FF60B1281957
:100AB000B0F5805F2CBF0020012007E04FF0000060
:100AC00004E04FF0000001E04FF0000003B030BD43
:100AD00008B5B0F57A7F21D279B14FEAD00340F65C
:100AE000D862C2F2000200F007004FF0010101FAE3
:100AF00000F0D15C0843D05408BD4FEAD00340F663
:100B0000D862C2F2000200F007004FF0010101FAC2
:100B100000F0D15C21EA0000D05408BD00F11800BB
:100B2000C0B24FF00102F8F74FFE08BD10B541F614
:100B30001874C2F200044FF4117303FB0044D4F89C
:100B40001C02F5F793F94FF00000C4F81C0210BD29
:100B500038B54FF4117101FB00F141F61872C2F281
:100B600000028C18D4F80831D4F80451AB420BD0F1
:100B70008958E3188A6A1979904728B1D4F808018E
:100B800000F10100C4F8080138BD00BF08B541F606
:100B90001873C2F200034FF4117202FB0031D1F856
:100BA000082101F10401D1F800319A420BD141F63C
:100BB0001871C2F200014FF4117202FB0010D0F85C
:100BC0001C02F4F711FF08BD70B582B005468DF820
:100BD000071041F61874C2F200044FF4117303FBBE
:100BE0000044D4F81802002850D11AB12846FFF763
:100BF000CDFE4BE0F5F708FDD4F82812431AC4F8EF
:100C00002802D4F81002D4F82422934204D800F128
:100C10000103B3F5807F04D12846FFF7B7FE4FF0FC
:100C20000103D4F81012621802A911F8010D82F81C
:100C30001001C4F81032B4F82C024FF00102F6F79C
:100C4000BDFFC4F82C0208BB04F5887694F8203266
:100C5000012B03D1304602F033FA38B994F8201250
:100C6000022913D1304600F041FD78B14FF0010266
:100C7000C4F8182241F61870C2F200004FF4117344
:100C800003FB0505D5F81C02F4F7AEFE02B070BDFB
:100C9000836B45F21452C2F200021360016C45F2FC
:100CA0001053C2F200031960C16B40F2FC12C2F291
:100CB000000211604FF0000383630364C363704755
:100CC00045F21453C2F200031968816345F21052D1
:100CD000C2F200021368036440F2FC11C2F2000188
:100CE0000A68C263704700BF2DE9F041804617468D
:100CF0001E4642F63C14C2F20004656BAD6808461D
:100D00002146FFF745FA002840D1606B0468002CAB
:100D100031D0616800292ED042F63C14C2F20004A2
:100D20002046FFF7B5FF204650F8342F13685C6863
:100D300041463A463346A04770B142F63C14C2F2EF
:100D400000042046FFF7BCFF28462146FFF720FAA3
:100D50004FF00000BDE8F08142F63C14C2F20004FE
:100D60002046FFF7ADFF28462146FFF711FA4FF066
:100D70000100BDE8F081284642F63C11C2F20001B4
:100D8000FFF706FA4FF00000BDE8F0814FF00000D9
:100D9000BDE8F081F0B583B00D461E46ADF80620E3
:100DA00041F61872C2F200024FF4117101FB0020EB
:100DB000D0F83002037BFF2B03D1427BFF2A00F0E7
:100DC000B5802C68B4F57A7F18D221464FF0020224
:100DD000FFF792FD002800F0AC80002E40F0AC80C0
:100DE00040F6D861C2F20001BDF8062062522868C0
:100DF00000F1020028604FF00100AEE0A4F57A7720
:100E0000B7F57A7F1AD239464FF00102FFF774FD29
:100E1000002800F09480002E40F09480BDF8062059
:100E20004FEA122140F6D860C2F20000C1552B688B
:100E300003F101032B604FF001008EE0A4F6B831FE
:100E4000B1F5FA6F1CD204F10044A4F6B8344FEAAD
:100E500044014FF00202FFF74FFD002875D0002E2D
:100E600076D140F6D861C2F20001BDF8060021F843
:100E700014002B6803F101032B604FF001006CE0BC
:100E8000A4F5BB50A0F11000B0F57A7F0FD24EF65A
:100E90009003C7F6FF73E2184FEA42004FF00101DA
:100EA0000DF106024FF00203FFF71EFF55E0A4F517
:100EB000DA53A3F11803B3F57A7F0ED24EF2A841AC
:100EC000C7F6FF7160184FEA40004FF002010DF1C4
:100ED00006020B46FFF708FF3FE0A4F5FA52B2F511
:100EE0007A7F0CD24FEA4402A2F57A504FF0030108
:100EF0000DF106024FF00203FFF7F6FE2DE0A4F518
:100F00000C51A1F12801B1F57A7F24D24DF6D840D9
:100F1000C7F6FF7023184FEA43004FF004010DF1AC
:100F200006024FF00203FFF7DFFE16E04FF000006D
:100F300013E04FF0000010E04FF001000DE04FF023
:100F400000000AE04FF0010007E04FF0000004E06D
:100F50004FF0010001E04FF0000003B0F0BD00BF12
:100F60002DE9F04182B0804617461D464FF0000340
:100F7000ADF8063042F63C14C2F20004606B86689D
:100F800008462146FFF704F938B1002D42D04FF052
:100F900001032B704FF000003EE042F63C11C2F21C
:100FA00000014A6B13683BB3186828B342F63C143F
:100FB000C2F200042046FFF76BFE204650F8342FA3
:100FC00013681C6841460DF106024FF00203A0476A
:100FD00018B115B14FF001002870012F05D19DF80F
:100FE00006104FEA0122ADF8062042F63C10C2F28C
:100FF0000000FFF765FE03E015B14FF00101297015
:10100000304642F63C11C2F20001FFF7C1F8BDF8CC
:10101000060001E04FF0000002B0BDE8F08100BF23
:1010200010B504460B4611B14FF000020A70226859
:10103000B2F57A7F08D240F6D860C2F20000105AAA
:1010400002F10202226010BDA2F57A71B1F57A7F39
:101050000AD240F6D863C2F20003595C4FEA01207D
:1010600002F10102226010BDA2F5FA60262811D813
:101070004FF0000001460246F3F7F8FF2368A3F59E
:10108000FA6281184978805C40EA012003F102038A
:10109000236010BDA2F6B831B1F5FA6F0DD202F19E
:1010A0000041A1F6B83040F6D863C2F2000333F82D
:1010B000100002F10102226010BDA2F59C50A0F1C7
:1010C0000800B0F57A7F11D24EF67841C7F6FF716D
:1010D00050184FEA40004FF000014FF00202FFF7B6
:1010E0003FFF236803F10103236010BDA2F5BB514C
:1010F000A1F11001B1F57A7F11D24EF69001C7F639
:10110000FF7150184FEA40004FF001014FF002020A
:10111000FFF726FF226802F10102226010BDA2F54E
:10112000DA50A0F11800B0F57A7F10D24EF2A84044
:10113000C7F6FF7012184FEA42004FF002010A464C
:10114000FFF70EFF236803F10103236010BDA2F532
:10115000FA51B1F57A7F0ED24FEA4202A2F57A50E7
:101160004FF003014FF00202FFF7FAFE216801F190
:101170000101216010BDA2F50C50A0F12800B0F5CE
:101180007A7F11D24DF6D841C7F6FF7150184FEA59
:1011900040004FF004014FF00202FFF7E1FE236828
:1011A00003F10103236010BD2BB14FF001021A704F
:1011B0004FF0000010BD4FF0000010BD30B583B0FF
:1011C00004460D4602A840F8084D68460DF1070197
:1011D000FFF726FF9DF8073083B904F1FF34651946
:1011E00002A941F8085D68460DF10701FFF718FFF5
:1011F0009DF80720101C18BF012001E04FF00100EE
:1012000003B030BDF0B583B004464FF000038DF855
:101210000730B0F5805F07D240F6D862C2F2000214
:10122000135C8DF807303CE0A0F5FA60262806D85C
:101230000B19A3F5FA6001788DF8071031E045F23B
:101240001951C2F200010A785AB342F63C15C2F2B3
:1012500000056E6BB6684FF002002946FEF798FF56
:101260006B6B1868B0B10168A1B142F63C15C2F2CF
:1012700000052846FFF70CFD284650F8347F3A68F1
:10128000176821460DF107024FF00103B8472846C1
:10129000FFF716FD304642F63C11C2F20001FEF7A0
:1012A00077FF9DF8070003B0F0BD00BFF0B583B035
:1012B00004464FF00003ADF80630B0F5805F07D26A
:1012C00040F6D863C2F20003C05AADF806003EE013
:1012D000A0F5FA60262808D804460B185878095D4E
:1012E00041EA0022ADF8062031E045F21951C2F280
:1012F00000010A785AB342F63C15C2F200056E6B43
:10130000B6684FF002002946FEF742FF6B6B186883
:10131000B0B10168A1B142F63C15C2F20005284601
:10132000FFF7B6FC284650F8347F3A681768214624
:101330000DF106024FF00203B8472846FFF7C0FC44
:10134000304642F63C11C2F20001FEF721FFBDF823
:10135000060003B0F0BD00BFF0B583B004468DF8C1
:101360000710B0F5805F08D2CAB240F6D863C2F267
:1013700000031A544FF001043DE045F21953C2F244
:1013800000031878002834D042F63C15C2F200055C
:10139000696B8E684FF002002946FEF7F9FE6A6B12
:1013A0001368CBB15868D0B142F63C15C2F20005C3
:1013B0002846FFF76DFC284650F8347F39684F689F
:1013C00021460DF107024FF00103B8472846FFF709
:1013D00077FC4FF0010404E04FF0000401E04FF00F
:1013E0000004304642F63C11C2F20001FEF7D0FE86
:1013F00001E04FF00004204603B0F0BDF0B583B02B
:101400000446ADF80610B0F5805F08D240F6D86308
:10141000C2F200038AB2C2524FF001043DE045F22D
:101420001953C2F200031878002834D042F63C1554
:10143000C2F20005696B8E684FF002002946FEF784
:10144000A7FE6A6B1368CBB15868D0B142F63C1561
:10145000C2F200052846FFF71BFC284650F8347FEF
:1014600039684F6821460DF106024FF00203B84774
:101470002846FFF725FC4FF0010404E04FF000047C
:1014800001E04FF00004304642F63C11C2F2000188
:10149000FEF77EFE01E04FF00004204603B0F0BDF1
:1014A00010B545F21A53C2F200031B78032B47D83C
:1014B00041F61872C2F200024FF4117101FB0323CE
:1014C00040F2CC72C2F2000252E8001F01F10101A9
:1014D00042E80014012CF7D018B14FF00100C3F816
:1014E0003C0245F21854C2F200044FF00101217091
:1014F000D3F840221AB1D3F81C02F4F775FA40F27F
:10150000CC73C2F2000353E8002FA2F1010243E8BA
:101510000024012CF7D053E8002FB2F1004F0DD179
:101520004FF0000243E80024012CF4D04EF60450A2
:10153000CEF20000016841F080510160BFF32F8FAF
:1015400010BD00BF10B545F21A53C2F200034FF0B0
:1015500004041C70FFF7EAFA10BD00BF2DE9F04F3C
:101560008BB005460E4691F8029009EB49094AF204
:101570000478C0F6010809EB080308934FF4117BC7
:101580000BFB00FB41F6187AC2F2000A0BEB0A04CF
:1015900042F63C17C2F20007796B8A6809924FF055
:1015A0000201F8F755FE45F21A50C2F2000005702C
:1015B000C4F83062304604F5097104F50D7204F583
:1015C0000E73FFF7B1F92846FFF7E0F9F5F71CF8BD
:1015D000C4F828024FF0010300934AF68050C0F689
:1015E00001004FF0040141F65112C0F601022B46F2
:1015F000F4F746FBC4F81C025BF80A40F6784AF29E
:10160000D011C0F6010151F8261019F808200898E9
:101610004378867800964FF00000019040F65136EE
:10162000C0F60106029640F68D36C0F60106039616
:1016300040F6C936C0F60106049641F24556C0F69A
:1016400001060596069064682846A0474FF0020000
:101650003946FEF79DFD38B145F21951C2F200013D
:101660004FF00000087006E045F21953C2F2000383
:101670004FF001021A70099842F63C11C2F20001C3
:10168000FEF786FD0BB0BDE8F08F00BF08B545F250
:101690001C53C2F2000318604FF00100FFF700FF77
:1016A00008BD00BF45F21853C2F200034FF000021C
:1016B0001A70704708B545F21C53C2F2000318684F
:1016C00068B145F21A51C2F200010A78032A09D81A
:1016D0004FF00000FFF7E4FE4FF0000008BD4FF0B0
:1016E000480008BD4FF0480008BD00BF10B4D0F856
:1016F0000031032B20D94278102A20D890F90140DC
:101700004FF0010101FA04F448F2600261F31F4254
:1017100014420CD114F00E0F11D0052B12D9807881
:1017200000F10500834214BF002001200CE0082BCB
:1017300014BF0020012007E04FF0000004E04FF04C
:10174000010001E04FF0000010BC7047072814D8DA
:1017500040B24FF0010303FA00F111F00A0F0FD16C
:1017600011F0050F03D111F0F00F03D105E04FF098
:10177000010070474FF0040070474FF000007047C1
:101780004FF00200704700BF2DE9F04F2DED028BA6
:1017900087B006460F4615461C464FF0000001462E
:1017A0000246F3F763FC83462846FFF7CFFF8046E7
:1017B000002800F0C180042805D04FF00100002F60
:1017C00000F0BF8003E017F0010FF6D0B7E045F25C
:1017D0001953C2F20003019342F63C1AC2F2000A06
:1017E0009FED5A8A0AF134020392A5F104000328FE
:1017F0003DD8B6F5805F08D240F6D863C2F2000348
:10180000F058F6F76BFA814631E001990B7873B323
:10181000DAF83420906802908DED058A4FF00200CE
:101820005146FEF7B5FCDAF834100B68DBB15A68A4
:10183000CAB15046FFF72CFADAF834000168D1F843
:1018400000C00398314605AA4FF00403E047DDEDE0
:10185000057ABCEEE70A10EE100AF6F73FFA814669
:101860005046FFF72DFA02985146FEF791FC072DDE
:1018700059D8DFE805F004140E1A24363F473046E5
:101880005946FFF7BFFC4FEA002141EA10222280AF
:1018900049E030465946FFF7B5FC208043E030462A
:1018A0005946FFF703FD20803DE030465946FFF7DB
:1018B000FDFC4FEA102343EA0020208033E04FEA8A
:1018C00019434FEA132040EA0322234623F8022B50
:1018D0001FFA89F04FEA102141EA002262801C467B
:1018E00021E0C9F30F42214621F8022BA4F802900F
:1018F0000C4618E0234623F8029BC9F30F40608092
:101900001C4610E01FFA89F04FEA102242EA00213B
:10191000234623F8021B4FEA19404FEA102242EAFD
:10192000002161801C46464404F10204013F7FF41B
:101930005CAF4FF0010004E04FF0000001E04FF019
:10194000000007B0BDEC028BBDE8F08F0000000086
:101950002DE9F04F8FB05FFA80FA41F61873C2F2AA
:1019600000034FF4117202FB0A394FF0000B02FB27
:101970000AF1029101F5887441F61875C2F200056A
:101980000395661901960CE0D9F80050AE695046EF
:101990004FF00001B0474FF00100C9F84002F3F7E3
:1019A000F1FF45F21857C2F200073B78002BEBD04D
:1019B00045F21C52C2F2000210680028E4D04FF039
:1019C0000001C9F840125C46D34600F083BCD9F848
:1019D0003C7247B14FF00004C9F83C4245F21C5339
:1019E000C2F200031C682278062A00F0D38007D8D0
:1019F000042A76D8032A45D2002A00F0378211E063
:101A0000802A00F0118206D80F2A00F0FB80102AED
:101A100040F02C82B7E1812A00F01F82822A40F038
:101A2000258210E22679B4F8051006F1FF35B5F5E8
:101A3000FA6F1FD24FEA112040EA012715FA87F307
:101A4000B3F5004F05D345F21952C2F200021178E6
:101A500099B1029D03982F1807F1040362783A7137
:101A60002178597065885D804FEA06269E804FF088
:101A7000060104E04FF0FF3101E04FF0FF314FF07D
:101A80000707EEE12779B4F8052007F1FF33FC2BB7
:101A90001FD84FEA122040EA022113FA81F5B5F56A
:101AA000805F05D345F21956C2F2000632789AB12A
:101AB000029B0398191801F1040566780E712278CB
:101AC0006A7063886B804FEA0727AF804FF006018A
:101AD00004E04FF0FF3101E04FF0FF314FF0080715
:101AE000BFE1029903980A1802F10405A3884FEA9E
:101AF000132646EA0327B9B201F007004FF00107A9
:101B000007FA00F74FEAD106B6F5805FC0F0088407
:101B100045F21953C2F200031978002940F0E68318
:101B200033E013680BB342F63C18C2F2000840469B
:101B3000FFF7AEF8404650F8341F0A68D2F800C0EC
:101B400031460DAA4FF00203E04740B9BDF83460BA
:101B50003E40002E14BF4FF47F470027AF8042F66F
:101B60003C10C2F20000FFF7ABF8504642F63C11C1
:101B7000C2F20001FEF70CFBA8884FEA102343EAEB
:101B80000021A9804FF0060101E04FF0FF314FF036
:101B9000060766E1A079FFF7D9FDA788014648B39B
:101BA0004FEA172646EA0725AAB202F1FF3043188A
:101BB000B3F5805F05D345F21957C2F200073978B3
:101BC000D9B1029E039D771907F10403607838713B
:101BD0002178597066885E8010464FF00101A27925
:101BE00003F10403FFF7D0FD002814BF06214FF0D6
:101BF000FF3104E04FF0FF3101E04FF0FF314FF0D3
:101C000007072EE123799A46B4F8051003F1FF3255
:101C1000B2F5F66F80F0AF804FEA112646EA012058
:101C200087B24FEAD705A918B1F5805F07D345F20F
:101C30001952C2F200021678002E00F09F8002991D
:101C400003980E1806F1040204926178317122782B
:101C500004984270618841804FEA0322828003F138
:101C600007014FEAD102827106F10B000690002BAA
